:100000000C944C2E0C947D2E0C947D2E0C947D2EF5
:100010000C947D2E0C947D2E0C947D2E0C947D2EB4
:100020000C947D2E0C947D2E0C947D2E0C947D2EA4
:100030000C947D2E0C947D2E0C947D2E0C947D2E94
:100040000C947D2E0C94078B0C947D2E0C947D2E9D
:100050000C947D2E0C947D2E0C947CF60D94C4345F
:100060000C947D2E0C94E6690C94DC690C947D2E26
:100070000C947D2E0C947D2E0C947D2E0C947D2E54
:100080000C947D2E0C947D2E0C947D2E0C947D2E44
:100090000C947D2E0C947D2E0C947D2E0C947D2E34
:1000A0000C947D2E0C947D2E0C947D2E0C947D2E24
:1000B0000C947D2E0C947D2E0C947D2E0C947D2E14
:1000C0000C947D2E0C947D2E0C947D2E0C948B6CB8
:1000D0000C94616C0C947D2E0C947D2E0C947D2ED2
:1000E0000C947D2E2C30723078309F30AC30B5308F
:1000F000C030C038DB39B33AE53AB546B546FD3BCA
:10010000723CA839B546B546093EA43FDC3FB5462A
:10011000DA41B546B5462B43B546B546B843C2436A
:10012000B546A2445D45EB3FF33F17403B406F406F
:10013000124126413341474154416D41196A1F6ABA
:10014000316A416A496A766A4D6A766A516A556AC5
:10015000766A596A5D6A616A696A766A736A1D9F1E
:10016000249FA19FA69FFFA004A114A131028F018B
:100170008B01CB016B02ED019B016102EB012502BA
:10018000BF01690141022302ED01390211023B0264
:100190002F021B028D01B501D501FB017701B901C9
:1001A000E9015702CD01F501FF01DF01FB01A501C6
:1001B000AB01450221020B02430217025102A901C1
:1001C0003F02D701E3019501C10187014F020702F8
:1001D000A901C301E501D90159021F0291012D02B4
:1001E0007B01EF016302B1015302F101F901470202
:1001F00055020F02EF01BB0167019301084AD73B8B
:100200003BCE016E84BCBFFDC12F3D6C74319ABDE5
:1002100056833DDA3D00C77F11BED9E4BB4C3E9109
:100220006BAAAABE000000803F05A84CCDB2D44EF8
:10023000B93836A9020C50B9918688083CA6AAAAFA
:100240002ABE000000803F07634236B79BD8A71A3A
:1002500039685618AEBAAB558C1D3CB7CC5763BD48
:100260006DEDFD753EF6177231BF000000803F084E
:10027000000000BE922449123EABAAAA2ABECDCCF1
:10028000CC4C3E00000080BEABAAAAAA3E000000F3
:1002900000BF000000803F0000000000084178D34C
:1002A000BB4387D1133D190E3CC3BD4282AD2B3EEB
:1002B00068EC8276BED98FE1A93E4C80EFFFBE018B
:1002C000C4FF7F3F0000000000000C9414A10D94B7
:1002D00042340D942E2B0C94696A0C94249F0C9438
:1002E000DC3F0C94496A0C94DB390C94416A0D9400
:1002F0003F2C0C9454410D94DD330C94B33A0C9480
:10030000736A0C94556A0C942D6B0C94EB3F0D940E
:1003100025310C94596A0D94132B0D94D02B0D9408
:100320000F2B0D94C9330D944C340D941B310C9448
:10033000DA410C9447410D941D2B0C942B430C94E3
:100340005D6A0C94C0300C94A43F0D94632D0C9402
:1003500033410D9440310D94882D0C94A8390C94A0
:10036000FFA00D94EF330C94736B0D94F52B0C944C
:100370005D450D94622C0D9438340C94093E0D9417
:100380002A2B0D941F310D9433310C943B400C9467
:10039000A69F0C9472300D94162B0D94CF2C0C94B8
:1003A000A2440D949B430C9478300D941A2C0D9418
:1003B00011310D943B310C94196A0C94DC6A0D9444
:1003C0003E2D0C942C300D9417310D9437310D9433
:1003D000F6420D94852C0D94242B0D94432B0D94F3
:1003E00056340D9401340C946D410D94F42C0C94FE
:1003F0006F400D940B340D94D12D0C94C0380D9496
:10040000192D0C9412410C941D9F0C9404A10D9471
:100410002D310C949F300D9409310C94766A0D9413
:100420002E340D943B2B0C94B8430C94B5460D948C
:10043000FC300C94C06B0D94B02B0C94E53A0D94E9
:10044000C4330D9406310D94342B0D94272B0C944A
:100450000A6B0C94A19F0C94B5300D94D3330D947A
:100460008E2B0D940C2B0C94723C0C94C2430C9468
:10047000FD3B0D94382B0D943E2B0C94196B0D9471
:100480000D310D94312B0D94F8300D94AD2D0D944C
:1004900015340C941F6A0C94AC300C94316A0D9492
:1004A00029310D9402310D94F7330D9424340D94B9
:1004B000AA2C0D94BF330C94F33F0C944D6A0C940A
:1004C000616A0D94202B0D94E7330C94516A0C94BF
:1004D00026410C9417400D94192B0C943B6B4E4104
:1004E0004E494E495459494E46CDCCCC3D0AD723AE
:1004F0003C17B7D13877CC2B329595E6241FB14FF6
:100500000A000020410000C84200401C4620BCBE3A
:100510004CCA1B0E5AAEC59D7400407A10F35A00A7
:10052000A0724E18090010A5D4E80000E87648171C
:100530000000E40B54020000CA9A3B000000E1F501
:1005400005000080969800000040420F000000A0C7
:100550008601000000102700000000E803000000F2
:10056000006400000000000A00000000000100001C
:100570000000002C76D888DC674F0823DFC1DFAE8F
:1005800059E1B1B796E5E3E453C63AE65199769658
:10059000E8E6C28426EB898C9B62ED407C6FFCEF21
:1005A000BC9C9F40F2BAA56FA5F490055A2AF75C4F
:1005B000936B6CF9676DC11BFCE0E40D47FEF52001
:1005C000E6B500D0ED902E030094357705008084C9
:1005D0001E080000204E0A000000C80C33333333DD
:1005E0000F986E12831141EF8D2114893BE6551649
:1005F000CFFEE6DB18D1844B381BF77C1D901DA481
:10060000BBE424203284725E228100C9F124ECA173
:10061000E53D274D323520500A4D32340050726985
:100620006E742050617573656400526573756D65F5
:10063000005549205061757365004E6F204D6174FF
:100640006368203A004D3837365031004D38373620
:100650005031000A202A2A2A7265636461742E646C
:100660006174615B305D203D004732380A473120BC
:100670004631303030205A313000556E737570700D
:100680006F72746564204F7074696F6E2053656C6F
:100690006563746564004D3139305335350A47322E
:1006A000380A47323950310A47323950330A4D310E
:1006B0003039533231350A47323953310A473239EA
:1006C00053300A47323946302E300A473239410A10
:1006D0004732380A4731583135305931353046358F
:1006E0003030300A47315A300A4D3530300A4D34F7
:1006F00030300A4D31313720536574205A204F660F
:1007000066736574004731204631303030205A30EE
:100710002E30004732380A47312046313030302001
:100720005A302E30004D353030004D3530300047D6
:1007300032385A0A473146313530305A302E30007F
:100740004732380A473146313530305A302E300082
:100750004D383400473146313030305A302E300079
:100760004732380A473146313030305A302E300067
:100770004D353030004D383400426567696E53772F
:1007800069746368007265636461742E6164647285
:10079000203D3D007265636461742E646174615B29
:1007A000305D203D3D0077616974776179203D3D82
:1007B000000A202A2A2A4E6F7A7A6C6554656D7079
:1007C0005374617475735B325D203D00434F4D4D32
:1007D000554E49434154494F4E0044525952554E8B
:1007E000004552524F525300494E464F0045434830
:1007F0004F0047322F47332062616420706172617D
:100800006D65746572730A00536C6565702E2E2ECB
:1008100000486F6D652058592046697273740A004C
:10082000486F6D6520585920466972737400205ACC
:100830003A200020593A200042656420583A2000AE
:100840004D65736820706F696E742063616E6E6FA2
:1008500074206265207265736F6C7665640A004D62
:10086000302F3120427265616B2043616C6C65648E
:1008700000436F6E74696E7565004D302F312042F4
:100880007265616B2043616C6C6564004E6F204D36
:100890006F76652E00456E642066696C65206C6914
:1008A00073740A00426567696E2066696C65206C26
:1008B0006973740A00526573756D6520534400288E
:1008C0006E6F2066696C65290043757272656E747F
:1008D0002066696C653A20002E0A0044656C6574D8
:1008E000696F6E206661696C65642C2046696C6571
:1008F0003A200046696C652064656C657465643AED
:10090000005072696E742074696D653A20000A5354
:10091000746174733A2046696C616D656E742075FC
:100920007365643A20002C204C6F6E6765737420E9
:100930006A6F623A2000546F74616C2074696D654F
:100940003A200053746174733A20002C2046616988
:100950006C65643A20002C2046696E697368656492
:100960003A20005072696E74733A200053746174B7
:10097000733A20004520436F6F6C696E672E2E2EF0
:1009800000452048656174696E672E2E2E006F66E3
:100990006600ED07E807E107DA07CC074445425552
:1009A000473A004D31313320530042656420436F94
:1009B0006F6C696E672E2E2E00426564204865615B
:1009C00074696E672E2E2E006F6B004348414D42B6
:1009D00045525F54454D5045524154555245004D86
:1009E0004F54494F4E5F4D4F444553005448455274
:1009F0004D414C5F50524F54454354494F4E004176
:100A000055544F5245504F52545F53445F535441D5
:100A10005455530050524F4D50545F535550504F02
:100A2000525400454D455247454E43595F5041523F
:100A300053455200434153455F4C494748545F4238
:100A400052494748544E45535300544F47474C452D
:100A50005F4C494748545300534F46545741524501
:100A60005F504F574552004255494C445F504552E4
:100A700043454E54004C4556454C494E475F444112
:100A80005441005A5F50524F4245004155544F4C1B
:100A90004556454C005052494E545F4A4F42005013
:100AA000524F4752455353004155544F5245504FB2
:100AB00052545F54454D5000564F4C554D4554527D
:100AC000494300454550524F4D0042494E4152590D
:100AD0005F46494C455F5452414E53464552005380
:100AE000455249414C5F584F4E5F584F464600466D
:100AF00049524D574152455F4E414D453A4D617205
:100B00006C696E20322E302E785F4352323942208B
:100B1000544D33442053534D444E5520534F55525A
:100B200043455F434F44455F55524C3A6874747077
:100B3000733A2F2F6769746875622E636F6D2F4942
:100B40006E73616E6974794175746F6D6174696FEC
:100B50006E2F4D61726C696E2F747265652F4372D2
:100B600065616C6974795F4D61726C696E322E30AB
:100B70002E782050524F544F434F4C5F564552539E
:100B8000494F4E3A312E30204D414348494E455F42
:100B9000545950453A544D3344203130532050720B
:100BA0006F2045585452554445525F434F554E545B
:100BB0003A3120555549443A63656465326132667D
:100BC0002D343161322D343734382D396231322DA4
:100BD0006335356336326633363766660A002F2F43
:100BE0002000205400205200416363656C657261EF
:100BF00074696F6E3A2050003F4A206F7574206F01
:100C0000662072616E67652028302E303120746F47
:100C100020302E33290A0020466C6F773A2000508E
:100C2000726F7465637465642050696E0A00507257
:100C30006F6265205A204F66667365743A200049DA
:100C40006E76616C69642065787472756465720A89
:100C50000020643A0020693A0020703A0020643A8B
:100C60000020693A0020703A0064697300656E00E4
:100C700043290A0061626C656420286D696E2074E6
:100C8000656D702000436F6C6420657874727564C4
:100C900065732061726520004F4646004F4E004646
:100CA000696C616D656E742072756E6F7574206409
:100CB000697374616E636520286D6D293A20004662
:100CC000696C616D656E742072756E6F757420004D
:100CD0004F666673657473204170706C696564005B
:100CE0004572723A20546F6F206661722100546F12
:100CF0006F206661722066726F6D20726566657224
:100D0000656E636520706F696E740A0045455052C8
:100D10004F4D204F4B0A003F5A206F7574206F666D
:100D20002072616E676520282D323020746F20326A
:100D300030290A0050726F6265205A204F66667330
:100D400065743A20005072696E7465722073746F16
:100D5000707065642064756520746F206572726FB1
:100D600072732E2046697820746865206572726FF0
:100D70007220616E6420757365204D393939207495
:100D80006F20726573746172742E202854656D70C3
:100D9000657261747572652069732072657365741C
:100DA0002E20536574206974206166746572207208
:100DB000657374617274696E67290A0053544F50E9
:100DC0005045442E200024F404D9201BC40C5C0E92
:100DD0009804C4095F0265077101F405F900FB047A
:100DE000B30048048700C10369005803550003039A
:100DF0004500BE023A008402310053022A00290253
:100E0000250004022000E4011C00C8011900AF0104
:100E10001700980114008401130071011000610192
:100E2000100051010E0043010D0036010B002B0193
:100E30000B0020010B00150109000C010900030142
:100E40000800FB000800F3000800EB000700E400C6
:100E50000600DE000600D8000600D2000600CC0026
:100E60000500C7000500C2000500BD000400B90070
:100E70000400B5000400B1000400AD000400A900A6
:100E80000400A5000300A20003009F0004009B00D3
:100E900003009800030095000200930003009000F7
:100EA00003008D0002008B00030088000200860012
:100EB000020084000300810002007F0002007D0028
:100EC00002007B000200790002007700010076003A
:100ED00002007400020072000100710002006F0045
:100EE00002006D0001006C0002006A000100690050
:100EF0000200670001006600010065000100640057
:100F000002006200010061000100600001005F005A
:100F100002005D0001005C0001005B0001005A005E
:100F2000010059000100580001005700010056005F
:100F3000010055000100540001005300000053005F
:100F400001005200010051000100500001004F005B
:100F500001004E0000004E0001004D0001004C0059
:100F600001004B0000004B0001004A000100490055
:100F70000100480000004800010047000100460051
:100F8000000046000100450000004500010044004B
:100F90000100430000004300010042000000420045
:100FA00001004100000041000100400001003F003D
:100FB00000003F0001003E0000003E0001003D0037
:100FC00000003D0001003C0000003C0000003C002F
:100FD00001003B0000003B0001003A0000003A0025
:100FE000010039000000390001003800000038001D
:100FF0000000380001003700000037000100360013
:101000000000360000003600010035000000350009
:1010100000003500010034000000340000003400FE
:1010200001003300000033000000330001003200F3
:1010300000003200000032000100310000003100E9
:1010400000003100010030000000300000003000DE
:1010500001002F0000002F0000002F0000002F00D3
:1010600001002E0000002E0000002E0001002D00C7
:1010700000002D0000002D0000002D0001002C00BC
:1010800000002C0000002C0000002C0001002B00B0
:1010900000002B0000002B0000002B0001002A00A4
:1010A00000002A0000002A0000002A000100290098
:1010B000000029000000290000002900000029008C
:1010C000010028000000280000002800000028007F
:1010D0000000280001002700000027000000270072
:1010E0000000270000002700010026000000260065
:1010F0000000260000002600000026000100250058
:10110000000025000000250000002500000025004B
:10111000000025000100240000002400000024003D
:101120000000240000002400010023000000230030
:101130000000230000002300000023000000230023
:101140000000230001002200000022000000220015
:101150000000220000002200000022000100210007
:1011600000002100000021000000210000002100FB
:1011700000002100000021000100200000002000EC
:1011800000002000000020000000200000002000DF
:10119000000020000000200001001F0000001F00D0
:1011A00000001F0000001F0000001F0000001F00C3
:1011B00000001F0001001E0000001E0000001E00B5
:1011C00000001E00000024F4D43050C38E20C2A2C0
:1011D0004017828B7011127A910D816CD90AA86127
:1011E000E108C7586607615143061E4B5D05C145BE
:1011F000A7041A411104093D98037139310340369F
:10120000DB0265339102D4305402802E1D02632C20
:10121000EE01752AC501B028A001102781018F2594
:1012200064012B244B01E0223401AC211F018D20ED
:101230000D01801FFC00841EED00971DDF00B81C0F
:10124000D200E61BC600201BBC00641AB200B21913
:10125000A8000A19A0006A189900D1179100401738
:101260008B00B516840031167E00B31579003A154F
:101270007300C7146F0058146A00EE1366008813D9
:10128000630025135E00C7125B006C125700151235
:101290005400C111510070114F0021114B00D610A4
:1012A00049008D1047004610440002104200C00F54
:1012B0004000800F3E00420F3C00060F3B00CB0E6B
:1012C0003800930E37005C0E3500270E3400F30D06
:1012D0003200C10D3100900D3000600D2E00320D36
:1012E0002D00050D2C00D90C2B00AE0C2900850C0F
:1012F00029005C0C2700350C27000E0C2600E80B9B
:101300002400C40B2400A00B23007D0B23005A0BE8
:101310002100390B2100180B2000F80A1F00D90A00
:101320001E00BB0A1E009D0A1D00800A1D00630AE4
:101330001C00470A1B002C0A1B00110A1A00F7099F
:101340001A00DD091900C4091900AB091900920936
:1013500017007B091800630917004C0916003609AD
:101360001600200916000A091500F5081500E00806
:101370001400CC081400B8081400A4081400900845
:1013800013007D0812006B0813005808120046086D
:10139000120034081100230811001208110001087E
:1013A0001100F0071000E0071000D0071000C00780
:1013B0001000B0070F00A107100091070E0083076F
:1013C0000F0074070F0065070E0057070E0049074E
:1013D0000E003B070D002E070E0020070D0013071F
:1013E0000D0006070D00F9060C00ED060D00E006E5
:1013F0000C00D4060C00C8060C00BC060C00B0069D
:101400000C00A4060B0099060C008D060B0082064A
:101410000B0077060B006C060B0061060A005706EE
:101420000B004C060A0042060A0038060A002E0687
:101430000A0024060A001A060A0010060900070618
:101440000A00FD050900F4050900EB050900E205A5
:101450000900D9050900D0050900C7050900BE0526
:101460000900B5050800AD050800A50509009C05A3
:101470000800940508008C050800840508007C0518
:101480000800740508006C050700650508005D0587
:101490000700560508004E050700470507004005F0
:1014A000080038050700310507002A050700230555
:1014B00007001C050600160507000F0507000805B4
:1014C000060002050700FB040600F5040700EE0411
:1014D0000600E8040600E2040700DB040600D50469
:1014E0000600CF040600C9040600C3040600BD04BC
:1014F0000600B7040600B1040500AC040600A6040B
:101500000600A00405009B04060095040500900455
:1015100006008A04050085040500800406007A049C
:10152000050075040500700405006B0405006604E1
:101530000500610405005C04050057040500520421
:1015400005004D04050048040500430405003E0461
:1015500004003A04050035040500300404002C049E
:10156000050027040400230405001E0404001A04D7
:10157000040016040500110404000D04040009040D
:1015800005000404040000040400FC030400F80344
:101590000400F4030400F0030400EC030400E80377
:1015A0000400E4030400E0030400DC030400D803A7
:1015B0000400D4030400D0030400CC030400C803D7
:1015C0000300C5030300726F746174696F6E206D50
:1015D00061747269783A0A0024F404D9201BC40C9F
:1015E0005C0E9804C4095F0265077101F405F900F7
:1015F000FB04B30048048700C10369005803550089
:1016000003034500BE023A008402310053022A005F
:101610002902250004022000E4011C00C801190071
:10162000AF0117009801140084011300710110002C
:101630006101100051010E0043010D0036010B0045
:101640002B010B0020010B00150109000C01090002
:1016500003010800FB000800F3000800EB0007008E
:10166000E4000600DE000600D8000600D2000600F6
:10167000CC000500C7000500C2000500BD00040045
:10168000B9000400B5000400B1000400AD0004007E
:10169000A9000400A5000300A20003009F000400AD
:1016A0009B000300980003009500020093000300D4
:1016B000900003008D0002008B00030088000200F0
:1016C0008600020084000300810002007F00020007
:1016D0007D0002007B00020079000200770001001B
:1016E0007600020074000200720001007100020026
:1016F0006F0002006D0001006C0002006A00010032
:101700006900020067000100660001006500010039
:10171000640002006200010061000100600001003D
:101720005F0002005D0001005C0001005B00010041
:101730005A00010059000100580001005700010043
:101740005600010055000100540001005300000044
:10175000530001005200010051000100500001003F
:101760004F0001004E0000004E0001004D0001003E
:101770004C0001004B0000004B0001004A0001003A
:101780004900010048000000480001004700010036
:101790004600000046000100450000004500010031
:1017A000440001004300000043000100420000002B
:1017B0004200010041000000410001004000010022
:1017C0003F0000003F0001003E0000003E0001001D
:1017D0003D0000003D0001003C0000003C00000016
:1017E0003C0001003B0000003B0001003A0000000B
:1017F0003A00010039000000390001003800000003
:1018000038000000380001003700000037000100F8
:1018100036000000360000003600010035000000F0
:1018200035000000350001003400000034000000E5
:1018300034000100330000003300000033000100D9
:1018400032000000320000003200010031000000D0
:1018500031000000310001003000000030000000C5
:10186000300001002F0000002F0000002F000000BA
:101870002F0001002E0000002E0000002E000100AD
:101880002D0000002D0000002D0000002D000100A3
:101890002C0000002C0000002C0000002C00010097
:1018A0002B0000002B0000002B0000002B0001008B
:1018B0002A0000002A0000002A0000002A0001007F
:1018C0002900000029000000290000002900000074
:1018D0002900010028000000280000002800000066
:1018E0002800000028000100270000002700000059
:1018F000270000002700000027000100260000004C
:10190000260000002600000026000000260001003E
:101910002500000025000000250000002500000033
:101920002500000025000100240000002400000024
:101930002400000024000000240001002300000017
:10194000230000002300000023000000230000000B
:1019500023000000230001002200000022000000FC
:1019600022000000220000002200000022000100EE
:1019700021000000210000002100000021000000E3
:1019800021000000210000002100010020000000D3
:1019900020000000200000002000000020000000C7
:1019A0002000000020000000200001001F000000B7
:1019B0001F0000001F0000001F0000001F000000AB
:1019C0001F0000001F0001001E0000001E0000009C
:1019D0001E0000001E00000024F4D43050C38E20EE
:1019E000C2A24017828B7011127A910D816CD90AB4
:1019F000A861E108C7586607615143061E4B5D05A3
:101A0000C145A7041A411104093D980371393103F6
:101A10004036DB0265339102D4305402802E1D0221
:101A2000632CEE01752AC501B028A00110278101A1
:101A30008F2564012B244B01E0223401AC211F01CE
:101A40008D200D01801FFC00841EED00971DDF001E
:101A5000B81CD200E61BC600201BBC00641AB200F2
:101A6000B219A8000A19A0006A189900D1179100AC
:101A700040178B00B516840031167E00B31579002F
:101A80003A157300C7146F0058146A00EE1366000D
:101A90008813630025135E00C7125B006C125700A9
:101AA00015125400C111510070114F0021114B004B
:101AB000D61049008D104700461044000210420025
:101AC000C00F4000800F3E00420F3C00060F3B005D
:101AD000CB0E3800930E37005C0E3500270E340015
:101AE000F30D3200C10D3100900D3000600D2E005D
:101AF000320D2D00050D2C00D90C2B00AE0C290049
:101B0000850C29005C0C2700350C27000E0C2600E4
:101B1000E80B2400C40B2400A00B23007D0B230042
:101B20005A0B2100390B2100180B2000F80A1F0066
:101B3000D90A1E00BB0A1E009D0A1D00800A1D0056
:101B4000630A1C00470A1B002C0A1B00110A1A001A
:101B5000F7091A00DD091900C4091900AB091900B9
:101B6000920917007B091800630917004C09160039
:101B700036091600200916000A091500F508150097
:101B8000E0081400CC081400B8081400A4081400DD
:101B9000900813007D0812006B081300580812000B
:101BA0004608120034081100230811001208110021
:101BB00001081100F0071000E0071000D007100026
:101BC000C0071000B0070F00A107100091070E001A
:101BD00083070F0074070F0065070E0057070E00FC
:101BE00049070E003B070D002E070E0020070D00D1
:101BF00013070D0006070D00F9060C00ED060D0099
:101C0000E0060C00D4060C00C8060C00BC060C0054
:101C1000B0060C00A4060B0099060C008D060B0004
:101C200082060B0077060B006C060B0061060A00AB
:101C300057060B004C060A0042060A0038060A0046
:101C40002E060A0024060A001A060A0010060900D9
:101C500007060A00FD050900F4050900EB05090067
:101C6000E2050900D9050900D0050900C7050900EA
:101C7000BE050900B5050800AD050800A505090069
:101C80009C050800940508008C05080084050800E0
:101C90007C050800740508006C0507006505080050
:101CA0005D050700560508004E05070047050700BB
:101CB0004005080038050700310507002A05070020
:101CC000230507001C050600160507000F05070081
:101CD0000805060002050700FB040600F5040700DE
:101CE000EE040600E8040600E2040700DB04060038
:101CF000D5040600CF040600C9040600C30406008C
:101D0000BD040600B7040600B1040500AC040600DB
:101D1000A6040600A00405009B0406009504050027
:101D2000900406008A04050085040500800406006E
:101D30007A04050075040500700405006B040500B5
:101D400066040500610405005C04050057040500F5
:101D5000520405004D040500480405004304050035
:101D60003E0404003A040500350405003004040074
:101D70002C04050027040400230405001E040400AD
:101D80001A04040016040500110404000D040400E4
:101D9000090405000404040000040400FC0304001A
:101DA000F8030400F4030400F0030400EC0304004F
:101DB000E8030400E4030400E0030400DC0304007F
:101DC000D8030400D4030400D0030400CC030400AF
:101DD000C8030300C503030024F404D9201BC40C6A
:101DE0005C0E9804C4095F0265077101F405F900EF
:101DF000FB04B30048048700C10369005803550081
:101E000003034500BE023A008402310053022A0057
:101E10002902250004022000E4011C00C801190069
:101E2000AF01170098011400840113007101100024
:101E30006101100051010E0043010D0036010B003D
:101E40002B010B0020010B00150109000C010900FA
:101E500003010800FB000800F3000800EB00070086
:101E6000E4000600DE000600D8000600D2000600EE
:101E7000CC000500C7000500C2000500BD0004003D
:101E8000B9000400B5000400B1000400AD00040076
:101E9000A9000400A5000300A20003009F000400A5
:101EA0009B000300980003009500020093000300CC
:101EB000900003008D0002008B00030088000200E8
:101EC0008600020084000300810002007F000200FF
:101ED0007D0002007B000200790002007700010013
:101EE000760002007400020072000100710002001E
:101EF0006F0002006D0001006C0002006A0001002A
:101F00006900020067000100660001006500010031
:101F10006400020062000100610001006000010035
:101F20005F0002005D0001005C0001005B00010039
:101F30005A0001005900010058000100570001003B
:101F4000560001005500010054000100530000003C
:101F50005300010052000100510001005000010037
:101F60004F0001004E0000004E0001004D00010036
:101F70004C0001004B0000004B0001004A00010032
:101F8000490001004800000048000100470001002E
:101F90004600000046000100450000004500010029
:101FA0004400010043000000430001004200000023
:101FB000420001004100000041000100400001001A
:101FC0003F0000003F0001003E0000003E00010015
:101FD0003D0000003D0001003C0000003C0000000E
:101FE0003C0001003B0000003B0001003A00000003
:101FF0003A000100390000003900010038000000FB
:1020000038000000380001003700000037000100F0
:1020100036000000360000003600010035000000E8
:1020200035000000350001003400000034000000DD
:1020300034000100330000003300000033000100D1
:1020400032000000320000003200010031000000C8
:1020500031000000310001003000000030000000BD
:10206000300001002F0000002F0000002F000000B2
:102070002F0001002E0000002E0000002E000100A5
:102080002D0000002D0000002D0000002D0001009B
:102090002C0000002C0000002C0000002C0001008F
:1020A0002B0000002B0000002B0000002B00010083
:1020B0002A0000002A0000002A0000002A00010077
:1020C000290000002900000029000000290000006C
:1020D000290001002800000028000000280000005E
:1020E0002800000028000100270000002700000051
:1020F0002700000027000000270001002600000044
:102100002600000026000000260000002600010036
:10211000250000002500000025000000250000002B
:10212000250000002500010024000000240000001C
:10213000240000002400000024000100230000000F
:102140002300000023000000230000002300000003
:1021500023000000230001002200000022000000F4
:1021600022000000220000002200000022000100E6
:1021700021000000210000002100000021000000DB
:1021800021000000210000002100010020000000CB
:1021900020000000200000002000000020000000BF
:1021A0002000000020000000200001001F000000AF
:1021B0001F0000001F0000001F0000001F000000A3
:1021C0001F0000001F0001001E0000001E00000094
:1021D0001E0000001E00000024F4D43050C38E20E6
:1021E000C2A24017828B7011127A910D816CD90AAC
:1021F000A861E108C7586607615143061E4B5D059B
:10220000C145A7041A411104093D980371393103EE
:102210004036DB0265339102D4305402802E1D0219
:10222000632CEE01752AC501B028A0011027810199
:102230008F2564012B244B01E0223401AC211F01C6
:102240008D200D01801FFC00841EED00971DDF0016
:10225000B81CD200E61BC600201BBC00641AB200EA
:10226000B219A8000A19A0006A189900D1179100A4
:1022700040178B00B516840031167E00B315790027
:102280003A157300C7146F0058146A00EE13660005
:102290008813630025135E00C7125B006C125700A1
:1022A00015125400C111510070114F0021114B0043
:1022B000D61049008D10470046104400021042001D
:1022C000C00F4000800F3E00420F3C00060F3B0055
:1022D000CB0E3800930E37005C0E3500270E34000D
:1022E000F30D3200C10D3100900D3000600D2E0055
:1022F000320D2D00050D2C00D90C2B00AE0C290041
:10230000850C29005C0C2700350C27000E0C2600DC
:10231000E80B2400C40B2400A00B23007D0B23003A
:102320005A0B2100390B2100180B2000F80A1F005E
:10233000D90A1E00BB0A1E009D0A1D00800A1D004E
:10234000630A1C00470A1B002C0A1B00110A1A0012
:10235000F7091A00DD091900C4091900AB091900B1
:10236000920917007B091800630917004C09160031
:1023700036091600200916000A091500F50815008F
:10238000E0081400CC081400B8081400A4081400D5
:10239000900813007D0812006B0813005808120003
:1023A0004608120034081100230811001208110019
:1023B00001081100F0071000E0071000D00710001E
:1023C000C0071000B0070F00A107100091070E0012
:1023D00083070F0074070F0065070E0057070E00F4
:1023E00049070E003B070D002E070E0020070D00C9
:1023F00013070D0006070D00F9060C00ED060D0091
:10240000E0060C00D4060C00C8060C00BC060C004C
:10241000B0060C00A4060B0099060C008D060B00FC
:1024200082060B0077060B006C060B0061060A00A3
:1024300057060B004C060A0042060A0038060A003E
:102440002E060A0024060A001A060A0010060900D1
:1024500007060A00FD050900F4050900EB0509005F
:10246000E2050900D9050900D0050900C7050900E2
:10247000BE050900B5050800AD050800A505090061
:102480009C050800940508008C05080084050800D8
:102490007C050800740508006C0507006505080048
:1024A0005D050700560508004E05070047050700B3
:1024B0004005080038050700310507002A05070018
:1024C000230507001C050600160507000F05070079
:1024D0000805060002050700FB040600F5040700D6
:1024E000EE040600E8040600E2040700DB04060030
:1024F000D5040600CF040600C9040600C304060084
:10250000BD040600B7040600B1040500AC040600D3
:10251000A6040600A00405009B040600950405001F
:10252000900406008A040500850405008004060066
:102530007A04050075040500700405006B040500AD
:1025400066040500610405005C04050057040500ED
:10255000520405004D04050048040500430405002D
:102560003E0404003A04050035040500300404006C
:102570002C04050027040400230405001E040400A5
:102580001A04040016040500110404000D040400DC
:10259000090405000404040000040400FC03040012
:1025A000F8030400F4030400F0030400EC03040047
:1025B000E8030400E4030400E0030400DC03040077
:1025C000D8030400D4030400D0030400CC030400A7
:1025D000C8030300C503030070012C01900127010B
:1025E000B0012201C0011D01F00118011002130108
:1025F00030020E016002090190020401C002FF00D6
:102600000003FA004003F5008003F000D003EB0064
:102610002004E6007004E100E004DC004005D7007F
:10262000C005D2004006CD00D006C8008007C30018
:102630003008BE00F008B900C009B400B00AAF000D
:10264000B00BAA00D00CA500000EA000500F9B00FC
:10265000C01096005012910000148C00C015870025
:10266000B0178200B0197D00D01B7800001E7300E7
:1026700040206E0090226900F024640040275F0033
:1026800090295A00E02B5500102E500020304B00AE
:1026900010324600E033410090353C0010373700DF
:1026A00070383200A0392D00B03A2800A03B23003A
:1026B000603C1E00103D1900903D1400103E0F00BC
:1026C000703E0A00C03E0500003F0000403FFBFF97
:1026D000803FF6FFC03FF1FF1000C90210012C013E
:1026E0004001220170011801B0010E01F001040146
:1026F0005002FA00B002F0003003E600D003DC0024
:102700009004D2007005C800A006BE000008B40006
:10271000B009AA00D00BA000600E960060118C00DA
:102720000015820020197800C01D6E00A0226400F0
:10273000B0275A00902C500000314600E0343C0095
:1027400010383200903A2800603C1E00A03D140072
:10275000803E0A00203F000024F404D9201BC40C52
:102760005C0E9804C4095F0265077101F405F90065
:10277000FB04B30048048700C103690058035500F7
:1027800003034500BE023A008402310053022A00CE
:102790002902250004022000E4011C00C8011900E0
:1027A000AF0117009801140084011300710110009B
:1027B0006101100051010E0043010D0036010B00B4
:1027C0002B010B0020010B00150109000C01090071
:1027D00003010800FB000800F3000800EB000700FD
:1027E000E4000600DE000600D8000600D200060065
:1027F000CC000500C7000500C2000500BD000400B4
:10280000B9000400B5000400B1000400AD000400EC
:10281000A9000400A5000300A20003009F0004001B
:102820009B00030098000300950002009300030042
:10283000900003008D0002008B000300880002005E
:102840008600020084000300810002007F00020075
:102850007D0002007B000200790002007700010089
:102860007600020074000200720001007100020094
:102870006F0002006D0001006C0002006A000100A0
:1028800069000200670001006600010065000100A8
:1028900064000200620001006100010060000100AC
:1028A0005F0002005D0001005C0001005B000100B0
:1028B0005A000100590001005800010057000100B2
:1028C00056000100550001005400010053000000B3
:1028D00053000100520001005100010050000100AE
:1028E0004F0001004E0000004E0001004D000100AD
:1028F0004C0001004B0000004B0001004A000100A9
:1029000049000100480000004800010047000100A4
:10291000460000004600010045000000450001009F
:102920004400010043000000430001004200000099
:102930004200010041000000410001004000010090
:102940003F0000003F0001003E0000003E0001008B
:102950003D0000003D0001003C0000003C00000084
:102960003C0001003B0000003B0001003A00000079
:102970003A00010039000000390001003800000071
:102980003800000038000100370000003700010067
:10299000360000003600000036000100350000005F
:1029A0003500000035000100340000003400000054
:1029B0003400010033000000330000003300010048
:1029C000320000003200000032000100310000003F
:1029D0003100000031000100300000003000000034
:1029E000300001002F0000002F0000002F00000029
:1029F0002F0001002E0000002E0000002E0001001C
:102A00002D0000002D0000002D0000002D00010011
:102A10002C0000002C0000002C0000002C00010005
:102A20002B0000002B0000002B0000002B000100F9
:102A30002A0000002A0000002A0000002A000100ED
:102A400029000000290000002900000029000000E2
:102A500029000100280000002800000028000000D4
:102A600028000000280001002700000027000000C7
:102A700027000000270000002700010026000000BA
:102A800026000000260000002600000026000100AD
:102A900025000000250000002500000025000000A2
:102AA0002500000025000100240000002400000093
:102AB0002400000024000000240001002300000086
:102AC000230000002300000023000000230000007A
:102AD000230000002300010022000000220000006B
:102AE000220000002200000022000000220001005D
:102AF0002100000021000000210000002100000052
:102B00002100000021000000210001002000000041
:102B10002000000020000000200000002000000035
:102B20002000000020000000200001001F00000025
:102B30001F0000001F0000001F0000001F00000019
:102B40001F0000001F0001001E0000001E0000000A
:102B50001E0000001E00000024F4D43050C38E205C
:102B6000C2A24017828B7011127A910D816CD90A22
:102B7000A861E108C7586607615143061E4B5D0511
:102B8000C145A7041A411104093D98037139310365
:102B90004036DB0265339102D4305402802E1D0290
:102BA000632CEE01752AC501B028A0011027810110
:102BB0008F2564012B244B01E0223401AC211F013D
:102BC0008D200D01801FFC00841EED00971DDF008D
:102BD000B81CD200E61BC600201BBC00641AB20061
:102BE000B219A8000A19A0006A189900D11791001B
:102BF00040178B00B516840031167E00B31579009E
:102C00003A157300C7146F0058146A00EE1366007B
:102C10008813630025135E00C7125B006C12570017
:102C200015125400C111510070114F0021114B00B9
:102C3000D61049008D104700461044000210420093
:102C4000C00F4000800F3E00420F3C00060F3B00CB
:102C5000CB0E3800930E37005C0E3500270E340083
:102C6000F30D3200C10D3100900D3000600D2E00CB
:102C7000320D2D00050D2C00D90C2B00AE0C2900B7
:102C8000850C29005C0C2700350C27000E0C260053
:102C9000E80B2400C40B2400A00B23007D0B2300B1
:102CA0005A0B2100390B2100180B2000F80A1F00D5
:102CB000D90A1E00BB0A1E009D0A1D00800A1D00C5
:102CC000630A1C00470A1B002C0A1B00110A1A0089
:102CD000F7091A00DD091900C4091900AB09190028
:102CE000920917007B091800630917004C091600A8
:102CF00036091600200916000A091500F508150006
:102D0000E0081400CC081400B8081400A40814004B
:102D1000900813007D0812006B0813005808120079
:102D2000460812003408110023081100120811008F
:102D300001081100F0071000E0071000D007100094
:102D4000C0071000B0070F00A107100091070E0088
:102D500083070F0074070F0065070E0057070E006A
:102D600049070E003B070D002E070E0020070D003F
:102D700013070D0006070D00F9060C00ED060D0007
:102D8000E0060C00D4060C00C8060C00BC060C00C3
:102D9000B0060C00A4060B0099060C008D060B0073
:102DA00082060B0077060B006C060B0061060A001A
:102DB00057060B004C060A0042060A0038060A00B5
:102DC0002E060A0024060A001A060A001006090048
:102DD00007060A00FD050900F4050900EB050900D6
:102DE000E2050900D9050900D0050900C705090059
:102DF000BE050900B5050800AD050800A5050900D8
:102E00009C050800940508008C050800840508004E
:102E10007C050800740508006C05070065050800BE
:102E20005D050700560508004E0507004705070029
:102E30004005080038050700310507002A0507008E
:102E4000230507001C050600160507000F050700EF
:102E50000805060002050700FB040600F50407004C
:102E6000EE040600E8040600E2040700DB040600A6
:102E7000D5040600CF040600C9040600C3040600FA
:102E8000BD040600B7040600B1040500AC0406004A
:102E9000A6040600A00405009B0406009504050096
:102EA000900406008A0405008504050080040600DD
:102EB0007A04050075040500700405006B04050024
:102EC00066040500610405005C0405005704050064
:102ED000520405004D0405004804050043040500A4
:102EE0003E0404003A0405003504050030040400E3
:102EF0002C04050027040400230405001E0404001C
:102F00001A04040016040500110404000D04040052
:102F1000090405000404040000040400FC03040088
:102F2000F8030400F4030400F0030400EC030400BD
:102F3000E8030400E4030400E0030400DC030400ED
:102F4000D8030400D4030400D0030400CC0304001D
:102F5000C8030300C5030300256C642E25696D00BA
:102F60004D61726C696E20322E302E785F43523282
:102F7000394200206D61783A00206D696E3A004157
:102F800078697320004572726F7220777269746974
:102F90006E6720746F20454550524F4D210A003610
:102FA0003726033C3D380E2E303E121A1C180844BA
:102FB0000AFF430809070001627573793A207061BE
:102FC0007573656420666F7220696E7075740A008F
:102FD000627573793A2070617573656420666F72EB
:102FE00020757365720A00627573793A2070726F8A
:102FF00063657373696E670A007061757365004D70
:10300000363030200A204D313137200A00206669E1
:103010006C616D656E745F72756E6F75742000669D
:10302000696C616D656E745F72756E6F7574205436
:103030000046696C616D656E7452756E6F757420B3
:1030400054004B494C4C2063617573656420627970
:1030500020746F6F206D75636820696E6163746999
:1030600076652074696D65202D2063757272656EBA
:103070007420636F6D6D616E643A2000706F7765C8
:10308000726F6666004B494C4C45442E20005072CE
:10309000696E7465722068616C7465642E206B695A
:1030A0006C6C28292063616C6C6564210A0065637F
:1030B000686F3A004572726F723A00204A00202011
:1030C0004D343231204900202047323920493939E6
:1030D0000A006163746976650A00696E0000205316
:1030E000797374656D2076312E30312000202050A8
:1030F0006C616E6E65724275666665724279746562
:10310000733A20002046726565204D656D6F7279B7
:103110003A2000436F6D70696C65643A20417567B1
:1031200020323320323031390A00207C204175743E
:10313000686F723A2054696E794D616368696E6593
:103140007333440A00323031392D30372D3330009B
:10315000204C61737420557064617465643A20007A
:10316000322E302E785F43523239420A004D61725E
:103170006C696E0020536F667477617265205265CA
:103180007365740A00205761746368646F67205226
:10319000657365740A002042726F776E206F7574D4
:1031A0002052657365740A002045787465726E61FB
:1031B0006C2052657365740A00506F7765725570A4
:1031C0000A0073746172740A006175746F25632E4E
:1031D00067006572726F722077726974696E67201A
:1031E000746F2066696C650A00446F6E65207361B8
:1031F00076696E672066696C652E0A004D3239006B
:10320000205A3A0020593A0020583A00656E6473FB
:10321000746F7073206869743A20004732385859C7
:103220000043616E6E6F74206F70656E20737562FF
:10323000646972200053442063617264206F6B0ADA
:10324000006F70656E526F6F74206661696C6564A3
:103250000A00766F6C756D652E696E697420666103
:10326000696C65640A00534420696E697420666164
:10327000696C0A004D3234004D32332025730057FB
:10328000726974696E6720746F2066696C653A2094
:10329000002E0A006F70656E206661696C65642C93
:1032A0002046696C653A20002E0A006F70656E201A
:1032B0006661696C65642C2046696C653A2000463D
:1032C000696C652073656C65637465640A002053DE
:1032D000697A653A200046696C65206F70656E6595
:1032E000643A2000667265736800646F696E6700F7
:1032F0002066696C653A20004E6F772000454E4489
:1033000020535542524F5554494E450A00222070D1
:103310006F73002220706172656E743A22005355FB
:1033200042524F5554494E452043414C4C20746104
:10333000726765743A2200747279696E6720746FDF
:103340002063616C6C207375622D67636F64652008
:1033500066696C6573207769746820746F6F206D7F
:10336000616E79206C6576656C732E204D41582016
:103370006C6576656C2069733A310A00534420709D
:1033800072696E74696E67206279746520004E6F91
:1033900074205344207072696E74696E670A00204D
:1033A000746F6F206C6F6E672065787472757369C7
:1033B0006F6E2070726576656E7465640A002063B6
:1033C0006F6C6420657874727573696F6E207072AB
:1033D0006576656E7465640A00486F6D65202573B7
:1033E00025732573204669727374002046697273D1
:1033F000740A00486F6D65200000000000000000A6
:103400000000000000000048420000484200008028
:10341000405761726E696E673A20486F6D696E67DA
:103420002042756D702044697669736F72203C206C
:10343000310A000202040000A0400000A040000089
:10344000004000809D4300009B430000C843FFFFF5
:10345000FF496E76616C6964206578747275646585
:10346000720A007C3C3E5E2B3D3F2F5B5D3B2C2A6D
:10347000225C0050726F62696E67204661696C65FC
:10348000640A0050726F62696E67204661696C65FC
:1034900064002020207C0A004E414E0020202E2077
:1034A000202000207C004C43443A0A004353563A03
:1034B0000A0020666F7220003A0A0A000A42656418
:1034C00020546F706F677261706879205265706FF9
:1034D0007274004732380000446F6E652E0A003F58
:1034E000496E76616C69642073746F7261676520E0
:1034F000736C6F742E0A3F557365203020746F20F3
:10350000003F454550524F4D2073746F726167659F
:10351000206E6F7420617661696C61626C652E0A41
:1035200000446F6E652E0A003F496E76616C6964D7
:103530002073746F7261676520736C6F742E0A3F1D
:10354000557365203020746F20003F454550524F21
:103550004D2073746F72616765206E6F74206176A1
:1035600061696C61626C652E0A003F50342069739A
:10357000206F6E6C7920617661696C61626C652088
:103580007768656E20616E204C434420697320701B
:10359000726573656E742E0A003F50322069732085
:1035A0006F6E6C7920617661696C61626C65207701
:1035B00068656E20616E204C4344206973207072F0
:1035C0006573656E742E0A00292E0A0A0050726F08
:1035D00062696E672061726F756E642028004D65A8
:1035E000736820696E76616C6964617465642E200D
:1035F00050726F62696E67206D6573682E0A004DA8
:10360000657368207A65726F65642E0A004465668A
:1036100061756C742073746F7261676520736C6F71
:103620007420302073656C65637465642E0A004CE9
:103630006F6164696E6720746573745F7061747420
:1036400065726E2076616C7565732E0A0A00496E8C
:1036500076616C696420746573745F7061747465FD
:10366000726E2076616C75652E20282D3120746F66
:103670002032290A0A004C6F636174696F6E7320EF
:10368000696E76616C6964617465642E0A0A00452E
:103690006E74697265204D65736820696E76616C21
:1036A0006964617465642E0A0A00220A00556E6B13
:1036B0006E6F776E20636F6D6D616E643A202200CD
:1036C00020746F6F206C6F6E6720657874727573ED
:1036D000696F6E2070726576656E7465640A00208D
:1036E000636F6C6420657874727573696F6E207097
:1036F000726576656E7465640A0024F4D43050C334
:103700008E20C2A24017828B7011127A910D816CAB
:10371000D90AA861E108C7586607615143061E4BE4
:103720005D05C145A7041A411104093D980371398B
:1037300031034036DB0265339102D4305402802ECF
:103740001D02632CEE01752AC501B028A0011027C7
:1037500081018F2564012B244B01E0223401AC212F
:103760001F018D200D01801FFC00841EED00971DA0
:10377000DF00B81CD200E61BC600201BBC00641A88
:10378000B200B219A8000A19A0006A189900D1174E
:10379000910040178B00B516840031167E00B315DA
:1037A00079003A157300C7146F0058146A00EE13BD
:1037B00066008813630025135E00C7125B006C125D
:1037C000570015125400C111510070114F00211102
:1037D0004B00D61049008D104700461044000210DF
:1037E0004200C00F4000800F3E00420F3C00060F19
:1037F0003B00CB0E3800930E37005C0E3500270ED1
:103800003400F30D3200C10D3100900D3000600D19
:103810002E00320D2D00050D2C00D90C2B00AE0C06
:103820002900850C29005C0C2700350C27000E0CA4
:103830002600E80B2400C40B2400A00B23007D0B02
:1038400023005A0B2100390B2100180B2000F80A25
:103850001F00D90A1E00BB0A1E009D0A1D00800A17
:103860001D00630A1C00470A1B002C0A1B00110ADA
:103870001A00F7091A00DD091900C4091900AB097B
:103880001900920917007B091800630917004C09F9
:10389000160036091600200916000A091500F50859
:1038A0001500E0081400CC081400B8081400A4089F
:1038B0001400900813007D0812006B0813005808CC
:1038C00012004608120034081100230811001208E3
:1038D000110001081100F0071000E0071000D007E8
:1038E0001000C0071000B0070F00A10710009107DB
:1038F0000E0083070F0074070F0065070E005707BF
:103900000E0049070E003B070D002E070E00200792
:103910000D0013070D0006070D00F9060C00ED065B
:103920000D00E0060C00D4060C00C8060C00BC0616
:103930000C00B0060C00A4060B0099060C008D06C6
:103940000B0082060B0077060B006C060B0061066D
:103950000A0057060B004C060A0042060A00380609
:103960000A002E060A0024060A001A060A0010069B
:10397000090007060A00FD050900F4050900EB052A
:103980000900E2050900D9050900D0050900C705AD
:103990000900BE050900B5050800AD050800A5052C
:1039A00009009C050800940508008C0508008405A2
:1039B00008007C050800740508006C050700650513
:1039C00008005D050700560508004E05070047057D
:1039D00007004005080038050700310507002A05E3
:1039E0000700230507001C050600160507000F0544
:1039F00007000805060002050700FB040600F504A1
:103A00000700EE040600E8040600E2040700DB04F9
:103A10000600D5040600CF040600C9040600C3044E
:103A20000600BD040600B7040600B1040500AC049E
:103A30000600A6040600A00405009B0406009504E9
:103A40000500900406008A04050085040500800432
:103A500006007A04050075040500700405006B0477
:103A6000050066040500610405005C0405005704B8
:103A70000500520405004D040500480405004304F8
:103A800005003E0404003A04050035040500300436
:103A900004002C04050027040400230405001E0470
:103AA00004001A04040016040500110404000D04A7
:103AB0000400090405000404040000040400FC03DD
:103AC0000400F8030400F4030400F0030400EC0312
:103AD0000400E8030400E4030400E0030400DC0342
:103AE0000400D8030400D4030400D0030400CC0372
:103AF0000400C8030300C503030024F404D9201BF9
:103B0000C40C5C0E9804C4095F0265077101F405DA
:103B1000F900FB04B30048048700C103690058039F
:103B2000550003034500BE023A00840231005302EF
:103B30002A002902250004022000E4011C00C8011B
:103B40001900AF01170098011400840113007101DE
:103B500010006101100051010E0043010D003601FB
:103B60000B002B010B0020010B00150109000C01BB
:103B7000090003010800FB000800F3000800EB0047
:103B80000700E4000600DE000600D8000600D200B0
:103B90000600CC000500C7000500C2000500BD00FE
:103BA0000400B9000400B5000400B1000400AD0039
:103BB0000400A9000400A5000300A20003009F0068
:103BC00004009B000300980003009500020093008E
:103BD0000300900003008D0002008B0003008800AA
:103BE00002008600020084000300810002007F00C2
:103BF00002007D0002007B000200790002007700D5
:103C000001007600020074000200720001007100E1
:103C100002006F0002006D0001006C0002006A00EB
:103C200001006900020067000100660001006500F4
:103C300001006400020062000100610001006000F8
:103C400001005F0002005D0001005C0001005B00FC
:103C500001005A00010059000100580001005700FE
:103C600001005600010055000100540001005300FE
:103C700000005300010052000100510001005000FB
:103C800001004F0001004E0000004E0001004D00F9
:103C900001004C0001004B0000004B0001004A00F5
:103CA00001004900010048000000480001004700F1
:103CB00001004600000046000100450000004500EC
:103CC00001004400010043000000430001004200E5
:103CD00000004200010041000000410001004000DE
:103CE00001003F0000003F0001003E0000003E00D8
:103CF00001003D0000003D0001003C0000003C00D0
:103D000000003C0001003B0000003B0001003A00C5
:103D100000003A00010039000000390001003800BD
:103D200000003800000038000100370000003700B4
:103D300001003600000036000000360001003500AA
:103D400000003500000035000100340000003400A0
:103D50000000340001003300000033000000330095
:103D6000010032000000320000003200010031008A
:103D70000000310000003100010030000000300080
:103D80000000300001002F0000002F0000002F0075
:103D900000002F0001002E0000002E0000002E0069
:103DA00001002D0000002D0000002D0000002D005E
:103DB00001002C0000002C0000002C0000002C0052
:103DC00001002B0000002B0000002B0000002B0046
:103DD00001002A0000002A0000002A0000002A003A
:103DE000010029000000290000002900000029002E
:103DF0000000290001002800000028000000280021
:103E00000000280000002800010027000000270013
:103E10000000270000002700000027000100260006
:103E200000002600000026000000260000002600FA
:103E300001002500000025000000250000002500ED
:103E400000002500000025000100240000002400DF
:103E500000002400000024000000240001002300D2
:103E600000002300000023000000230000002300C6
:103E700000002300000023000100220000002200B7
:103E800000002200000022000000220000002200AA
:103E9000010021000000210000002100000021009D
:103EA000000021000000210000002100010020008E
:103EB0000000200000002000000020000000200082
:103EC00000002000000020000000200001001F0072
:103ED00000001F0000001F0000001F0000001F0066
:103EE00000001F0000001F0001001E0000001E0057
:103EF00000001E0000001E000000043700001E2904
:103F00000000511B00005810000010090000CC04F4
:103F100000007802000041010000626564002C206E
:103F200073797374656D2073746F7070656421208C
:103F30004865617465725F49443A200042656420B7
:103F400048656174696E67204661696C6564004804
:103F5000656174696E67206661696C6564004245DD
:103F60004420544845524D414C2052554E415741F2
:103F70005900546865726D616C2052756E6177618D
:103F8000790045312048656174696E672046616932
:103F90006C65640048656174696E67206661696C70
:103FA000656400453120544845524D414C205255DE
:103FB0004E4157415900546865726D616C205275CD
:103FC0006E61776179004D313137004D33310053E7
:103FD000442072656164206572726F720A00446FDA
:103FE0006E65207072696E74696E672066696C65B3
:103FF0000A0043616E6E6F74206F70656E2073757A
:104000006264697220002569730025696D20256945
:1040100073002569682025696D202569730025696D
:1040200064202569682025696D202569730025694C
:104030007920256964202569682025696D20256916
:10404000730023646566696E652044454641554C9E
:10405000545F0000626564004B6420004B692000DF
:104060004B702000504944204175746F74756E6523
:104070002066696E697368656421205075742074C8
:104080006865206C617374204B702C204B69206133
:104090006E64204B6420636F6E7374616E74732062
:1040A00066726F6D2062656C6F7720696E746F2029
:1040B000436F6E66696775726174696F6E2E680A08
:1040C00000504944204175746F74756E65206661B7
:1040D000696C6564212074696D656F75740A0045AB
:1040E0003120544845524D414C2052554E41574184
:1040F000590042454420544845524D414C205255A8
:104100004E4157415900546865726D616C2052757B
:104110006E617761790045312048656174696E6729
:10412000204661696C65640042656420486561747D
:10413000696E67204661696C6564004865617469F1
:104140006E67206661696C65640050494420417562
:10415000746F74756E65206661696C6564212054A6
:10416000656D706572617475726520746F6F20681B
:104170006967680A00204B643A2000204B693A20A6
:1041800000204B703A20000A20436C61737369630E
:1041900020504944200A00204B643A2000204B69FB
:1041A0003A2000204B703A20000A204E6F206F7694
:1041B000657273686F6F740A002054753A2000208E
:1041C0004B753A2000206D61783A2000206D696EB1
:1041D0003A200020643A200020626961733A20008E
:1041E000504944204175746F74756E652073746115
:1041F00072740A00504944204175746F74756E657D
:10420000206661696C6564212054656D706572611A
:104210007475726520746F6F20686967680A005052
:104220004944204175746F74756E65206661696CD0
:1042300065642120426164206578747275646572DA
:10424000206E756D6265720A00646F6E650A0049C2
:104250006E73756666696369656E74206461746106
:104260000A00000070410000AA4200001B43000049
:104270006143008093430080B6430080D9430080AF
:10428000FC4300C00F440040214400C032440040C1
:10429000444400C055440040674400C078440020B6
:1042A0008544000070410000AC4200001D43000046
:1042B0006443008095430000B9430080DC43000064
:1042C000004400C0114400802344004035440000F5
:1042D000474400C0584400806A4400407C440000C9
:1042E00087444578747261706F6C6174696E672081
:1042F0006D6573682E2E2E002F2F616374696F6EAB
:104300003A00627574746F6E00656E640070726F4F
:104310006D70745F0073686F77004D3837362052C8
:104320006573706F6E64696E672050524F4D5054C4
:104330005F00554E4B4E4F574E205354415445004D
:1043400047434F44455F494E464F004C43445F50FE
:10435000415553455F524553554D450046494C41E3
:104360004D454E545F52554E4F55545F434F4E543A
:10437000494E55450046494C414D454E545F5255B6
:104380004E4F5554004D323400436F6E74696E7554
:10439000650044697361626C6552756E6F75740077
:1043A0005075726765204D6F726500506175736559
:1043B000640070617573656400486F74656E642095
:1043C000746F6F20636F6C640A00506175736500D1
:1043D000507265737320627574746F6E20286F72EB
:1043E000204D3130382920746F20726573756D65EA
:1043F0000A00496E736572742066696C616D656E42
:104400007420616E642070726573732062757474B9
:104410006F6E20286F72204D313038290A00436FAB
:104420006E74696E75650052656865617420446FCD
:104430006E6500526568656174696E672E2E2E0088
:10444000526568656174696E67004865617465727C
:1044500054696D656F7574005265686561740048D4
:10446000656174657254696D656F7574005072652D
:10447000737320627574746F6E20286F72204D31D3
:1044800030382920746F2068656174206E6F7A7AE5
:104490006C650A004E6F7A7A6C65205061726B65AC
:1044A0006400436F6E74696E7565004E6F7A7A6C46
:1044B00065205061726B656400486F74656E64209E
:1044C000746F6F20636F6C640A00726573756D653D
:1044D0006400626567696E00436F6E74696E75652E
:1044E0000044697361626C6552756E6F757400503B
:1044F000757267654D6F7265005061757365640014
:104500004C6F61642046696C616D656E7400436F29
:104510006E74696E7565004C6F61642046696C61EC
:104520006D656E74205400496E73657274206669FF
:104530006C616D656E7420616E642070726573735A
:1045400020627574746F6E20286F72204D31303880
:10455000290A00526573756D65003F556E61626C86
:104560006520746F2073617665206D6573682064C3
:104570006174612E0A003F556E61626C6520746F34
:10458000206C6F6164206D65736820646174612EB6
:104590000A00EE020000EE020000640000003C0091
:1045A00000000000FA430000FA4300002041000030
:1045B0008C420000A0420000A0420000C84300005E
:1045C0000C43556E696669656420426564204C65DC
:1045D00076656C696E67003A0A0020204D363033EC
:1045E000200020440020204D343132205300466901
:1045F0006C616D656E742072756E6F757420736575
:104600006E736F723A0A002055004C0046696C6167
:104610006D656E74206C6F61642F756E6C6F616474
:10462000206C656E677468733A0A0020204D383537
:1046300031205A005A2D50726F6265204F666673A2
:1046400065740020440020490020204D3330342080
:10465000500020440020490020204D3330312050AC
:10466000005049442073657474696E67733A0A0098
:10467000206D65736865732E0A0A00454550524FD8
:104680004D2063616E20686F6C6420000A41637482
:10469000697665204D65736820536C6F743A20000D
:1046A000205A0020204D3432302053003A0A002096
:1046B0005A0020590020204D323036205800486FD3
:1046C0006D65206F66667365743A0A00204A0020A3
:1046D000540020530020204D323035204200204A23
:1046E0003C6A756E635F6465763E00416476616E18
:1046F0006365643A20423C6D696E5F7365676D6502
:104700006E745F74696D655F75733E20533C6D69AF
:104710006E5F66656564726174653E20543C6D69C8
:104720006E5F74726176656C5F66656564726174F4
:10473000653E0020540020520020204D32303420AD
:104740005000416363656C65726174696F6E202807
:10475000756E6974732F7332293A20503C707269F8
:104760006E745F616363656C3E20523C7265747267
:104770006163745F616363656C3E20543C74726175
:1047800076656C5F616363656C3E0A0020450020BE
:104790005A0020590020204D3230312058004D6100
:1047A00078696D756D20416363656C6572617469CC
:1047B0006F6E2028756E6974732F7332293A0A0060
:1047C000204500205A0020590020204D323033204F
:1047D00058004D6178696D756D206665656472611C
:1047E0007465732028756E6974732F73293A0A00F3
:1047F00053746570732070657220756E69743A0A1F
:104800000020204D3230302044300A0020204D322C
:1048100030302044002044697361626C65640A0092
:1048200046696C616D656E742073657474696E673A
:10483000733A0020286D6D29002020473231202056
:1048400020203B20556E69747320696E206D6D00C9
:10485000486F6D696E67204661696C6564006F70B2
:10486000656E00545249474745524544003A20007E
:1048700066696C616D656E74007A5F6D696E007952
:104880005F6D696E00785F6D696E005265706F7262
:1048900074696E6720656E6473746F7020737461E1
:1048A0007475730A00205A3A0020593A0020436F69
:1048B000756E7420583A0020453A00205A3A00207C
:1048C000593A00583A0057616974696E6720666FFB
:1048D00072206865617475702E0A004C6561766996
:1048E0006E6720473236003F5370656369666965BD
:1048F0006420582C5920636F6F7264696E6174650F
:10490000206F7574206F6620626F756E64732E0A57
:10491000003F28522965706561742076616C756569
:10492000206E6F7420706C61757369626C653B20DA
:104930006D757374206265206174206C6561737499
:1049400020312E0A003F2852296570656174206D60
:104950007573742062652073706563696669656448
:10496000207768656E206E6F74207573696E67209E
:10497000616E204C43442E0A003F537065636966A4
:10498000696564206E6F7A7A6C652074656D7065F8
:10499000726174757265206E6F7420706C617573CE
:1049A00069626C652E0A003F5370656369666965CC
:1049B000642066696C616D656E742073697A652028
:1049C0006E6F7420706C61757369626C652E0A007D
:1049D0003F537065636966696564207072696D65CF
:1049E000206C656E677468206E6F7420706C6175E2
:1049F0007369626C652E0A003F5072696D65206CA8
:104A0000656E677468206D757374206265207370BD
:104A100065636966696564207768656E206E6F748A
:104A2000207573696E6720616E204C43442E0A0026
:104A30003F537065636966696564206E6F7A7A6C4E
:104A4000652073697A65206E6F7420706C61757370
:104A500069626C652E0A003F526574726163746905
:104A60006F6E204D756C7469706C696572206D7520
:104A70007374206265207370656369666965642E6E
:104A80000A003F5370656369666965642052657406
:104A900072616374696F6E204D756C7469706C69B6
:104AA0006572206E6F7420706C61757369626C65DD
:104AB0002E0A003F537065636966696564206C6106
:104AC00079657220686569676874206E6F742070FC
:104AD0006C61757369626C652E0A0043292E0A00A9
:104AE0003F5370656369666965642062656420741C
:104AF000656D7065726174757265206E6F7420707B
:104B00006C61757369626C65202834302D00473202
:104B100036207374617274696E672E2E2E0A0043FC
:104B200061703A00220A00656E7175657565696E7F
:104B3000672022002042002050006F6B00526573F6
:104B4000656E643A200053544F505045442E200067
:104B50005072696E7465722073746F707065642032
:104B600064756520746F206572726F72732E2046B3
:104B7000697820746865206572726F7220616E6456
:104B800020757365204D39393920746F2072657333
:104B9000746172742E202854656D7065726174752D
:104BA00072652069732072657365742E2053657475
:104BB0002069742061667465722072657374617215
:104BC00074696E67290A004E6F20436865636B73D2
:104BD000756D2077697468206C696E65206E756DDF
:104BE0006265722C204C617374204C696E653A20AA
:104BF000004E6F20436865636B73756D2077697431
:104C000068206C696E65206E756D6265722C204C33
:104C1000617374204C696E653A2000636865636B4C
:104C200073756D206D69736D617463682C204C61C0
:104C30007374204C696E653A20004C696E65204E95
:104C4000756D626572206973206E6F74204C61739C
:104C500074204C696E65204E756D6265722B312C27
:104C6000204C617374204C696E653A20004D3131DF
:104C70003000776169740A0070012C0190012701EE
:104C8000B0012201C0011D01F00118011002130141
:104C900030020E016002090190020401C002FF000F
:104CA0000003FA004003F5008003F000D003EB009E
:104CB0002004E6007004E100E004DC004005D700B9
:104CC000C005D2004006CD00D006C8008007C30052
:104CD0003008BE00F008B900C009B400B00AAF0047
:104CE000B00BAA00D00CA500000EA000500F9B0036
:104CF000C01096005012910000148C00C01587005F
:104D0000B0178200B0197D00D01B7800001E730020
:104D100040206E0090226900F024640040275F006C
:104D200090295A00E02B5500102E500020304B00E7
:104D300010324600E033410090353C001037370018
:104D400070383200A0392D00B03A2800A03B230073
:104D5000603C1E00103D1900903D1400103E0F00F5
:104D6000703E0A00C03E0500003F0000403FFBFFD0
:104D7000803FF6FFC03FF1FF202D20496E76616C29
:104D80006964206578747275646572206E756D62F1
:104D9000657220210A001000C90210012C01400197
:104DA000220170011801B0010E01F001040150024E
:104DB000FA00B002F0003003E600D003DC009004FB
:104DC000D2007005C800A006BE000008B400B009FB
:104DD000AA00D00BA000600E960060118C00001598
:104DE000820020197800C01D6E00A0226400B02748
:104DF0005A00902C500000314600E0343C0010383E
:104E00003200903A2800603C1E00A03D1400803E15
:104E10000A00203F0000453120544845524D414C86
:104E20002052554E4157415900424544205448456F
:104E3000524D414C2052554E4157415900546865DE
:104E4000726D616C2052756E617761790045312019
:104E50004572723A204D415854454D50004572728A
:104E60003A204D415854454D5020424544004D4153
:104E70005854454D502074726967676572656400C7
:104E80004531204572723A204D494E54454D5000EF
:104E90004572723A204D494E54454D50204245448A
:104EA000004D494E54454D502074726967676572D4
:104EB0006564000A0A0020205A5F4D494E3A0020DE
:104EC00020595F4D494E3A002020585F4D494E3AD7
:104ED000004D383420582059205A204500202F00FA
:104EE0002042403A0020403A0020573A0020573AEA
:104EF00000544D3344203130532050726F2052659E
:104F00006164792E005072696E74696E672E2E2E60
:104F1000005072696E74205061757365640063613E
:104F20006E63656C005072696E742041626F7274BA
:104F300065640055492041626F7274007265737533
:104F40006D65004D32340000809D4300009B43009E
:104F500000C8430000000000000000000000004EF8
:104F60006F20454550524F4D2E0A004F46460A00CD
:104F7000466164652048656967687420004265641D
:104F8000204C6576656C696E6720004661696C65CA
:104F90006420746F20656E61626C652042656420D8
:104FA0004C6576656C696E670A00496E76616C695E
:104FB00064206D6573682E0A0076616C69640A531B
:104FC000746F7261676520736C6F743A2000696E4C
:104FD000004D65736820697320003F55736520306C
:104FE00020746F20003F496E76616C696420737491
:104FF0006F7261676520736C6F742E0A003F4545C0
:1050000050524F4D2073746F72616765206E6F74DC
:1050100020617661696C61626C652E0A004D657372
:105020006820706F696E742063616E6E6F742062A9
:1050300065207265736F6C7665640A004D34323199
:1050400020696E636F727265637420706172616D46
:10505000657465722075736167650A0046696E69DB
:1050600073686564210A00206F662000205A0020C2
:105070005900476F696E6720746F3A205800435794
:105080000A00206469723A0020616E676C653A001C
:105090005374617274207261646975733A00506F61
:1050A000736974696F6E696E6720746865207072C9
:1050B0006F62652E2E2E0A003F4E756D626572205E
:1050C0006F66206C65677320696E206D6F76656D05
:1050D000656E74206E6F7420706C61757369626C9C
:1050E000652028302D3135292E0A003F2028582CE4
:1050F0005929206F7574206F6620626F756E647316
:105100002E0A003F53616D706C652073697A6520CB
:105110006E6F7420706C61757369626C65202834E1
:105120002D3530292E0A004D3438205A2D50726FFB
:105130006265205265706561746162696C69747939
:1051400020546573740A003F2856296572626F7394
:1051500065206C6576656C20697320696D706C6183
:10516000757369626C652028302D34292E0A005A27
:105170005F53544F505F50494E005A5F535445504F
:105180005F50494E005A5F4D494E5F50494E005A9C
:105190005F454E41424C455F50494E005A5F44497D
:1051A000525F50494E005A5F43535F50494E005979
:1051B0005F53544F505F50494E00595F5354455010
:1051C0005F50494E00595F4D494E5F50494E00595E
:1051D0005F454E41424C455F50494E00595F44493E
:1051E000525F50494E00595F43535F50494E00583B
:1051F0005F53544F505F50494E00585F53544550D1
:105200005F50494E00585F4D494E5F50494E00581F
:105210005F454E41424C455F50494E00585F4449FE
:10522000525F50494E00585F43535F50494E005300
:10523000535F50494E00534552564F335F50494ECD
:1052400000534552564F325F50494E005345525617
:105250004F315F50494E00534552564F305F5049D1
:105260004E00534453530053445F44455445435404
:105270005F50494E0053434B5F50494E0052414DE1
:1052800050535F44395F50494E0052414D50535F77
:1052900044385F50494E0052414D50535F443130C5
:1052A0005F50494E004D4F53495F50494E004D4F9E
:1052B000534645545F445F50494E004D49534F5F3C
:1052C00050494E004D4158363637355F53535F5085
:1052D000494E004C45445F50494E004845415445B5
:1052E000525F4245445F50494E0048454154455243
:1052F0005F305F50494E0046494C5F52554E4F5506
:10530000545F50494E0046414E315F50494E004671
:10531000414E5F50494E0045315F535445505F50F8
:10532000494E0045315F454E41424C455F50494E24
:105330000045315F4449525F50494E0045315F435B
:10534000535F50494E0045305F535445505F5049BC
:105350004E0045305F454E41424C455F50494E003E
:1053600045305F4449525F50494E0045305F4353DA
:105370005F50494E00455F4D5558325F50494E00D1
:10538000455F4D5558315F50494E00455F4D55586A
:10539000305F50494E004156525F53535F50494E63
:1053A000004156525F53434B5F50494E00415652A5
:1053B0005F4D4F53495F50494E004156525F4D4932
:1053C000534F5F50494E0054454D505F4245445F36
:1053D00050494E0054454D505F315F50494E005486
:1053E000454D505F305F50494E0046494C57494447
:1053F00054485F50494E00545844005258440020CD
:10540000202000202020416E616C6F6720696E2093
:105410003D2025356C64003C756E757365642F7591
:105420006E6B6E6F776E3E00202841253264292016
:1054300020002533642000257350494E3A20004F48
:105440007574707574203D2000496E70757420204D
:105450003D2000416E616C6F6720696E203D202504
:10546000356C640070726F7465637465642000202D
:10547000284125326429202000253364200025732B
:1054800050494E3A2000FB530001F7530101EA5303
:105490003B00DF534300D4534500C7534400BA5385
:1054A0003201AD533301A1533401965335018B536F
:1054B000280180532A0175532C016B532A01605334
:1054C0001C015253180146531A013C532C0131530D
:1054D000220123531E01175324010F5309010653C0
:1054E0000701F7520201EA520A01DB520801D352C6
:1054F0000D01C4524201BB523201AE520701A55206
:10550000330197520A018A5208017D5209017552EE
:105510003401675231016252350157520B014C522E
:10552000060141520501365204012F52350126521F
:1055300035011C5237010F52260105520301FA5161
:105540003601EF510301E6513101DC513D01CF51EC
:105550003801C5510E01BA513C01AF510E01A6519F
:1055600028019C5130018F513E01855112017A5121
:105570002E016F511201446F6E652E0A0053455281
:10558000564F206E6F74207365742075702E0A005C
:105590004D343320576169742043616C6C6564003D
:1055A000436F6E74696E7565004D343320576169C1
:1055B000742043616C6C6564005761746368696E44
:1055C000672070696E730A0064697300656E00611C
:1055D000626C65640A00656E6473746F70206D6F31
:1055E0006E69746F722000204500205A0020590017
:1055F000204D3932205800205A00205900580020F0
:10560000204D61783A2000205A002059005800208F
:10561000204D696E3A2000536F667420656E647386
:10562000746F70733A200020496E76616C69642053
:10563000657874727564657220003F4D65736820EB
:10564000746F6F2062696720666F72204545505203
:105650004F4D2E0A004E6F20454550524F4D2E0A99
:10566000000A20696E6974207A70726F62655F7AD1
:105670006F6666736574203D2000454550524F4D5E
:1056800020496E697469616C697A65640A00232037
:105690006F662073616D706C65733A200050726F95
:1056A00062696E6720506F696E742025692F2569C5
:1056B000002E0A0A002F000A50726F62696E67207E
:1056C0006D65736820706F696E742000496E766135
:1056D0006C6964206D617020747970652E0A0A000F
:1056E0003F2846296164652068656967687420669B
:1056F0006F7220426564204C6576656C20436F7242
:1057000072656374696F6E206E6F7420706C617562
:105710007369626C652E0A0A003F43616E2774202C
:10572000616374697661746520616E64206465618B
:105730006374697661746520617420746865207390
:10574000616D652074696D652E0A0A00426F746888
:10575000205820262059206C6F636174696F6E7326
:10576000206D757374206265207370656369666966
:1057700065642E0A0A003F496E76616C6964206791
:105780007269642073697A6520284A2920737065DC
:105790006369666965642028322D39292E0A0A005A
:1057A0003F285029686173652076616C75652069B2
:1057B0006E76616C69642028302D36292E0A0A0025
:1057C0003F2856296572626F7365206C6576656C3B
:1057D00020697320696D706C61757369626C6520F6
:1057E00028302D34292E0A0A003F28522965706579
:1057F000746974696F6E20636F756E7420696E765C
:10580000616C69642028312B292E0A0A00040000EB
:105810000501000300050100050400000005000368
:10582000001C58175812580D585D0A00436F756CCC
:1058300064206E6F7420636F6D706C657465204CAE
:1058400053462100436F727265637465645F5A3D0D
:105850000054696C74696E6720506F696E742025FE
:10586000692F2569000A0A002F0054696C74696E5B
:1058700067206D65736820706F696E7420003F4506
:1058800072726F722070726F62696E6720706F69DA
:105890006E742E2041626F7274696E67206F70653E
:1058A000726174696F6E2E0A00436F727265637461
:1058B00065645F5A3D0054696C74696E6720506F6F
:1058C000696E7420332F330054696C74696E6720DD
:1058D0006D6573682028332F33290A00436F727275
:1058E00065637465645F5A3D0054696C74696E67E2
:1058F00020506F696E7420322F330054696C7469C4
:105900006E67206D6573682028322F33290A0043A3
:105910006F727265637465645F5A3D0054696C749C
:10592000696E6720506F696E7420312F330054699F
:105930006C74696E67206D6573682028312F332978
:105940000A0050574D3A20202534640050574D3AF4
:1059500020202534640050574D3A2020253464001F
:1059600050574D3A20202534640050574D3A20209E
:105970002534640050574D3A202025346400505798
:105980004D3A20202534640050574D3A20202534CC
:10599000640050574D3A20202534640050574D3A4A
:1059A00020202534640050574D3A202025346400CF
:1059B00050574D3A20202534640050574D3A20204E
:1059C0002534640050574D3A202025346400505748
:1059D0004D3A20202534640050574D3A202025347C
:1059E0006400433A2000423A2000413A200020203F
:1059F0002020434F4D002020206E6F6E2D73746168
:105A00006E646172642050574D206D6F6465002094
:105A10002020636F6D7061726520696E74657272AB
:105A200075707420656E61626C6564002020206F63
:105A3000766572666C6F7720696E746572727570C8
:105A40007420656E61626C6564003A20002020203D
:105A50002054494D534B00423A200020202020542E
:105A600043435200413A2000202020205443435217
:105A7000002020202043533A200020202020574798
:105A80004D3A200050574D3A20202534640050579D
:105A90004D3A20202534640047004800000088006B
:105AA0008A008C00B300B400000098009A009C00AB
:105AB000A800AA00AC0028012A012C0120202020E7
:105AC00054494D455200440045006E00800081005D
:105AD0006F00B000B1007000900091007100A00054
:105AE000A100720020012101730020697320616C04
:105AF000736F207469656420746F20746869732003
:105B000070696E0054494D45523143000A202E0001
:105B10002020002020506F72743A20002E0A006F5F
:105B200070656E206661696C65642C2046696C65E1
:105B30003A200000002100240027002A002D003018
:105B400000330001010000040107010A01000022E6
:105B500000250028002B002E003100340002010037
:105B600000050108010B0100002000230026002988
:105B7000002C002F00320000010000030106010983
:105B80000105050505070508080808020202020AC2
:105B90000A080804040404010101010101010103D0
:105BA00003030303030303040707070C0C0C0C0C8B
:105BB0000C0C0C0202020206060606060606060B7E
:105BC0000B0B0B0B0B0B0B010210202008081020F5
:105BD0004010204080020102010804020101020479
:105BE0000810204080804020100804020180040238
:105BF000018040201008040201080402010102048F
:105C00000810204080010204081020408000000A93
:105C10000B02090C0D0E0807030401000000000030
:105C20000000000000000000000000000000000074
:105C30000000000000000000001211100000000031
:105C40000000000000000000000000000000000054
:105C50000000004469666665723A200046726F6D06
:105C60005374703A00537465707065723A00556EE3
:105C70004C6576656C3A004C6576656C65643A00F7
:105C80005261773A20202020000A4C6F67696361D7
:105C90006C3A0000D101E70111241FBECFEFD1E221
:105CA000DEBFCDBF00E00CBF18E0A0E0B2E0E0E353
:105CB000FBEA02E00BBF02C007900D92AA30B107C9
:105CC000D9F72CE1AAE0B8E001C01D92AB38B207C9
:105CD000E1F71EE2CBE4DEE200E006C02197010915
:105CE000802FFE010F946E50CA34D10780E0080760
:105CF000A9F70F94893A0D9486550C9400002F92C1
:105D00003F924F925F926F927F928F929F92AF924B
:105D1000BF92CF92DF92EF92FF920F931F93CF9398
:105D2000DF93CDB7DEB7A8970FB6F894DEBF0FBEEE
:105D3000CDBF80910901817091E0982720912D08B5
:105D4000921781F190932D08811116C00E94636D06
:105D50008091AD1683FF09C089E893E00E947264C8
:105D600061E080E00F940E351DC060E081E00F948B
:105D70000E3582EA93E014C00091AD1603FB0027B4
:105D800000F90E94F26C8091AD16877F8093AD166A
:105D9000002341F060E081E00F940E358BEB93E03F
:105DA0000E94726480910A0881FF11C18091AD1434
:105DB0009091AE14891B8F70843008F008C18CE07C
:105DC000E6E5FBE0DE01119601900D928A95E1F780
:105DD0008091690B90916A0BA0916B0BB0916C0B49
:105DE0008D8F9E8FAF8FB8A39C01AD016091560B34
:105DF0007091570B8091580B9091590B0F947650DE
:105E00006B017C016093560B7093570B8093580B7A
:105E10009093590B80916D0B90916E0BA0916F0B2D
:105E2000B091700B89A39AA3ABA3BCA39C01AD0155
:105E300060915A0B70915B0B80915C0B90915D0BA4
:105E40000F9476506D8B7E8B8F8B988F60935A0B4F
:105E500070935B0B80935C0B90935D0B8091710B47
:105E60009091720BA091730BB091740B8DA39EA3B4
:105E7000AFA3B8A79C01AD0160915E0B70915F0B61
:105E80008091600B9091610B0F9476504B015C01F7
:105E900060935E0B70935F0B8093600B9093610B2C
:105EA000A7019601C701B6010F94F3492B013C01EC
:105EB0002D893E894F89588DCA01B9010F94F34944
:105EC0009B01AC01C301B2010F9477502B013C013F
:105ED000A5019401C501B4010F94F3499B01AC01E4
:105EE000C301B2010F9477500F9475539B01AC011D
:105EF00060E070E080E89FE30F94715120913F02D1
:105F00003091400240914102509142020F94F34976
:105F10002DEC3CEC4CEC5DE30F94F34920E030E0D9
:105F200040E85EE30F94F3492B013C0120E030E0B0
:105F300040E85FE30F948D4987FF83C6A301920178
:105F4000C701B6010F94F3492D8D3E8D4F8D58A199
:105F50000F9477506093560B7093570B8093580BA8
:105F60009093590BA30192016D897E898F89988D39
:105F70000F94F34929A13AA14BA15CA10F9477504A
:105F800060935A0B70935B0B80935C0B90935D0B4B
:105F9000A3019201C501B4010F94F3492DA13EA1C3
:105FA0004FA158A50F94775060935E0B70935F0BD1
:105FB0008093600B9093610B0E94DF788CE0FE0170
:105FC0003196A6E5BBE001900D928A95E1F78091AC
:105FD0002C0881110C94EC4980912A0890912B088F
:105FE0009C012F5F3F4F30932B0820932A08883E57
:105FF000934010F40C94EC4981E080932C081092AB
:106000002B0810922A0880912D0B882309F42AC6A8
:106010000E9423BF811126C6809129088F5F80933B
:10602000290880912908853620F0109229081092BD
:106030002D0BE0912D0B8E2FEE0F990BAA0BBB0BA6
:10604000FC013197E730F10508F0A0C08827EE5831
:10605000FF4F8F4F0D946E500E941BBF882309F491
:1060600095C081E080933E028EEC93E00E947264C2
:1060700080E190E0909332158093311585E0809314
:10608000251502E80093281584E190E1A0E0B0E036
:106090008093291590932A15A0932B15B0932C1556
:1060A0000F94732E81E09AE5909332158093311509
:1060B00086E390E0909334158093331587E08093C6
:1060C00025150093281584E890E0A0E0B0E08093C7
:1060D000291590932A15A0932B15B0932C150F9486
:1060E000732E52C00E941BBF882309F44FC048C0C2
:1060F0008CED93E00E94726481E09AE590933215F2
:106100008093311580E490E090933415809333159B
:1061100007E00093251582E88093281584E890E035
:10612000A0E0B0E08093291590932A15A0932B1539
:10613000B0932C150F94732E00932D0B27C08091D4
:106140002808882319F10E941BBF8823F9F00E94B8
:1061500023BF81111BC089C50E941BBF8823B1F0DA
:106160000E9423BF811112C0AEC50E9423BF8111BE
:106170000DC042E060E070E0CB010E9439BF04C076
:106180000E9423BF811102C010922D0B80913E020C
:10619000882309F43FC58091100890911108892B3C
:1061A00009F091C18091250890912608892B09F06A
:1061B0001EC184E096E0909332158093311580EAF9
:1061C00090E8909334158093331517E010932515BC
:1061D00002E80093281580EA90E0A0E0B0E0809308
:1061E000291590932A15A0932B15B0932C150F9475
:1061F000732E8091060290910702A0910802B0913F
:1062000009020097A105B10511F5109232151092FF
:10621000311515E010932515009328158AE890E1B3
:10622000A0E0B0E08093291590932A15A0932B1538
:10623000B0932C150F94732E89E090E09093321553
:1062400080933115109325150093281540C00196B1
:10625000A11DB11DF5E0B695A79597958795FA957F
:10626000D1F70197A109B109009731E0A307B10562
:1062700058F0B0933215A093311590933415809354
:1062800033151093251507C090933215809331155F
:1062900085E08093251512E8109328158AE890E18F
:1062A000A0E0B0E08093291590932A15A0932B15B8
:1062B000B0932C150F94732E88E090E090933215D4
:1062C0008093311585E080932515109328158CE86F
:1062D00090E1A0E0B0E08093291590932A15A09357
:1062E0002B15B0932C150F94732E8091060290916C
:1062F0000702A0910802B09109020097E1E0AE0701
:10630000B10550F0B0933215A09331159093341528
:106310008093331587E005C0909332158093311533
:1063200085E08093251582E88093281588E890E120
:10633000A0E0B0E08093291590932A15A0932B1527
:10634000B0932C150F94732E809106029091070242
:10635000A0910802B0910902BA2FA92F982F88277F
:106360000097F1E0AF07B10550F0B0933215A0935C
:106370003115909334158093331587E005C09093C1
:1063800032158093311585E08093251512E810931E
:10639000281581EA90E0A0E0B0E080932915909361
:1063A0002A15A0932B15B0932C150F94732E809162
:1063B0002A0B882319F082E090E002C083E090E08D
:1063C000909332158093311585E0809325151093B5
:1063D000281585E490E1A0E0B0E080932915909322
:1063E0002A15A0932B15B0932C150F94732E0091A2
:1063F000250810912608053611057CF410933215F6
:106400000093311585E08093251582E88093281547
:1064100080E090E1A0E0B0E011C0C801845691098D
:10642000909332158093311585E08093251582E88D
:106430008093281581E090E1A0E0B0E080932915D9
:1064400090932A15A0932B15B0932C150F94732EAF
:106450000F5F1F4F1093260800932508093C110574
:1064600074F18AEE93E00E94726481E090E0909370
:1064700011088093100880933E0210920F0881E06B
:106480009AE590933215809331158DE290E09093C8
:1064900034158093331587E08093251582E8809327
:1064A000281584E890E0A0E0B0E08093291590934F
:1064B0002A15A0932B15B0932C150F94732E1092C0
:1064C0002C080C94EC4980910F08882309F4FEC035
:1064D0008091AD149091AE14891B8F7041F40E948D
:1064E000C2C8811104C08091AD1682FFEFC08CE05C
:1064F00090E0909332158093311505E000932515B7
:1065000082E88093281584E190E1A0E0B0E08093D8
:10651000291590932A15A0932B15B0932C150F9441
:10652000732E0E94F3FF20E13EE040E050E00F9424
:10653000E34F2115310581E04807510560F0509384
:10654000321540933115309334152093331587E07D
:106550008093251506C03093321520933115009392
:10656000251502E80093281580E190E1A0E0B0E055
:106570008093291590932A15A0932B15B0932C1571
:106580000F94732E0E94F3FF20E13EE040E050E0C4
:106590000F94E34F2CE330E040E050E00F94E34FE2
:1065A000309332152093311515E010932515009383
:1065B000281582E190E1A0E0B0E080932915909346
:1065C0002A15A0932B15B0932C150F94732E0F94AE
:1065D000E302882399F10F94E3028F5F80932408EC
:1065E000C82ED12C833340F4C601880F991F909395
:1065F00032158093311526C084E690E090933215D1
:106600008093311510932515009328158EE090E1A5
:10661000A0E0B0E08093291590932A15A0932B1544
:10662000B0932C150F94732EC60182539048880F97
:10663000991F90933215809331151AC0109232151C
:106640001092311510932515009328158EE090E1D6
:10665000A0E0B0E08093291590932A15A0932B1504
:10666000B0932C150F94732E109232151092311591
:1066700010932515009328158FE090E1A0E0B0E07D
:106680008093291590932A15A0932B15B0932C1560
:106690000F94732E0F94E30290E090933215809341
:1066A000311585E08093251582E88093281586E1D1
:1066B00090E1A0E0B0E08093291590932A15A09373
:1066C0002B15B0932C150F94732E66C08090740810
:1066D00090907508A0907608B0907708609178083F
:1066E00070917908072E000C880B990B0F94944930
:1066F0002B013C0120E030E040E050E40F94765064
:10670000A50194010F94D75218160CF406C380917A
:10671000A80B9091A90BA091AA0BB091AB0B8D8BFC
:106720009E8BAF8BB88F6091AC0B7091AD0B072E29
:10673000000C880B990B0F9494496B017C0120E0AD
:1067400030E040E251E40F9476502D893E894F8924
:10675000588D0F94D75218160CF4DFC220E030E0A9
:1067600040E050E4C301B2010F947750A5019401B9
:106770000F948D4987FDF1C220E030E040E251E402
:10678000C701B6010F9477502D893E894F89588DE6
:106790000F948D4987FDE1C220E030E048EC52E4DF
:1067A00060914B0B70914C0B80914D0B90914E0B67
:1067B0000F94F3490F94E3517093321560933115A0
:1067C00015E01093251502E80093281586E290E164
:1067D000A0E0B0E08093291590932A15A0932B1583
:1067E000B0932C150F94732E6091A80B7091A90B88
:1067F0008091AA0B9091AB0B0F94E35170933215DB
:1068000060933115109325150093281586E390E1C8
:10681000A0E0B0E08093291590932A15A0932B1542
:10682000B0932C150F94732E6091740870917508B5
:1068300080917608909177080F94E3517093321508
:106840006093311510932515009328158CE390E182
:10685000A0E0B0E08093291590932A15A0932B1502
:10686000B0932C150F94732E8091AC0B9091AD0BBF
:1068700090933215809331151093251500932815A8
:1068800084E390E1A0E0B0E08093291590932A156D
:10689000A0932B15B0932C150F94732E809178082C
:1068A00090917908909332158093311510932515A6
:1068B000009328158AE390E1A0E0B0E080932915C9
:1068C00090932A15A0932B15B0932C150F94732E2B
:1068D00000912108011105C080912308882309F443
:1068E000F8C020E030E048EC52E46091A80B7091D1
:1068F000A90B8091AA0B9091AB0B0F94F3496B01FC
:106900007C016091AC0B7091AD0B072E000C880BD5
:10691000990B0F9494499B01AC01C701B6010F94E8
:1069200071510F94EA516436710510F064E670E01D
:10693000709332156093311545E0A42EA092251571
:1069400052E8B52EB092281584E290E1A0E0B0E0C4
:106950008093291590932A15A0932B15B0932C158D
:106960000F94732EC090A80BD090A90BE090AA0BA7
:10697000F090AB0B20E030E040E253E4C701B601F9
:106980000F94D75218160CF067C0002309F464C0A6
:106990001092210820E030E040E251E460911908B3
:1069A00070911A0880911B0890911C080F94F3496C
:1069B0000F94E3517093321560933115A092251511
:1069C000B092281584E590E1A0E0B0E0809329150D
:1069D00090932A15A0932B15B0932C150F94732E1A
:1069E00020E030E040E251E460911D0870911E0803
:1069F00080911F08909120080F94F3490F94E35160
:106A00007093321560933115A0922515B092281518
:106A100088E590E1A0E0B0E08093291590932A15D5
:106A2000A0932B15B0932C150F94732E80E895E04E
:106A30000E94726481E09AE590933215809331153B
:106A400081E490E0909334158093331587E0809330
:106A50002515B0922815E1C16091AC0B7091AD0B7A
:106A6000072E000C880B990B0F9494499B01AC01E5
:106A7000C701B6010F94D7526091230887FF8FC1D9
:106A8000662339F180912508909126089C012F5F9B
:106A90003F4F309326082093250865E070E00F945F
:106AA0005A50909332158093311585E080932515C7
:106AB00082E8809328158EE890E1A0E0B0E0809312
:106AC000291590932A15A0932B15B0932C150F948C
:106AD000732E80912808882319F18091180801E00D
:106AE000080F0093180890E09093321580933115A9
:106AF00085E08093251582E88093281582E490E153
:106B0000A0E0B0E08093291590932A15A0932B154F
:106B1000B0932C150F94732E0A3010F010921808B1
:106B20008091D9149091DA14A091DB14B091DC1407
:106B30008C34E0E19E07A105B10509F46BC08A34ED
:106B40009041A105B10509F465C080E00E9417C01D
:106B500020E030E040E251E40F94F3490F94E35118
:106B6000709332156093311515E01093251502E8E6
:106B70000093281588E490E1A0E0B0E08093291507
:106B800090932A15A0932B15B0932C150F94732E68
:106B900081E00E9417C020E030E040E251E40F9411
:106BA000F3490F94E35170933215609331151093AC
:106BB0002515009328158AE490E1A0E0B0E08093C9
:106BC000291590932A15A0932B15B0932C150F948B
:106BD000732E82E00E9417C020E030E040E251E4D2
:106BE0000F94F3490F94E35170933215609331156C
:106BF00010932515009328158CE490E1A0E0B0E0F7
:106C00008093291590932A15A0932B15B0932C15DA
:106C10000F94732E35E7C32E35E1D32E0AE189E9AF
:106C200093E10E943B6BE0901608F090170818164D
:106C300019060CF01FC12AE1E216F1040CF4F2C0AF
:106C400019C18CE0FE013196A6E5BBE001900D92E2
:106C50008A95E1F70E94DF7880910A088D7F809302
:106C60000A08B5C910922908DCC984E695E00E949B
:106C700072648091270890E0A0E0B0E0895B9F4FAC
:106C8000AE4FB54A21E03AE53093321520933115E5
:106C9000909334158093331587E08093251582E80F
:106CA0008093281584E890E0A0E0B0E08093291557
:106CB00090932A15A0932B15B0932C150F94732E37
:106CC0001092280861CA81E080933E0210922D0B39
:106CD00082E795E00E94726481E09AE59093321514
:106CE000809331158EE490E09093341580933315A2
:106CF00087E08093251582E88093281584E890E04A
:106D0000A0E0B0E08093291590932A15A0932B154D
:106D1000B0932C150F94732E39CA8DE090E09093A8
:106D200032158093311585E08093251582E8809394
:106D3000281584E190E1A0E0B0E0809329159093BC
:106D40002A15A0932B15B0932C150F94732E8091B8
:106D50002C0B811121C081E01FC084E190E0909351
:106D600032158093311585E08093251582E8809354
:106D7000281584E190E1A0E0B0E08093291590937C
:106D80002A15A0932B15B0932C150F94732E809178
:106D90002C0B811101C082E080932C0BFDCC66236B
:106DA00009F497CE062E000C770B81EB97E00E943A
:106DB0006A6310922308109226081092250881E039
:106DC00080930F0884E090E0909332158093311502
:106DD00085E08093251502E8009328158EE890E160
:106DE000A0E0B0E08093291590932A15A0932B156D
:106DF000B0932C150F94732E81E09AE59093321581
:106E00008093311583E590E090933415809333158A
:106E100087E0809325150093281584E890E0A0E092
:106E2000B0E04DCE89E993E10E94196BF701EB5870
:106E3000FA4E8083809175158A3571F01E141F04F7
:106E40000CF0EDCED601E02F1D92EA95E9F71092F5
:106E5000170810921608E3CE62E070E080E090E040
:106E60000E942BC0FFEFEF1AFF0AF0921708E09282
:106E70001608D5CE1E141F040CF021CB9091D61409
:106E800080917515981322C09091D7148091761532
:106E900098131CC023E0E216F104C4F0909177151A
:106EA0009093D514809178158093D8149330D1F4B1
:106EB000982F9D7F9038B1F4909179159F3409F007
:106EC00059C090917A159B3409F054C08AE1E5E7E6
:106ED000F5E1DF011D928A95E9F7109217081092EB
:106EE0001608EDCA833809F045C080917915909154
:106EF0007A15982789279827A0E0B0E08093D914C5
:106F00009093DA14A093DB14B093DC14C0907B153B
:106F1000D12CE12CF12CC092DD14D092DE14E09241
:106F2000DF14F092E014ACE7B5E140E050E0BA01C4
:106F30004C155D056E057F0508F04AC04A015B01EE
:106F4000B694A79497948794F4013696EE0FFF1F9A
:106F5000EB52FB4E8C9190E0982F882711962C9144
:106F60001197822B918380834E5F5F4F6F4F7F4FCE
:106F70001296DECF813861F58091791590E0A0E01E
:106F8000B0E08093D9149093DA14A093DB14B093FB
:106F9000DC1480917A15482F50E060E070E0409357
:106FA000DD145093DE146093DF147093E014ABE7AC
:106FB000B5E1E1EEF4E190E020E030E02817390798
:106FC00039F04D9150E0419351932F5F3F4FF6CFF1
:106FD0008AE1E5E7F5E1DF011D928A95E9F7109274
:106FE0001708109216088BEF93E00E94726460916C
:106FF0002D0B16165CF4062E000C770B86EA97E034
:107000000E946A638AE00E9404628DC06091E1146C
:107010007091E21484E997E00E9431638AE00E9453
:1070200004624091D9145091DA146091DB1470918C
:10703000DC1485E897E00E9420638AE00E940462E5
:107040008091D9149091DA14A091DB14B091DC14E2
:10705000EBE6F2E000E010E0419151916191719115
:107060004115510561057105D1F1481759076A07A6
:107070007B0791F5AC01BD01485050416109710990
:10708000453051056105710568F1AC01BD01477FCF
:10709000423350416105710541F18433F0E19F07AE
:1070A000A105B10511F1AC01BD0146545041610982
:1070B00071094730510561057105D0F0AC01BD0182
:1070C000445550416109710945305105610571050B
:1070D00088F402E110E00EC00F5F1F4FBDCF0FEF2D
:1070E0001FEF08C003E010E005C008E010E002C098
:1070F0000FE010E08A509042A109B109833D91054B
:10710000A105B10528F00F3F2FEF120719F40BC0AE
:1071100009E110E0FCE1CF2EF4E0DF2E12C004976D
:1071200011F410923E0280E5E5EDF4E1DF011D92DD
:107130008A95E9F78AE58093D61485EA8093D71477
:10714000BEC9F60181916F01882319F00E94046283
:10715000F8CF6AE070E0C8010E945A630E946C6434
:1071600089E797E00E9472640A31110510F00C94CF
:10717000B546F8018827E758FF4F8F4F0D946E50A2
:107180008091E1149091E21481309105E1F4109224
:107190003E028FEF8093621960E080E00F940E351D
:1071A0000AE214E0D8018D918D01882319F00E9424
:1071B0000462F8CF81E09AE59093321580933115FF
:1071C0008EE290E0E8C08230910509F0AEC081E027
:1071D00080933E0210920F080F94540385E797E0C6
:1071E0009093AE088093AD088BE090E090933215B9
:1071F0008093311505E00093251512E810932815AA
:1072000080E092E1A0E0B0E08093291590932A15E8
:10721000A0932B15B0932C150F94732E109232154A
:107220001092311500932515109328158EE090E1EA
:10723000A0E0B0E08093291590932A15A0932B1518
:10724000B0932C150F94732E1092321510923115A5
:1072500000932515109328158FE090E1A0E0B0E091
:107260008093291590932A15A0932B15B0932C1574
:107270000F94732E1092321510923115009325152C
:107280001093281586E190E1A0E0B0E080932915E5
:1072900090932A15A0932B15B0932C150F94732E51
:1072A00062E070E080E090E00E942BC01092321506
:1072B00010923115009325151093281580E190E167
:1072C000A0E0B0E08093291590932A15A0932B1588
:1072D000B0932C150F94732E109232151092311515
:1072E000009325151093281582E190E1A0E0B0E00D
:1072F0008093291590932A15A0932B15B0932C15E4
:107300000F94732E04E514E0F80181918F01882316
:1073100019F00E940462F8CF81E09AE5909332154B
:10732000809331158DE290E036C08330910509F0ED
:10733000F6CE81E080933E0210920F080EE714E033
:10734000D8018D918D018823C9F00E940462F8CF85
:107350008091D9149091DA14A091DB14B091DC14CF
:107360008233F0E19F07A105B10509F030C4809197
:10737000E1149091E214009709F0F8C3809105029E
:10738000882309F4EBC281E09AE59093321580934B
:1073900031158AE390E0909334158093331587E09C
:1073A0008093251582E88093281584E890E0A0E07A
:1073B000B0E00C94CD458091E1149091E2148130BD
:1073C0009105D9F410923E0280910502882319F0AC
:1073D00082E090E002C083E090E0909332158093C9
:1073E000311585E08093251582E8809328158EE17C
:1073F00090E1A0E0B0E00C94CD458230910519F504
:1074000008EA14E0F80181918F01882319F00E94A5
:107410000462F8CF81E080933E0280912C0B84308F
:1074200049F081E09AE5909332158093311585E318
:1074300090E0B1CF81E09AE59093321580933115B9
:1074400086E390E0A8CF8330910509F04AC02091EF
:107450000502222311F1909332158093311585E0B6
:107460008093251582E8809328158EE190E1A0E0B5
:10747000B0E08093291590932A15A0932B15B09313
:107480002C150F94732E40E060E070E088EC92E4DD
:107490000F94D8031092050246CE82E090E09093BC
:1074A00032158093311585E08093251582E880930D
:1074B00028158EE190E1A0E0B0E08093291590932B
:1074C0002A15A0932B15B0932C150F94732E40E022
:1074D00060E070E0CB010F94D80381E08093050257
:1074E00022CE049709F01FCE809187088823E9F007
:1074F00082E090E0909332158093311585E080937F
:10750000251582E8809328158FE190E1A0E0B0E096
:107510008093291590932A15A0932B15B0932C15C1
:107520000F94732E10928708FECD83E090E0909325
:1075300032158093311585E08093251582E880937C
:1075400028158FE190E1A0E0B0E080932915909399
:107550002A15A0932B15B0932C150F94732E81E050
:1075600080938708E0CD6091E1147091E21480E08F
:1075700090E00F9492496B017C0120E030E04AEFEB
:1075800053E40F948D4987FF11C020E030E040E2C2
:1075900051E4C701B6010F94D75218166CF0C12CF4
:1075A000D12C70E2E72E71E4F72E06C0C12CD12C4D
:1075B000EAEFEE2EE3E4FE2EC701B6010F94E3518D
:1075C0007093170260931602AECD8091D9149091FA
:1075D000DA14A091DB14B091DC148830F0E19F073D
:1075E000A105B10509F050C081E09AE590933215EC
:1075F000809331158DE290E090933415809333158C
:1076000087E08093251512E81093281584E890E010
:10761000A0E0B0E08093291590932A15A0932B1534
:10762000B0932C150F94732E1092321510923115C1
:1076300005E0009325151093281580E190E1A0E066
:10764000B0E08093291590932A15A0932B15B09341
:107650002C150F94732E1092321510923115009341
:1076600025151093281582E190E1A0E0B0E0809309
:10767000291590932A15A0932B15B0932C150F94D0
:10768000732E0F9454038EC08A3020E19207A10517
:10769000B105D9F58091E1149091E214813F9105F3
:1076A00009F041CD81E09AE5909332158093311530
:1076B00086E390E0909334158093331587E08093B0
:1076C000251582E88093281584E890E0A0E0B0E0DA
:1076D0008093291590932A15A0932B15B0932C1500
:1076E0000F94732E4AE256E061E376E084E00E9454
:1076F000E2CB60E08DE196E00F94150383E196E024
:107700009093AE088093AD084DC08C309041A10598
:10771000B10509F047C08091E1149091E2140197FE
:1077200009F040C00F947F4310922C0B81E08093AE
:107730003E028CE090E0909332158093311585E005
:107740008093251512E81093281584E190E1A0E0BC
:10775000B0E08093291590932A15A0932B15B09330
:107760002C150F94732E81E09AE590933215809337
:10777000311585E390E0909334158093331587E0BD
:10778000809325151093281584E890E0A0E0B0E0E0
:107790008093291590932A15A0932B15B0932C153F
:1077A0000F94732E8091D9149091DA14A091DB1468
:1077B000B091DC148C309041A105B10509F0B3CC37
:1077C0008091E1149091E214029709F0ACCC0F94EF
:1077D0007F4381E08093230810922C0B80933E021C
:1077E000109226081092250881E09AE590933215B0
:1077F0008093311582E590E0CECD2091E114309157
:10780000E214B90180E090E037FF09C00F9492497B
:1078100020E030E040E857E40F94765002C00F9427
:10782000924920E030E048EC52E40F9471516B0132
:107830007C0120E030E040EA51EC0F94D75287FD04
:1078400031C020E030E040EA51E4C701B6010F94B6
:107850008D4918163CF1A701960160914B0B709170
:107860004C0B80914D0B90914E0B0F94765020E075
:1078700030E048EC53E40F94F34990580F94E351EF
:10788000CB010F94B730C0924B0BD0924C0BE092CF
:107890004D0BF0924E0B80E797E09093AE088093EB
:1078A000AD0841CC20E030E048EC52E460914B0B55
:1078B00070914C0B80914D0B90914E0B0F94F349AE
:1078C0000F94E351709332156093311585E08093E6
:1078D000251582E88093281586E290E1A0E0B0E0CB
:1078E0000C94CD458091E1149091E214009731F40D
:1078F00081E080933E0210920F0815CC81309105F3
:10790000B1F480910502882349F081E09AE59093D3
:107910003215809331158CE390E03DCD81E09AE5FE
:1079200090933215809331158BE390E034CD823003
:10793000910521F481E080933E02F5CB83309105DF
:10794000F9F48091050240E0882389F060E070E05E
:1079500088EC92E40F94D8031092050281E09AE536
:10796000909332158093311589E390E014CD60E057
:1079700070E0CB010F94D80381E08093050203CD22
:107980008530910559F540E060E070E084E393E4D0
:107990000E94AEBE46E060E070E08CE892E40E9497
:1079A000AEBE84EB90E0909332158093311505E0E4
:1079B0000093251512E81093281584E390E1A0E0C8
:1079C000B0E08093291590932A15A0932B15B093BE
:1079D0002C150F94732E86E490E02DC0863091050F
:1079E00099F540E060E070E080E793E40E94AEBE6D
:1079F00046E060E070E08CED92E40E94AEBE80EF65
:107A000090E0909332158093311505E00093251591
:107A100012E81093281584E390E1A0E0B0E0809391
:107A2000291590932A15A0932B15B0932C150F941C
:107A3000732E8EE690E0909332158093311500936B
:107A4000251510932815BEC0813F910509F06BCB19
:107A500040E060E070E0CB010F94D80341E060E0CB
:107A600070E0CB010F94D8031092050240E060E073
:107A700070E0CB010E94AEBE46E060E070E0CB015A
:107A80000E94AEBE109232151092311505E000939F
:107A9000251512E81093281584E390E1A0E0B0E0EA
:107AA0008093291590932A15A0932B15B0932C152C
:107AB0000F94732E61E070E080E090E00E942BC094
:107AC0001092321510923115009325151093281538
:107AD0008AE390E1A0E0B0E08093291590932A1505
:107AE000A0932B15B0932C150F94732E61E070E0CA
:107AF00080E090E00E942BC084E190E090933215EA
:107B000080933115009325151093281584E190E199
:107B1000A0E0B0E08093291590932A15A0932B152F
:107B2000B0932C150F94732E81E09AE59093321543
:107B30008093311589E390E0909334158093331549
:107B400087E0809325151093281584E890E0A0E045
:107B5000B0E08093291590932A15A0932B15B0932C
:107B60002C150F94732E82E00C94B1468130910550
:107B7000B1F440E060E070E0CB010E94AEBE109234
:107B800032151092311585E08093251582E8809397
:107B9000281584E390E1A0E0B0E00C94CD45029775
:107BA00009F0C1CA46E060E070E0CB010E94AEBEC1
:107BB000109232151092311585E08093251582E8D8
:107BC000809328158AE390E1A0E0B0E0E6C7843313
:107BD00020E19207A105B10551F46091E114709183
:107BE000E21480E090E00F94924940E00FC08A33A5
:107BF0009041A105B10509F096CA6091E114709118
:107C0000E21480E090E00F94924946E00E94AEBEFC
:107C10008ACA8091E1149091E214009709F468CE29
:107C20008130910509F04CC080912A0B882319F00E
:107C300083E090E002C082E090E090933215809360
:107C4000311585E08093251582E88093281585E419
:107C500090E1A0E0B0E08093291590932A15A093BD
:107C60002B15B0932C150F94732E8AE090E090930F
:107C700032158093311585E08093251582E8809335
:107C8000281580E092E1A0E0B0E080932915909360
:107C90002A15A0932B15B0932C150F94732E0E94C8
:107CA0001BBF811103C080E697E002C084E597E026
:107CB0009093AE088093AD0882E080932D0B73C142
:107CC0008230910509F0AAC081E080933E021092B3
:107CD0000F0888E0E9E1F8E0DF011D928A95E9F7F5
:107CE00080E090E0A0E2B1E48093190890931A0834
:107CF000A0931B08B0931C0880931D0890931E0846
:107D0000A0931F08B093200884E690E0909332156A
:107D10008093311505E00093251512E8109328157E
:107D200084E590E1A0E0B0E08093291590932A15B6
:107D3000A0932B15B0932C150F94732E20E030E0F8
:107D400040E251E460911D0870911E0880911F0867
:107D5000909120080F94F3490F94E35170933215DA
:107D600060933115009325151093281588E590E14F
:107D7000A0E0B0E08093291590932A15A0932B15CD
:107D8000B0932C150F94732E6091A80B7091A90BD2
:107D90008091AA0B9091AB0B0F94E3517093321525
:107DA00060933115009325151093281586E390E113
:107DB000A0E0B0E08093291590932A15A0932B158D
:107DC000B0932C150F94732E8091AC0B9091AD0B4A
:107DD0009093321580933115009325151093281533
:107DE00084E390E1A0E0B0E08093291590932A15F8
:107DF000A0932B15B0932C150F94732E62E070E0B6
:107E000080E090E00E942BC081E09AE590933215CB
:107E10008093311581E490E00C947747833091058D
:107E200009F076C01092270880E00E9417C020E079
:107E300030E040E251E40F94F3490F94E351709322
:107E400032156093311505E00093251512E8109363
:107E5000281588E490E1A0E0B0E080932915909384
:107E60002A15A0932B15B0932C150F94732E81E037
:107E70000E9417C020E030E040E251E40F94F34943
:107E80000F94E351709332156093311500932515CB
:107E9000109328158AE490E1A0E0B0E080932915C2
:107EA00090932A15A0932B15B0932C150F94732E35
:107EB00082E00E9417C020E030E040E251E40F94DD
:107EC000F3490F94E3517093321560933115009389
:107ED0002515109328158CE490E1A0E0B0E0809384
:107EE000291590932A15A0932B15B0932C150F9458
:107EF000732E62E070E080E090E00E942BC081E091
:107F00009AE5909332158093311587E490E0EFC79E
:107F10008430910509F407C98530910549F44EE78D
:107F200050E160E070E08FEC94E00F94222EFBC8EB
:107F3000069709F0F8C880E597E09093AE08809323
:107F4000AD088BE090E02BC28091E1149091E21497
:107F5000019711F510923E0281E09AE59093321557
:107F6000809331158FE390E090933415809333150F
:107F700087E08093251582E88093281584E890E0B7
:107F8000A0E0B0E08093291590932A15A0932B15BB
:107F9000B0932C150F94732E8091E1149091E214FC
:107FA000029709F0C0C881E09AE59093321580935A
:107FB000311580E490E0EFC9E091E114F091E21412
:107FC0003197EB30F10508F0E4C18827ED56FF4FFB
:107FD0008F4F0D946E508091981380FFCCC686957C
:107FE00080FDCCC6C8C62DEC3CEC4CEC5DE360914A
:107FF0004B0B70914C0B80914D0B90914E0B0F944D
:1080000077506B017C0120E030E040EA51EC0F94A6
:10801000D75287FDC2C120E030E040EA51E4C701F9
:10802000B6010F948D4918160CF0AFC6B6C12DECF1
:108030003CEC4CEC5DE360914B0B70914C0B8091F0
:108040004D0B90914E0B0F9476506B017C0120E00C
:1080500030E040EA51EC0F94D75287FD9EC120E0FA
:1080600030E040EA51E4C701B6010F948D4918167B
:108070000CF0E4C692C180E00E94F15F0E941BBF39
:10808000811103C083E197E002C085E097E09093FF
:10809000AE088093AD0882E080932D0B81E09AE5D5
:1080A000909332158093311584E590E090933415C8
:1080B0008093331587E08093251582E880932815F7
:1080C00084E890E0A0E0B0E08093291590932A1511
:1080D000A0932B15B0932C150F94732E5EC183E0E3
:1080E00080932D0B83E090E09093321580933115AF
:1080F00085E08093251582E8809328158DE890E12E
:10810000A0E0B0E08093291590932A15A0932B1539
:10811000B0932C150F94732EE12CF12C80E001E02C
:10812000AA24A39445E0942E55E0852E62E8762E8D
:10813000002331F0CC24C39435E0B32E10E005C009
:10814000CC24CA94BB24BA9414E00A25B116D9F100
:10815000DD24D394D80E893198F5F701919EE00D76
:10816000F11D1124EE0FFF1FEE0FFF1FEA55F54F13
:1081700020E030E04AE754E460817181828193819C
:108180000F94F3490F94E3517093321560933115B6
:1081900080922515709228158D2D90E08158974F6B
:1081A000880F991F092E000CAA0BBB0B8093291571
:1081B00090932A15A0932B15B0932C150F94732E22
:1081C0001C0D8D2DC3CFBFEFEB1AFB0AE5E0EE16B9
:1081D000F10409F0ADCF81E09AE5909332158093D8
:1081E000311585E590E0909334158093331587E041
:1081F0008093251582E88093281584E890E0A0E01C
:10820000B0E08093291590932A15A0932B15B09375
:108210002C150F94732E86E996E09093AE08809308
:10822000AD08BBC042E060E070E080E890E40E94EE
:1082300039BF40E060E070E08DE193E40E9439BF17
:1082400041E060E070E08BE193E441C042E060E037
:1082500070E080E890E40E9439BF40E060E070E0A8
:1082600080E292E40CC042E060E070E080E890E4DC
:108270000E9439BF40E060E070E089E893E40E942A
:1082800039BF41E060E070E080E292E420C042E06B
:1082900060E070E080E890E40E9439BF40E060E078
:1082A00070E089E893E40CC042E060E070E080E8B0
:1082B00090E40E9439BF40E060E070E080E292E428
:1082C0000E9439BF41E060E070E087E893E40E94DB
:1082D00039BF86E080932D0B60C080912A0B8111FD
:1082E0001CC083E090E0909332158093311585E0B7
:1082F0008093251582E88093281585E490E1A0E01D
:10830000B0E08093291590932A15A0932B15B09374
:108310002C150F94732E81E01BC082E090E09093A7
:1083200032158093311585E08093251582E880937E
:10833000281585E490E1A0E0B0E0809329159093A2
:108340002A15A0932B15B0932C150F94732E80E053
:108350000E94F15F20E030E048EC52E460914B0B6A
:1083600070914C0B80914D0B90914E0B0F94F349F3
:108370000F94E351709332156093311585E080932B
:10838000251582E88093281586E290E1A0E0B0E010
:108390009BCE8AE796E00E9472648AE090E0909318
:1083A00032158093311585E08093251582E88093FE
:1083B00028154CC184E080932D0B8091D9149091A5
:1083C000DA14A091DB14B091DC146091E114709187
:1083D000E2148834F0E19F07A105B10509F454C007
:1083E0008A3420E19207A105B10509F457C08C3405
:1083F00030E19307A105B10509F45BC086349041D3
:10840000A105B10509F05FC063307105B9F589E6D2
:1084100096E09093AE088093AD0881E080932808A1
:1084200080933E021092180881E09AE590933215ED
:10843000809331158AE490E090933415809333153E
:1084400087E08093251512E81093281584E890E0C2
:10845000A0E0B0E08093291590932A15A0932B15E6
:10846000B0932C150F94732E8AE090E09093321500
:108470008093311585E080932515E6C06093270829
:1084800010922D0B0C94933880E090E8ADE9B3E4A2
:10849000898F9A8FAB8FBC8F312C15C080E090E014
:1084A000ABE9B3E4898F9A8FAB8FBC8F33243394BD
:1084B0000AC080E090E0A8ECB3E4898F9A8FAB8F7C
:1084C000BC8F82E0382E80E090E00F94924920E04B
:1084D00030E040E251E40F9471516B017C0120E0E7
:1084E00030E0A9010F948D4987FF09C0109212084E
:1084F0001092130810921408109215081FC0298DAD
:108500003A8D4B8D5C8DC701B6010F94D75218166A
:108510004CF0C0921208D0921308E0921408F09226
:1085200015080CC0898D9A8DAB8DBC8D8093120877
:1085300090931308A0931408B09315086091120843
:10854000709113088091140890911508432D0E9492
:1085500039BF61E070E080E090E00E942BC080E0D5
:108560000E9417C020E030E040E251E40F94F3494C
:108570000F94E351709332156093311505E0009329
:10858000251512E81093281588E490E1A0E0B0E0EA
:108590008093291590932A15A0932B15B0932C1531
:1085A0000F94732E81E00E9417C020E030E040E27B
:1085B00051E40F94F3490F94E35170933215609393
:1085C000311500932515109328158AE490E1A0E059
:1085D000B0E08093291590932A15A0932B15B093A2
:1085E0002C150F94732E82E00E9417C020E030E01B
:1085F00040E251E40F94F3490F94E3517093321524
:108600006093311500932515109328158CE490E1A3
:10861000A0E0B0E08093291590932A15A0932B1524
:10862000B0932C150F94732E61E070E080E090E021
:108630000E942BC010922D0B8AE090E0909332158F
:1086400080933115009325151093281580E092E151
:10865000A0E0B0E0A2C28091D9149091DA14A09168
:10866000DB14B091DC148635E0E19E07A105B1056D
:1086700009F041C020E030E040E253E46091A80BF3
:108680007091A90B8091AA0B9091AB0B0F948D491F
:108690002091E1143091E21487FF34C42530310574
:1086A00008F030C480EA90E0909332158093311541
:1086B00085E08093251512E81093281580E290E15B
:1086C000A0E0B0E08093291590932A15A0932B1574
:1086D000B0932C150F94732E65E070E080E090E06D
:1086E0000E942BC081E09AE590933215809331155A
:1086F00082E490E0FCC38435F0E19F07A105B10559
:10870000C1F46091E1147091E21480E090E00F9464
:10871000924920E030E040E251E40F9471516093BF
:10872000190870931A0880931B0890931C080C94E6
:10873000933888359041A105B10511F00C94933818
:108740006091E1147091E21480E090E00F949249FE
:1087500020E030E040E251E40F94715160931D0835
:1087600070931E0880931F08909320080C949338F0
:108770006091E1147091E21483E596E00E94316308
:108780000C94933882EE94E00E9472648091E1141C
:108790009091E2148130910509F048C080910B0856
:1087A0008230B1F5649902C00C94933881E00E9444
:1087B000CBCA8DE090E0909332158093311585E01F
:1087C0008093251512E81093281584E190E1A0E02C
:1087D000B0E08093291590932A15A0932B15B093A0
:1087E0002C150F94732E83E080932C0B81E09AE577
:1087F000909332158093311585E390E09093341572
:108800008093331587E0809325151093281588C031
:10881000833011F00C94933881E09AE590933215EF
:108820008093311581E490E00C94CB39892B11F0C1
:108830000C94933880EF94E00E94726480910B084E
:10884000813049F587E095E00E94726481E09AE505
:1088500090933215809331158EE290E09093341509
:108860008093331587E08093251582E8809328153F
:1088700084E890E0A0E0B0E08093291590932A1559
:10888000A0932B15B0932C150F94732E10922B0BD5
:108890008CE496E028C0823059F58BE195E00E9487
:1088A000726481E09AE5909332158093311586E3E6
:1088B00090E0909334158093331587E080932515CD
:1088C00082E88093281584E890E0A0E0B0E08093EF
:1088D000291590932A15A0932B15B0932C150F945E
:1088E000732E85E496E09093AE088093AD0826C081
:1088F000833021F58FE295E00E94726481E09AE571
:10890000909332158093311581E490E09093341563
:108910008093331587E08093251582E8809328158E
:1089200084E890E0A0E0B0E08093291590932A15A8
:10893000A0932B15B0932C150F94732E10920B0847
:108940000C9493388091E1149091E2148F3F91053B
:1089500031F028F08FEF90E0A0E0B0E002C0A0E09E
:10896000B0E08093060290930702A0930802B093B0
:1089700009028091060290910702A0910802B0912D
:1089800009020097A105B10509F510923215109260
:10899000311505E00093251512E8109328158AE893
:1089A00090E1A0E0B0E08093291590932A15A09360
:1089B0002B15B0932C150F94732E89E090E09093B3
:1089C000321580933115009325153DC00196A11DE8
:1089D000B11D05E0B695A795979587950A95D1F7AE
:1089E0000197A109B109009731E0A307B10550F043
:1089F000B0933215A09331159093341580933315AD
:108A000087E005C0909332158093311585E08093FF
:108A1000251512E8109328158AE890E1A0E0B0E04F
:108A20008093291590932A15A0932B15B0932C159C
:108A30000F94732E88E090E0909332158093311557
:108A400085E080932515109328158CE890E1A0E02F
:108A5000B0E08093291590932A15A0932B15B0931D
:108A60002C150F94732E8091060290910702A0910D
:108A70000802B0910902BA2FA92F982F88270097D2
:108A8000E1E0AE07B10550F0B0933215A093311577
:108A9000909334158093331587E005C09093321579
:108AA0008093311585E08093251582E88093281501
:108AB00081EA90E0A0E0B0E070C083E495E00E941D
:108AC00072640E94A2BE4091D9145091DA14609150
:108AD000DB147091DC14882309F46BC0433DF0E291
:108AE0005F076105710509F064C014C321303105C9
:108AF00081F480E00F9469432091190830911A089D
:108B000040911B0850911C080F94765040E00F9440
:108B1000404320E030E040E251E460911908709158
:108B20001A0880911B0890911C080F94F3490F9428
:108B3000E351709332156093311505E000932515CC
:108B400012E81093281584E590E1A0E0B0E080934E
:108B5000291590932A15A0932B15B0932C150F94DB
:108B6000732E20E030E040E251E460911D087091E6
:108B70001E0880911F08909120080F94F3490F94CC
:108B8000E3517093321560933115009325151093BE
:108B9000281588E590E1A0E0B0E080932915909336
:108BA0002A15A0932B15B0932C150F94732E0C94AB
:108BB0009338423D50426105710511F00C94933891
:108BC0008091E1149091E214019709F0FBC30E9497
:108BD000A2BE882309F4F6C38091621987FF02C000
:108BE0000C949338A2E18A02C0011124835E944E52
:108BF0000E940B6DC12C90E2D92EE12CF12C05E0E6
:108C000012E8109232151092311500932515109329
:108C10002815C0922915D0922A15E0922B15F092B2
:108C20002C150F94732EBFEFCB1ADB0AEB0AFB0A4D
:108C3000EAE0CE16E0E2DE06E104F10411F700916D
:108C40006219F2E10F02800111240B54164EF80153
:108C500001900020E9F7C8018E1B9F0B439697FDFA
:108C600001967C01F594E7941E141F040CF0A4C334
:108C70009E012F5F3F4F690184E1D9011D928A95C2
:108C8000E9F7A70164E575E0C9010F943D55B80106
:108C9000C6018E0D9F1D0F94285540E050E260E004
:108CA00070E0C6010F94222E62E070E080E090E058
:108CB0000E942BC040E060E070E08FE793E40F94E7
:108CC000D80341E060E070E08FE793E40F94D803AD
:108CD000109205028DE090E090933215809331154B
:108CE00085E08093251512E81093281584E190E122
:108CF000A0E0B0E08093291590932A15A0932B153E
:108D0000B0932C150F94732E62E070E080E090E039
:108D10000E942BC081E09AE5909332158093311523
:108D200085E390E0909334158093331587E080932A
:108D300025151093281584E890E0A0E0B0E080931A
:108D4000291590932A15A0932B15B0932C150F94E9
:108D5000732E81E080933E0280930F0880932B0B4B
:108D600083E080932C0B0C9493388AE396E00E9466
:108D700072640C94933880E497E002C08FE297E02D
:108D80009093AE088093AD08E5CA88E290E00F9416
:108D9000B7302DEC3CEC4CEC5DE360914B0B7091EB
:108DA0004C0B80914D0B90914E0B0F9477506B01B3
:108DB0007C0120E030E040EA51EC0F94D75287FD6F
:108DC00012C020E030E040EA51E4C701B6010F9440
:108DD0008D49181644F0C0924B0BD0924C0BE09288
:108DE0004D0BF0924E0B20E030E048EC52E46091E5
:108DF0004B0B70914C0B80914D0B90914E0B0F943F
:108E0000F3490F94E351709332156093311585E067
:108E10008093251582E88093281586E290E1A0E0F2
:108E2000B0E08093291590932A15A0932B15B09349
:108E30002C150F94732E8AE297E0EFC988ED9FEF0F
:108E40000F94B7302DEC3CEC4CEC5DE360914B0B98
:108E500070914C0B80914D0B90914E0B0F9476506E
:108E60006B017C0120E030E040EA51EC0F94D752D6
:108E700087FD12C020E030E040EA51E4C701B601AE
:108E80000F948D49181644F0C0924B0BD0924C0BA6
:108E9000E0924D0BF0924E0B20E030E048EC52E4B3
:108EA00060914B0B70914C0B80914D0B90914E0B40
:108EB0000F94F3490F94E351709332156093311579
:108EC00085E08093251582E88093281586E290E15D
:108ED000A0E0B0E08093291590932A15A0932B155C
:108EE000B0932C150F94732E85E297E096C990935A
:108EF00034158093331587E080932515109328153A
:108F00000C94D5392430310579F481E00F9469430C
:108F100020911D0830911E0840911F085091200893
:108F20000F94775041E0F3CD2530310518F522300C
:108F3000310571F480E00F94694320911908309154
:108F40001A0840911B0850911C080F947750DECDF1
:108F50002330310508F4CACD81E00F946943209194
:108F60001D0830911E0840911F08509120080F9451
:108F70007650D8CF2630310509F581E09AE59093F7
:108F800032158093311581E490E0909334158093ED
:108F9000331587E08093251582E88093281584E8AF
:108FA00090E0A0E0B0E08093291590932A15A0935B
:108FB0002B15B0932C150F94732EABCD26303105A5
:108FC00008F09BC081E08093210840E060E070E001
:108FD0008EE393E40E94AEBE20E030E048EC52E421
:108FE0006091A80B7091A90B8091AA0B9091AB0B8B
:108FF0000F94F3496B017C016091AC0B7091AD0B48
:10900000072E000C880B990B0F9494499B01AC011F
:10901000C701B6010F9471510F94EA51643671057E
:1090200010F064E670E0709332156093311505E03E
:109030000093251512E81093281584E290E1A0E032
:10904000B0E08093291590932A15A0932B15B09327
:109050002C150F94732E6091A80B7091A90B809121
:10906000AA0B9091AB0B0F94E35170933215609360
:109070003115009325151093281586E390E1A0E0A3
:10908000B0E08093291590932A15A0932B15B093E7
:109090002C150F94732E8091AC0B9091AD0B909387
:1090A000321580933115009325151093281584E30C
:1090B00090E1A0E0B0E08093291590932A15A09349
:1090C0002B15B0932C150F94732E65E070E080E0A3
:1090D00090E00E942BC081E09AE590933215809336
:1090E000311584E490E0909334158093331587E034
:1090F000809325151093281552CF213F310509F093
:1091000008CD1092210861E070E080E090E00E94BC
:109110002BC033CF81EA95E00E947264809163197D
:109120009091641999272091E1143091E2148217EB
:10913000930710F40C9493388CE495E00E947264C9
:109140008091E114815080936219A4ED8A2EA0E2EF
:109150009A2EA12CB12C05E012E810923215109233
:10916000311500932515109328158092291590929A
:109170002A15A0922B15B0922C150F94732E2FEF59
:10918000821A920AA20AB20A3EED831630E29306D0
:10919000A104B10411F780916219A2E18A02C00111
:1091A0001124FC01EB54F64E7F0101900020E9F7F9
:1091B000C7018E1B9F0B439697FD01968C01159559
:1091C000079510161106FCF49E012F5F3F4F6901B1
:1091D00084E1D9011D928A95E9F7A80164E575E05B
:1091E000C9010F943D55B701C601800F911F0F941F
:1091F000285544ED50E260E070E0C6010F94222E45
:1092000005E012E806C044ED50E260E070E0C701FE
:10921000F5CF109232151092311500932515109349
:1092200028158092291590922A15A0922B15B0929C
:109230002C150F94732EBFEF8B1A9B0AAB0ABB0A37
:10924000E6EE8E16E0E29E06A104B10411F78E014F
:109250000F5F1F4F84E1D8011D928A95E9F7809135
:1092600064198F93809163198F938091E2148F9387
:109270008091E1148F938EE595E09F938F931F93D8
:109280000F930F9457554EED50E260E070E0C80127
:109290000F94222E62E070E080E090E00E942BC0EC
:1092A0000FB6F894DEBF0FBECDBF31E2C32E32E160
:1092B000D32EE12CF12C43E1442E40E6542E612CB8
:1092C000712C88248394912CAA24AA94BA2C75E03A
:1092D000272EE2E83E2E0AE010E08091631990917B
:1092E00064198815990594F1B0923215A092311540
:1092F00020922515309228154092291550922A1552
:1093000060922B1570922C150F94732E10933215BA
:10931000009331152092251530922815C0922915F9
:10932000D0922A15E0922B15F0922C150F94732EE3
:10933000FFEF8F1A9F0A20E1420E511C611C711C25
:109340003FEFC31AD30AE30AF30AC7CF8091E114AF
:109350009091E21424E0880F991F2A95E1F78D5F20
:109360009F49A0E0B0E020EF37E83093321520931A
:10937000311505E00093251512E810932815809308
:10938000291590932A15A0932B15B0932C150F94A3
:10939000732E8091E1149091E214805E9D4EA0E0C6
:1093A000B0E026E030E03093321520933115009381
:1093B000251510932815F1CB40E050E260E070E0F5
:1093C000C80170CC8091E1149091E214892B11F4C2
:1093D0000C94783C0C949338A8960FB6F894DEBFA2
:1093E0000FBECDBFDF91CF911F910F91FF90EF90F6
:1093F000DF90CF90BF90AF909F908F907F906F90B5
:109400005F904F903F902F9008952F923F924F92F0
:109410005F926F927F928F929F92AF92BF92CF9204
:10942000DF92EF92FF920F931F93CF93DF93CDB70D
:10943000DEB7C154D1090FB6F894DEBF0FBECDBF61
:1094400022968FAF2297209142082CAF21E02093E3
:109450004208809109128D3409F43CC4843511F41A
:109460000C94B25B873411F00C94B95B80910712B5
:10947000909108128B31910509F41FC2B4F4843025
:10948000910534F482309105DCF597FF2DC01EC4A0
:109490008531910511F40C94BB5B8A31910509F477
:1094A00008C2049709F012C4C5C18A32910509F4B3
:1094B00085C354F48D31910509F43CC20CF42AC2E1
:1094C0004E9709F43BC202C48B35910509F4F4C2EE
:1094D0008C35910509F4F4C28A35910509F0F6C37B
:1094E000109241080C94BB5B80914E02882311F4CA
:1094F0000C94BB5B0F94C40C0E94DF780C94BB5B94
:1095000020914E02222311F40C94BB5B11E00297D0
:1095100009F010E00F94C40C19821A821B821C827D
:109520001D821E821F82188682E50E94369688233D
:1095300009F438C10E94B6954B015C0120E030E08F
:10954000A9010F948D49882309F442C18091690BC8
:1095500090916A0BA0916B0BB0916C0B8CA39DA3A7
:10956000AEA3BFA380916D0B90916E0BA0916F0B7A
:10957000B091700B88A799A7AAA7BBA78091560B9B
:109580009091570BA091580BB091590B8CA79DA7A8
:10959000AEA7BFA780915A0B90915B0BA0915C0B7B
:1095A000B0915D0B88AB99ABAAABBBAB2CA53DA52D
:1095B0004EA55FA56CA17DA18EA19FA10F948D49A1
:1095C00081110DC028A939A94AA95BA968A579A567
:1095D0008AA59BA50F948D49882309F4F9C020E042
:1095E00030E0A901C501B4010F948D49881F882777
:1095F000881F181729F080E090E0A0E8BFEB04C0B6
:1096000080E090E0A0E8BFE388AF99AFAAAFBBAF1E
:109610002CA13DA14EA15FA16CA57DA58EA59FA506
:109620000F9476506CAB7DAB8EAB9FAB28A539A564
:109630004AA55BA568A979A98AA99BA90F94765028
:109640006B017C012CA93DA94EA95FA9CA01B901F2
:109650000F94F3492B013C01A7019601C701B60104
:109660000F94F3499B01AC01C301B2010F947750F1
:109670000F9475532B013C019B01AC0160E070E03D
:1096800080E89FE30F94715121966CAF7DAF8EAF50
:109690009FAF219720E030E040E05FE3C301B201DB
:1096A0000F94F3492B013C01A5019401C501B401BC
:1096B0000F94F3494B015C01A3019201C301B20174
:1096C0000F94F3499B01AC01C501B4010F9476508E
:1096D0000F94755328AD39AD4AAD5BAD0F94F34986
:1096E0004B015C01C701B601905821962CAD3DADF0
:1096F0004EAD5FAD21970F94F349A50194010F94EE
:10970000F3496B017C012CA53DA54EA55FA56CA17D
:109710007DA18EA19FA10F94775020E030E040E022
:109720005FE30F94F3499B01AC01C701B6010F94AD
:1097300077502CA13DA14EA15FA10F947650698373
:109740007A838B839C8328A939A94AA95BA968A538
:1097500079A58AA59BA50F94775020E030E040E0E2
:109760005FE30F94F3496B017C0121962CAD3DAD75
:109770004EAD5FAD21976CA97DA98EA99FA90F94CD
:10978000F349A50194010F94F3499B01AC01C70172
:10979000B6010F94775028A539A54AA55BA50F946B
:1097A000765012C089E40E943696882331F00E94D8
:1097B000B69569837A838B839C838AE40E9436966C
:1097C000882331F00E94B6956D837E838F839887BE
:1097D00020E030E0A90169817A818B819C810F941E
:1097E0008D4981110BC020E030E0A9016D817E819F
:1097F0008F8198850F948D498823A1F0412FBE0158
:109800006F5F7F4F86E59BE00E9405ED0F94B834B3
:10981000609390137093911380939213909393138A
:109820000C94BB5B0E94576282EF97E00E94166225
:109830000C94BB5B80E50E943696882329F00F9438
:10984000F52D6B017C0103C0C12CD12C760183E581
:109850000E943696882361F00E94B69520E030E0A1
:109860004AE754E40F94F3490F94EA516B017C01E9
:109870000E94ED9180912313811105C060E088E082
:1098800098E00F9415030F94B834C60ED71EE81E47
:10989000F91E0F94B834DC01CB018C199D09AE0977
:1098A000BF09B7FD02C00C94BB5B80E00E942E652F
:1098B000F0CF0E9409E00C94BB5B41E061E081E0E5
:1098C0000E946F7881110C94BB5B80E090E0A8E46B
:1098D000B2E489839A83AB83BC8380E090E0A0E20A
:1098E000B1E48D839E83AF83B88789879A87AB87DE
:1098F000BC8780E50E943696882321F00E94A295BD
:10990000862F01C080E0BE016F5F7F4F0F94420041
:109910000C94BB5B80911A0B8770873011F00C940C
:10992000C65B60E08FE40E94F4DF81110C94BB5BA6
:109930000C94C65B0E94C79A0C94BB5B20E030E09D
:1099400048ED51E46091690B70916A0B80916B0B4B
:1099500090916C0B0F947650AB01BC0188E50E948E
:1099600076C16C8F7D8F8E8F9F8F20E030E0A901B4
:1099700060916D0B70916E0B80916F0B9091700BDD
:109980000F947750AB01BC0189E50E9476C19B0121
:10999000AC0169837A838B839C836C8D7D8D8E8DE6
:1099A0009F8D0E9422EB882311F40C94BB5B80E016
:1099B0000E94F15F0E941A8261E085E40E94F4DF58
:1099C000182F01E021E0482FBE016F5F7F4FCE01CD
:1099D0004C960E94478D6B017C019B01AC010F945A
:1099E000C45381115FC08C8C9D8CAE8CBF8C20E0E9
:1099F00030E0A901C501B4010F948D4987FF05C06E
:109A000027E137EB41E558EB04C027E137EB41E5AF
:109A100058E3C501B4010F947750AB01BC0188E352
:109A200098E00E945B6489809A80AB80BC8020E0D3
:109A300030E0A901C501B4010F948D4987FF05C02D
:109A400027E137EB41E558EB04C027E137EB41E56F
:109A500058E3C501B4010F947750AB01BC0183E317
:109A600098E00E945B6420E030E0A901C701B601E4
:109A70000F948D4987FF05C027E137EB41E558EB8F
:109A800004C027E137EB41E558E3C701B6010F9465
:109A90007750AB01BC018EE298E00E945B648AE0E3
:109AA0000E9404620E940182113011F40E945B8CBA
:109AB0000E94BAD90C94BB5B209341080C94BB5B09
:109AC00053ED252E52E0352E6EE0E62E6BE0F62E9D
:109AD00029E63BE03DA32CA37FE3C72E7BE0D72EF6
:109AE00000E010E0D1018D911D010E94369688237F
:109AF00009F44BC00E94B6952B013C01133049F08C
:109B0000F60120813181428153810F9476502B01DF
:109B10003C01ACA1BDA12D913D914D915C91C30142
:109B2000B2010F9476504B015C012DEB37E346E810
:109B300055EB0F94D75287FD0AC02DEB37E346E86B
:109B400055E3C501B4010F948D491816F4F4133090
:109B500051F44092750B5092760B6092770B709295
:109B6000780B01E012C0A5019401F70160817181B9
:109B7000828193810F947750D7016D937D938D935C
:109B80009C931397812F0E9421771F5FB4E0EB0E07
:109B9000F11CECA1FDA13496FDA3ECA3F4E0CF0EE3
:109BA000D11C143009F09ECF002321F085E79BE003
:109BB0000E94FE910E94BAD90C94BB5B80914E0228
:109BC000882311F40C94BB5B89E40E943696182F0D
:109BD000882321F00E94B295E82E01C0E12C8AE48E
:109BE0000E943696F82E882321F00E94B295082F05
:109BF00001C000E0112319F024E02E1520F0FF2011
:109C000041F0053030F080E498E00E9416620C9438
:109C1000BB5B0E94B2DE112359F08E2D0E9480960C
:109C20006093560B7093570B8093580B9093590B7E
:109C3000FF2059F0802F0E94529660935A0B709328
:109C40005B0B80935C0B90935D0B60E080E50E9462
:109C5000F4DF8823C1F01123B1F020E030E048EDBB
:109C600051E46091560B7091570B8091580B909175
:109C7000590B0F9477506093560B7093570B80934A
:109C8000580B9093590B40E050E0BA0186E40E94D3
:109C900076C16B017C0120E030E0A9010F94D7521E
:109CA000181684F420E030E040E752E4C701B60122
:109CB0000F94715160933F02709340028093410270
:109CC000909342020E94DF780C94BB5B0E94F1B13A
:109CD0000C94BB5B80910712909108128337910519
:109CE00011F40C94A0560CF0E1C08934910509F4EC
:109CF00098C40CF069C08A31910509F41DC39CF524
:109D00008431910509F492C27CF48131910509F402
:109D100079C22CF4029708F4EEC10C94AF5B429721
:109D200009F43FC70C94AF5B8731910509F4A8C2D1
:109D30008CF48531910509F49FC2469711F00C947B
:109D4000AF5B0E94F26C8091AD16877F8093AD1659
:109D50000C94BB5B8831910509F4AAC2499709F4B8
:109D6000E0C20C94AF5B8F31910509F413C47CF40D
:109D70008C31910509F458C30CF4ECC28D31910576
:109D800009F45CC34E9709F460C30C94AF5B8A324C
:109D9000910509F41FC464F48032910509F4B4C339
:109DA000819711F00C94AF5B0E94E5C70C94BB5BEC
:109DB0008B32910509F431C4C09711F00C94AF5B5C
:109DC0000F9437040C94BB5B8836910509F453C596
:109DD000D4F58135910509F4D2C6C4F48C349105CB
:109DE00009F42EC44CF48B34910511F00C94AF5B44
:109DF0000E9434900C94BB5B8D34910509F457C4D8
:109E00008E34910509F4A6C40C94AF5B843591059A
:109E100009F4C7C674F48235910509F4BFC68335C9
:109E2000910511F00C94AF5B81E080933B080C949A
:109E3000BB5B8535910509F4E0C68C35910509F4C5
:109E4000F5C60C94AF5B8D36910509F433C58CF4DF
:109E50008A36910509F45BC60CF41FC68B36910552
:109E600009F47DC68C36910511F40C94BB5B0C94FF
:109E7000AF5B8037910511F40C94BB5B54F48E36C4
:109E8000910509F46EC58F36910509F47BC50C94D4
:109E9000AF5B8137910509F4BAC58237910511F09E
:109EA0000C94AF5B0F9489380C94BB5B8E3231E01D
:109EB000930711F40C94CB590CF088C0893C9105A0
:109EC00011F40C94A357DCF58937910509F4E7C721
:109ED000ECF48637910509F4ADC734F48537910564
:109EE00009F497C70C94AF5B8737910509F4D4C781
:109EF0008837910511F00C94AF5B81E080939C084A
:109F000080939B080E94E3D70C94BB5B8B3991052F
:109F100009F4D7C554F48D37910509F42DC68C3852
:109F2000910509F496C50C94AF5B8E3B910509F43D
:109F3000A2C5883C910509F4B9C70C94AF5B833D79
:109F4000910511F40C941B5814F58C3C910511F4F7
:109F50000C94E8573CF48B3C910511F40C94C757D2
:109F60000C94AF5B8D3C910511F40C94F2578E3C30
:109F7000910511F00C94AF5B13EDC12E12E0D12EC0
:109F800000EAE02E08E0F02E10E00C940858823E23
:109F9000910511F40C94815864F48C3D910511F4F1
:109FA0000C941E588D3D910511F40C942B580C9473
:109FB000AF5B8232B1E09B0711F40C94CD588D3227
:109FC000914011F40C94D8580C94AF5B843FF1E0AD
:109FD0009F0711F40C94C25A0CF043C0823931E04F
:109FE000930711F40C94155ADCF48033B1E09B070D
:109FF00011F40C94585914F40C940F5A8039F1E070
:10A000009F0711F40C94125A8139914011F00C946D
:10A01000AF5B81E00E94A38C0E94BAD90C94BB5B19
:10A02000843A31E0930711F40C94285A6CF48A397D
:10A03000B1E09B0711F40C94BB5B8C39914011F497
:10A040000C941D5A0C94AF5B853AF1E09F0711F414
:10A050000C942B5A8C3A914011F40C942E5A0C9477
:10A06000AF5B883532E0930711F40C94255B1CF547
:10A07000873FB1E09B0711F40C94C85A7CF4853FEC
:10A08000F1E09F0711F40C94C55A863F914011F0FE
:10A090000C94AF5B0E94FDD70C94BB5B883F31E012
:10A0A000930711F40C94CF5A8C30924011F40C9415
:10A0B000E05A0C94AF5B8C36B3E09B0711F40C9420
:10A0C000BB5B6CF48B35F2E09F0711F40C94285BBA
:10A0D0008335934011F40C94E85A0C94AF5B803AAA
:10A0E00033E0930709F446C2873E934011F40C9481
:10A0F000A15B0C94AF5B00913A1110913B1180E58C
:10A100000E943696882361F00F94F52D6B017C0137
:10A11000BB24B394672B682B692B31F4B12C04C09A
:10A12000B12CC12CD12C760183E50E943696882370
:10A1300011F40C94655D0E94B69520E030E04AE78A
:10A1400054E40F94F3490F94EA516B017C01B11070
:10A150000BC0672B682B692B39F40115110521F011
:10A16000F8018081811102C0B12C02C0BB24B394DC
:10A170000E94ED91B11003C080EB95E001C0C801D1
:10A180000E944AC11091420883E08093420881E016
:10A190008093641341E758E06AE778E082E00E9428
:10A1A00029CB8FE598E00E944AC1C114D104E10493
:10A1B000F104B1F00F94B834C60ED71EE81EF91E94
:10A1C0000F94B834DC01CB018C199D09AE09BF098D
:10A1D000B7FF0EC08091641381110C946A5D08C0B2
:10A1E00080916413882321F080E00E942E65F8CFCF
:10A1F00080E090E00E944AC11092641310934208DC
:10A200000C94BB5B8091031284FF02C00C946F5DC1
:10A210008091051287FF02C00C946F5D8091061239
:10A22000837011F00C946F5D0C948B5D84EA98E060
:10A230000E9416621092A10A8FE894E10E9478842D
:10A240008BE1EFE8F4E1DE01119601900D928A9521
:10A25000E1F740E050E0BE016F5F7F4F80E090E0AB
:10A260000E94786ECE0101960E94AE8585E998E045
:10A270000E9416620C94BB5B0E94636D0C94BB5BE6
:10A28000E0913A11F0913B118081882329F08032CE
:10A2900009F410823196F8CF40E061E080913A11E4
:10A2A00090913B110E944E70109265130C94BB5B11
:10A2B0008091330A8823E9F080E090E0A0EAB1E4DD
:10A2C00088A399A3AAA3BBA31C8E1D8E1E8E1F8ECE
:10A2D00019821A821B821C8220E0AE01405E5F4F11
:10A2E000BE01645E7F4FCE0101960E94E9CB0C94C3
:10A2F000BB5B0E94C2C8882321F00E94036D0E94AC
:10A30000349040E050E065EB78E085E00E94E2CBDD
:10A3100061E08CE39FE40E946FCA0F94B6030C9433
:10A32000BB5B8091AD1682FF03C08B7F8093AD161F
:10A330000F94A10E0C94BB5B8091AD1683FD02C0FF
:10A340000C94BB5B83E50E94369681110C94995D59
:10A350000C94BB5B83E40E94ED958823D9F189ECD2
:10A3600098E00E94166280913914882351F1BE0151
:10A370006F5F7F4F86E394E10E943F838E010F5F02
:10A380001F4FD8018D918D01882319F00E9404621E
:10A39000F8CFBE016F5F7F4F80E090E00E941670A3
:10A3A00080911319882389F080E20E94046203E1FE
:10A3B00019E1F80181918F01882339F00E9404622C
:10A3C000F8CF8FEB98E00E9416628AE00E94046248
:10A3D0000C94BB5B83E50E943696882309F10E94AA
:10A3E000D0DF182F90E0CD970CF01CE310933208CB
:10A3F0000F94B8346B017C01212F30E0A8EEB3E05C
:10A400000F943750C60ED71EE81EF91EC0922E08B4
:10A41000D0922F08E0923008F09231080C94BB5B88
:10A420000E94CB6C0C94BB5B40E060E080913A11E1
:10A4300090913B110E944E700C94BB5B8091AD16C5
:10A440008E7F8093AD160C94BB5B8091AD1683FD1F
:10A4500002C00C94BB5B0E94D7B18091AD1683FD06
:10A4600002C00C94BB5B60913A1170913B11CE011C
:10A470004C960F94CF2F8C01009711F40C94BB5B7A
:10A480006C8D7D8D19821C8222E0AC01CE0101967B
:10A490000E949189811102C0F12C14C0CE01019655
:10A4A0000F943D2F8823C1F361E0CE0101960E94F5
:10A4B0002383009789F325EEDC012C931C820E94F4
:10A4C0003285F82ECE0101960E94AE85B801FF209C
:10A4D00089F083EF98E00E9444628AE00E9404625F
:10A4E0001092A9161092AA161092AB161092AC16E2
:10A4F0000C94BB5B8BED98E00E94446288ED98E081
:10A500000E9416620C94BB5B8091AD1682FD0E9486
:10A51000ED918091AD1683FD02C00C94BB5B60E0B1
:10A5200080E50E94F4DF182F482F61E080913A11F6
:10A5300090913B110E944E7083E50E9436968823CD
:10A5400081F00E94A295AB01BC014093A9165093E3
:10A55000AA166093AB167093AC1686E394E10E9442
:10A5600039820E94036D11110C94BB5B0E943490E0
:10A570000C94BB5B20913A1130913B119091AD1638
:10A5800092609093AD1640E060E0C9010E944E7069
:10A590000C94BB5B0E94F3FF6C8F7D8F8E8F9F8F1F
:10A5A000BE016F5F7F4FCE014C960E9409C760E0ED
:10A5B000CE0101960F948D030E945B62BE016F5F16
:10A5C0007F4F81E099E00E9444628AE00E94046229
:10A5D0000C94BB5B83E50E943696882311F40C949F
:10A5E000BB5B0E94D0DFF82E6DE070E080E50E943A
:10A5F00043968C0197FF02C00C94BB5BE82E60E091
:10A6000089E40E94F4DF81110C94AA5D802F0E94DE
:10A610008061811193C50C94AA5D0F945F100C9416
:10A62000BB5B80E50E94ED95882311F40C94BB5B25
:10A630008091AD1682FF02C00C94BB5B0C94C35D8D
:10A6400080913A0B813069F482E080933A0B0F9449
:10A65000B8346093360B7093370B8093380B90931C
:10A66000390B83EC95E00E94726481E09AE5909347
:10A6700032158093311587E590E0909334158093DF
:10A68000331587E08093251582E88093281584E8A8
:10A6900090E0A0E0B0E08093291590932A15A09354
:10A6A0002B15B0932C150F94732E0C94BB5B0E944A
:10A6B000E2908AED95E00E94726480912D0B8330C8
:10A6C00011F40C94BB5B0F94540382EF95E00E944D
:10A6D00072648EEF95E00E94726440E060E070E08A
:10A6E000CB010F94D80341E060E070E0CB010F9400
:10A6F000D80381E08093050210922B0B21E030E01B
:10A70000309311082093100880933E0210920F0896
:10A7100081E09AE590933215809331158DE290E0B7
:10A72000909334158093331587E08093251582E844
:10A730008093281584E890E0A0E0B0E0809329158C
:10A7400090932A15A0932B15B0932C150F94732E6C
:10A750000C94BB5B60E070E083E50E9443968E340E
:10A76000910531F40E9453910F94B6030C94BB5B96
:10A770008CE699E00E94166260918B0870918C08BB
:10A7800083E699E00E94316360918D0870918E0894
:10A7900086E599E00E94316360918B0870918C0886
:10A7A00080918D0890918E08681B790B80913A0BEF
:10A7B000815021E030E0823010F020E030E0621B78
:10A7C000730B8BE499E00E9431638AE00E9404627B
:10A7D00083E499E00E94166280918F08909190081E
:10A7E000A0919108B09192088C8F9D8FAE8FBF8FF2
:10A7F000BE016F5F7F4FCE014C960E9409C7BE011C
:10A800006F5F7F4F86E399E00E94446280919308D6
:10A8100090919408A0919508B09196088C8F9D8F87
:10A82000AE8FBF8FBE016F5F7F4FCE014C960E94EF
:10A8300009C7BE016F5F7F4F86E299E00E944462C4
:10A8400020E030E04AE754E460919708709198085E
:10A850008091990890919A080F947151AB01BC01B5
:10A860008EE099E00E945B648DE60E9404628AE0BB
:10A870000E94046280C780913B1083FD7CC70F94C7
:10A88000730D87FD78C783E50E943696882379F09B
:10A890000E94B6950F94E3518B01CB010E94978AD9
:10A8A0000135110524F40E94E2900F94B6030F9431
:10A8B000104361C780913B1083FD5DC70F94730DFA
:10A8C000F82E87FD58C783E50E943696082F811120
:10A8D00006C082E50E943696182F8823C1F10E9497
:10A8E000B6950F94E351CB010E94978A0E94B695CA
:10A8F00020E030E040EA52E40F948D49181614F439
:10A900000C94CE5D0E94E2900F94B6036091AC0B64
:10A910007091AD0B072E000C880B990B0F94944986
:10A920004B015C014090A80B5090A90B6090AA0BC2
:10A930007090AB0BA30192010F94D752181614F428
:10A940000C94E15D002311F40C94D25D11E00F949E
:10A950001043112309F40FC7602F8F2D0E941DF3A0
:10A960000AC78EE40E943696882309F404C70E9421
:10A97000A29560938C1270938D1280938E12909397
:10A980008F12F9C683E50E94ED95882331F060E0CF
:10A9900083E50F942B0480933B100E945B628CE94B
:10A9A00099E00E94166280913B10882369F142E988
:10A9B000E42E49E0F42E00E010E020E080913B100E
:10A9C00090E0A0E0B0E0002E04C0B695A795979562
:10A9D00087950A94D2F780FF0EC0DD24D394D20E5F
:10A9E000222319F08CE20E940462F7018591949170
:10A9F0000E9416622D2D0F5F1F4FB2E0EB0EF11C6F
:10AA000005301105D9F6E1CC8EE899E0DCCC83E580
:10AA10000E943696882371F00E94D0DF282F30E004
:10AA20002D3331051CF480930002A5C68CE380937E
:10AA30000002A1C60E945B624091000250E060E00B
:10AA400070E083EA99E00E9420638AE00E94046239
:10AA500092C680913B1083FD8EC683E50E94369698
:10AA6000882309F488C60E94B6950F94E351CB0160
:10AA70000E94A4DE80C680913B1083FD7CC683E5E6
:10AA80000E943696182F81110C94E45D82E50E9495
:10AA9000369681110C94E45D6EC60F94730D182FD9
:10AAA00087FD0AC088EC99E00E941662812F0E94FF
:10AAB0002DF18AE00E940462ECADE09342080C9410
:10AAC000D75F83E50E943696882309F454C60E9416
:10AAD000D0DF182F90E0CD970CF01CE310933708CF
:10AAE0000F94B8346B017C01212F30E0A8EEB3E065
:10AAF0000F943750C60ED71EE81EF91EC0923308B9
:10AB0000D0923408E0923508F092360834C660E0FE
:10AB100080E50F942B04F82EF1E0F81708F42BC60B
:10AB200081E40E94ED95882321F06091910B062F1E
:10AB300002C00FEF10E083E50E943696882349F0AB
:10AB40000E94A2958B016F3F710519F010F00FEF75
:10AB500010E0EF2DF0E0EF56F44F00830CC660E0FC
:10AB600080E50F942B04823008F005C6E82FF0E052
:10AB7000EF56F44F1082FFC50F94A10EFCC50E9442
:10AB8000C2F80E94E2900E942E930E94C26168EE79
:10AB900073E080E090E00E945C61EDC510923B089C
:10ABA000EAC583E50E943696882399F00E94B695FF
:10ABB00020E030E04AE754E40F94F3490F94EA515F
:10ABC0006093010270930202809303029093040247
:10ABD000D2C58091031284FF02C00C94195E80914B
:10ABE000051287FF02C00C94195E809106128370D3
:10ABF00011F00C94195E0C94495E83E50E94ED956A
:10AC0000882309F4B8C50E94B69520E030E04AE7F1
:10AC100054E40F94F3490F94EA5160933C08709305
:10AC20003D0880933E0890933F08A5C50F94730D8F
:10AC300087FDA1C59091031294FD04C09091051267
:10AC400097FF0AC023EDC22E22E0D22E3CE3E32E72
:10AC500030E1F32E10E009C090910612937091F745
:10AC6000682F81E00F94241086C5D6018D916D0167
:10AC70000E943696882309F459C0133009F04FC05A
:10AC80000E94B6954B015C0120E030E040EA51E4BF
:10AC90000F948D4987FF3AC0A501940160915C1023
:10ACA00070915D1080915E1090915F100F947151C2
:10ACB0002B013C019B01AC0160916C1070916D10F7
:10ACC00080916E1090916F100F94F34960936C1007
:10ACD00070936D1080936E1090936F106091890B3C
:10ACE00070918A0B80918B0B90918C0B0F949249F1
:10ACF000A30192010F94F3490F94EA516093890BD9
:10AD000070938A0B80938B0B90938C0B80925C10CA
:10AD100090925D10A0925E10B0925F1007C00E94EA
:10AD2000B695F701648B758B868B978B1F5FF4E06C
:10AD3000EF0EF11C143009F098CF0E94C9911BC589
:10AD40008FEE9AE00E94166260E08FED9AE00E941A
:10AD5000E2F060E08AEC9AE00E94E2F061E083ECCD
:10AD60009AE00E94E2F061E088EB9AE00E94E2F053
:10AD700061E088EA9AE00E94E2F060E08FE99AE000
:10AD80000E94E2F061E085E99AE00E94E2F061E071
:10AD90008BE89AE00E94E2F061E083E89AE00E948A
:10ADA000E2F061E085E79AE00E94E2F061E087E688
:10ADB0009AE00E94E2F060E088E59AE00E94E2F00A
:10ADC00060E08AE49AE00E94E2F060E084E39AE0C6
:10ADD0000E94E2F061E083E29AE00E94E2F061E02A
:10ADE00084E19AE00E94E2F061E08FEF99E00E9436
:10ADF000E2F061E08CEE99E00E94E2F060E08FED1D
:10AE000099E00E94E2F060E08BEC99E00E94E2F0B1
:10AE1000B2C480913A1190913B11009741F0DC014E
:10AE20002C91222321F060E00F948D03A4C40F9491
:10AE3000B603A1C400913A1110913B1183E0F12CAB
:10AE400040E08150E1F0F8019081292F2B7F2134DF
:10AE5000C1F721812133A9F7913421F0953421F4F0
:10AE600041E002C0FF24F39498012E5F3F4F890117
:10AE70002F5F3F4FD8019C919032C9F3E2CF41112F
:10AE80000E945B62FF2021F08EED9BE00E94166223
:10AE9000C8010E9472646FC40E94C0D76CC4109233
:10AEA0009C0810929B080E94E3D765C40F94730D11
:10AEB000182F87FD60C484E40E94ED95882309F46F
:10AEC0003FC00E94B6956B017C0101E020E030E0BC
:10AED000A9010F948D49811101C000E000931B0B63
:10AEE00020E030E0A901C701B6010F948D49882305
:10AEF00039F10E94B695B4E01B02F0011124E05E26
:10AF0000F44F608371838283938320E030E0A90152
:10AF10006091200B7091210B8091220B9091230B5B
:10AF20000F948D4981110CC080E090E0A0EEBFE34A
:10AF30008093200B9093210BA093220BB093230BB3
:10AF40000E94557418C40F94730D87FD14C493EDBB
:10AF5000E92E92E0F92E0CE310E1F70181917F01D7
:10AF60000E94ED95882351F00E94B6950F94EA5106
:10AF7000D8016D937D938D939C9313970C5F1F4F16
:10AF8000B0E10C341B0749F70E948291F4C30F947F
:10AF9000730D87FDF0C383EDE82E82E0F82E0CE3FD
:10AFA00010E1F70181917F010E94ED95882349F01E
:10AFB0000E94B695D80194966D937D938D939C9342
:10AFC00097970C5F1F4FB0E10C341B0751F7D3C3A9
:10AFD0008091041287FD60C6809105128E7009F081
:10AFE0005BC6A0C68091031281FDC4C68091041285
:10AFF00081FDC0C6809105128C7009F0BBC6BBC331
:10B000001F5FB4E0EB0EF11C133011F40C94DA4D19
:10B01000F60181916F010E94ED95882389F30E94CA
:10B02000B695D7016D937D938D939C931397812F44
:10B030000E942177E5CF0F946F0F9DC383E50E9497
:10B040003696882309F497C30E94B295909317020D
:10B050008093160290C30F94730DF82E87FD8BC357
:10B0600083E50E9436960F2D0F2C000C110B8823C0
:10B0700069F10E94B295F801EE0FFF1FE05DFD4FF0
:10B0800091838083000F111F000F111FF801ED5BEA
:10B09000FD4F7F01BC01990F880B990B0F949449C8
:10B0A0002AE037ED43E25CE30F94F349F801E45EF4
:10B0B000F44F20813181428153810F94F349D701AC
:10B0C0006D937D938D939C93139755C30E945B6200
:10B0D00085E40E94046280E38F0D0E940462F801FF
:10B0E000EE0FFF1FE05DFD4F6081718187E19CE005
:10B0F0000E946A6385E20E9404628AE00E94046200
:10B100003AC380E50E94ED95882309F434C360E0DA
:10B1100070E080E50E944396F82E6FEF7FEF83E5A5
:10B120000E9443968C010196039708F024C3F7FC14
:10B1300022C38F2D0E948061882339F00E945762BC
:10B140008FE19CE00E94166216C30E94ED9160E0C0
:10B150008F2D0F945A330F3FBFEF1B0731F0013093
:10B16000110571F000E010E00DC08F2D0F94023337
:10B1700031E020E0892B09F030E0032F122F02C0CC
:10B1800001E010E08F2D0F9402338017910709F42E
:10B19000F2C280E00E942E65F5CF8AE50E943696C5
:10B1A000811141C683E50E94369681113CC6E3C2F7
:10B1B00060E085E40F942B04811173C080E50E9448
:10B1C000ED95882351F00E94B6956093AF0B709374
:10B1D000B00B8093B10B9093B20B89E40E94ED9574
:10B1E000882381F00E94B6952CEA35EC47E25EE3B5
:10B1F0000F94F3496093B30B7093B40B8093B50B2A
:10B200009093B60B84E40E94ED95882381F00E9410
:10B21000B6952CEA35EC47E25EE30F9471516093EA
:10B22000B70B7093B80B8093B90B9093BA0B0E9435
:10B230005B624091AF0B5091B00B6091B10B70917C
:10B24000B20B89E59CE00E945B642CEA35EC47E296
:10B250005EE36091B30B7091B40B8091B50B90914C
:10B26000B60B0F947151AB01BC0185E59CE00E94C7
:10B270005B642CEA35EC47E25EE36091B70B7091BA
:10B28000B80B8091B90B9091BA0B0F94F349AB01B5
:10B29000BC0181E59CE00E945B648AE00E9404623C
:10B2A0006AC20E9457628FE39CE00E94166263C2EA
:10B2B00080E50E94ED95882351F00E94B695609339
:10B2C0007B0870937C0880937D0890937E0889E4C6
:10B2D0000E94ED95882381F00E94B6952CEA35EC0A
:10B2E00047E25EE30F94F34960937F087093800810
:10B2F000809381089093820884E40E94ED958823CE
:10B3000081F00E94B6952CEA35EC47E25EE30F949B
:10B31000715160938308709384088093850890939B
:10B3200086080E945B6240917B0850917C08609186
:10B330007D0870917E0885E69CE00E945B642CEAA3
:10B3400035EC47E25EE360917F0870918008809160
:10B350008108909182080F947151AB01BC0181E684
:10B360009CE00E945B642CEA35EC47E25EE360916E
:10B3700083087091840880918508909186080F94C5
:10B38000F349AB01BC018DE59CE00E945B648AE05F
:10B390000E940462F0C183E50E94ED95182F882376
:10B3A00071F00E94B6950F94E35170934802609338
:10B3B000470221E0672B09F020E02093A30B80E5F2
:10B3C0000E94ED95882359F0209147023091480260
:10B3D000232B11F00E94E4DF8093A30BCCC1111149
:10B3E000CAC10E945B6285E89CE00E94166280915F
:10B3F000A30B882319F08DE69CE002C089E69CE04F
:10B400000E941662609147027091480284E79CE0B6
:10B410000E946A6380E79CE00E941662ACC10E94B1
:10B420008DC1A9C10E94ED91A6C180E00E94A38CAC
:10B430000E945B8C0E94BAD99EC1809103128878C9
:10B4400009F056C580910512867009F051C580C576
:10B450000F946C0990C10F949E088DC141E061E08A
:10B4600081E00E946F78811186C109EF13E3E9E65C
:10B47000FBE0FDA3ECA39E012F5F3F4F49014EE48B
:10B48000A42E44E3B42E1901F801659175918591BC
:10B490009491ACA1BDA1CD90DD90ED90FD90BDA3A8
:10B4A000ACA3A70196010F9476502B013C01F1014A
:10B4B000608371838283938320E030E040EA51EC23
:10B4C0000F94D75287FD0AC020E030E040EA51E4F3
:10B4D000C301B2010F948D4918162CF4F501849123
:10B4E00018160CF459C5D101CD90DD90ED90FD906A
:10B4F0001D0120E030E040EA51ECC701B6010F9495
:10B50000D75287FD0AC020E030E040EA51E4C7018D
:10B51000B6010F948D49181664F40E9457628EEE9E
:10B520009CE00E94166261E080EE9CE00F9415039F
:10B5300022C10C5F1F4FBFEFAB1ABB0AE4E305301B
:10B540001E0709F0A1CF30EAE32E38E0F32E10E019
:10B55000F40181919191A191B1914F01F7018193F2
:10B560009193A193B1937F01812F0E9421771F5F57
:10B57000133071F70E94BAD960E080ED9CE00F941F
:10B580001503F9C00E9493FAF6C00F94DC17F3C0BC
:10B5900061E083E50E94F4DF0E946BDAECC081E099
:10B5A000809373130F94E61110927313882309F498
:10B5B000E2C00E945B628CE09DE00E941662DBC0EC
:10B5C0008091AD1682FFD7C080628093AD16D3C044
:10B5D0008AE50E943696882331F10E94B6956B0168
:10B5E0007C0120E030E040EA51EC0F94D75287FD17
:10B5F00013C020E030E040EA51E4C701B6010F94E7
:10B600008D4918164CF0C0924B0BD0924C0BE09227
:10B610004D0BF0924E0BAFC00E94576287E19DE048
:10B620000E941662A8C00E945B6240914B0B509131
:10B630004C0B60914D0B70914E0B84E39DE00E948A
:10B640005B648AE00E94046296C00F949A0D93C0D6
:10B650000F94730D082F87FD8EC085E50E94ED9530
:10B660008823B1F1E02E002E000CFF080E94B69551
:10B670004B015C0120E030E0A9010F94D75287FF15
:10B6800004C0B7FAB094B7F8B094C70123E0880FAC
:10B69000991F2A95E1F79C01225A3E4E7901D90162
:10B6A0008D929D92AD92BC92139720E030E04AEFCC
:10B6B00053E4C501B4010F94D75218164CF480E03E
:10B6C00090E0AAEFB3E4F70180839183A283B38370
:10B6D0008CE40E94ED95882309F44DC0002E000CE7
:10B6E000110B0E94B6956B017C0120E030E0A901AE
:10B6F0000F94D75287FF04C0F7FAF094F7F8F0944C
:10B7000020E030E04AEF53E4C701B6010F94D7526E
:10B71000980193E0220F331F9A95E1F7F901E25A5D
:10B72000FE4E18162CF0C482D582E682F78223C022
:10B7300080E090E0AAEFB3E484839583A683B78387
:10B740001AC081E080934E021092631360E083E59B
:10B750000E94F4DF81110FC00E94A9E80CC00E9472
:10B76000F1B109C080910712882329F00E94828AD2
:10B7700002C00E94F1B12296FFAD2297F11102C0E2
:10B780000E9454E82CAD2093420811C40E94ED9110
:10B7900030912A0B3CAB80E00E94F15F0E941A823C
:10B7A00081E080939C080E94E3D788E50E94ED9594
:10B7B000182F89E50E94ED95082F8AE50E94ED95E6
:10B7C000101381C1181711F0012F7DC101E011E0A4
:10B7D00091E09CA70E94B2DE82E50E943696882303
:10B7E00061F00E94B6956B017C0120E030E0A90178
:10B7F0000F948D49882369F106C0C12CD12CE0E853
:10B80000EE2EE0E4FE2E111103C0002309F4FCC06B
:10B81000C0925E0BD0925F0BE092600BF092610BD6
:10B82000A70196016091710B7091720B8091730B5F
:10B830009091740B0F948D4987FF0BC019821A8267
:10B840001B821C82BE016F5F7F4F8EE59BE00E94D2
:10B85000A8D6112309F4D3C0002309F4CDC0109257
:10B860006D0B10926E0B10926F0B1092700B10926A
:10B87000690B10926A0B10926B0B10926C0B0E946A
:10B8800051D7EEE4F4E3A491A8AFE2E4F4E3C59069
:10B89000D590E590F490E6E4F4E385909590A5903A
:10B8A000B490A5019401C701B6010F94D7521816A0
:10B8B0002CF4A7019601C501B40104C0A5019401AF
:10B8C000C701B6010F9471512B013C01E9E0F4E38B
:10B8D00085919591A591B4918CA39DA3AEA3BFA38F
:10B8E000E5E0F4E385919591A591B49188A799A796
:10B8F000AAA7BBA79C01AD016CA17DA18EA19FA1B0
:10B900000F94D752181634F428A439A49AA598ABEA
:10B910001BA505C02CA03DA0AEA1A8AB1FA1A301F3
:10B920009201C301B2010F94F34920E030E040E8F6
:10B930005FE30F9477500F947553910148A9512FED
:10B940000F94F34968A379A38AA39BA3EFE4F4E3DC
:10B95000149120E030E040EC5FE3C501B4010F94A6
:10B96000F3494B015C01612F110F770B880B990B89
:10B970000F9494499B01AC01C501B4010F94F349A4
:10B9800069837A838B839C8320E030E040EC5FE323
:10B99000C701B6010F94F3496B017C01B8AD6B2F61
:10B9A000BB0F770B880B990B0F9494499B01AC014B
:10B9B000C701B6010F94F3496C8F7D8F8E8F9F8FD7
:10B9C000AE01405E5F4FBE016F5F7F4FCE014C9670
:10B9D0000E9486D60E94F2D710926D0B10926E0BC9
:10B9E00010926F0B1092700B1092690B10926A0BF1
:10B9F00010926B0B10926C0B80E00E944177002339
:10BA000019F081E00E944177ECA5EE2309F44DC0C6
:10BA1000809198138370833061F060E080E298E059
:10BA20000F9415030E945B6281E198E00E94166208
:10BA30003AC00E9451D780E090E0A8E4B2E480933D
:10BA40005A0B90935B0BA0935C0BB0935D0B8091B2
:10BA5000710B9091720BA091730BB091740B80934A
:10BA60005E0B90935F0BA093600BB093610B80E033
:10BA700090E0AAE9B2E48093560B9093570BA09301
:10BA8000580BB093590B19821A821B821C82AE018B
:10BA90004F5F5F4F6AE57BE086E59BE00E9486D6BC
:10BAA00082E00E9441770E945B8C0E9451D7809176
:10BAB0009B0880939C088CA90E94F15F0E940182E0
:10BAC0000E94BAD958CE8CA785CEB1100C94B45030
:10BAD0000C94AD5080E00E942E650C94E05088E5F7
:10BAE0000E94ED9581115F9889E50E94ED95811185
:10BAF0008A988AE50E94ED95882329F080910801B3
:10BB000081708093060185E40E94ED95882309F4F5
:10BB100032CE129830CE60E08CE898E00F94150396
:10BB20005F988A988091080181708093060112982D
:10BB300022CE0E94A295AB01BC014093A91650935E
:10BB4000AA166093AB167093AC1686E394E10E943C
:10BB5000398211CE61E0802F0F945A336F2D802FE0
:10BB60000F942B336F2D70E0802F0F94963387E066
:10BB7000E81203C0F092920BFECD99E0E912FBCDE2
:10BB8000F092910BF8CD0E94D0DF90E085369105C0
:10BB900014F084E690E080936513EDCD0E9434901C
:10BBA0000C948654A3019201C501B4010F94D7529D
:10BBB00018163CF084E799E060E00F9415030C94AC
:10BBC000A65481E899E0F8CF0E94B6950F94E3510E
:10BBD000CB010E94A4DE0E94B69520E030E040EA4E
:10BBE00050E40F94D752181614F40E9434906091C8
:10BBF000780870917908072E000C880B990B0F9428
:10BC000094492091740830917508409176085091BC
:10BC100077080F94D75218161CF489EB99E002C0EC
:10BC20008AEA99E060E00F941503812F0E949FF14A
:10BC3000A2CD0E94ED9188E50E94ED95882331F018
:10BC40005F9A809198138E7F8093981389E50E9464
:10BC5000ED95882331F08A9A809198138D7F809397
:10BC600098138AE50E94ED95882359F08091080188
:10BC70008095817080930601809198138B7F8093CB
:10BC8000981385E40E94ED95882309F474CD129AE7
:10BC900072CD0E942E936FCD83E50E943696882345
:10BCA00091F00E94B695609370107093711080931C
:10BCB0007210909373106093781070937910809342
:10BCC0007A1090937B1080E50E943696882351F07D
:10BCD0000E94B695609370107093711080937210EB
:10BCE0009093731082E50E943696882351F00E944B
:10BCF000B69560937410709375108093761090933E
:10BD0000771084E50E943696882309F434CD0E948A
:10BD1000B695609378107093791080937A10909311
:10BD20007B1029CD4091701050917110609172106C
:10BD30007091731088EE9BE00E945B6440917410D8
:10BD400050917510609176107091771085EE9BE0A0
:10BD50000E945B64409178105091791060917A1044
:10BD600070917B1082EE9BE00E945B648AE00E94EF
:10BD7000046201CD82E40E94ED95882351F00F9476
:10BD8000F52D60934C1070934D1080934E1090934E
:10BD90004F1083E50E94ED95882351F00E94B695DF
:10BDA00060937C1070937D1080937E1090937F1031
:10BDB00084E50E94ED95882351F00E94B69560932A
:10BDC00080107093811080938210909383108AE486
:10BDD0000E94ED95882309F4CECC0E94B6956B01A4
:10BDE0007C012AE037ED43E25CE30F94D75287FDF4
:10BDF00013C02AE939E949E95EE3C701B6010F94A6
:10BE00008D4918164CF0C092790BD0927A0BE092C3
:10BE10007B0BF0927C0BAFCC0E94576288EF9BE0CB
:10BE20000E941662A8CC0E94B69520E030E040E067
:10BE300050EC0F948D4987FD15C00E94B69520E007
:10BE400030E040E050E40F94D75218162CF00E94D6
:10BE5000B6956B017C010BC0C12CD12CE12C60E4A8
:10BE6000F62E05C0C12CD12CE12C50ECF52E2091E2
:10BE700058103091591040915A1050915B10C701E1
:10BE8000B6010F94F3490F94E351CB010F94B730EF
:10BE900080E50E94ED95882329F00E94E4DF882345
:10BEA00009F469CCA701960160914B0B70914C0B82
:10BEB00080914D0B90914E0B0F94775060934B0BEC
:10BEC00070934C0B80934D0B90934E0B0E945B62D2
:10BED00040914B0B50914C0B60914D0B70914E0B60
:10BEE0008EE29CE00E945B648AE00E94046243CC84
:10BEF00088E40E94ED95882321F00E94E4DF80937E
:10BF0000400882E50E94ED95082F83E50E94ED959B
:10BF1000182F011102C0882351F010926E080E9460
:10BF2000A561112321F00E94E4DF8093490284E49B
:10BF30000E94ED95882309F41ECC0E94B69560936B
:10BF4000540270935502809356029093570213CC7B
:10BF50000E945B628FEB9CE00E9416628091490216
:10BF6000811117C088E99CE00E9416628AE00E9455
:10BF700004624091540250915502609156027091B2
:10BF800057028FE99CE00E945B648AE00E94046291
:10BF9000F2CB8CE99CE0E8CFF7FAF094F7F8F09454
:10BFA000D101CD92DD92ED92FC9213979CCACF5BAA
:10BFB000DF4F0FB6F894DEBF0FBECDBFDF91CF913C
:10BFC0001F910F91FF90EF90DF90CF90BF90AF90B7
:10BFD0009F908F907F906F905F904F903F902F90A9
:10BFE000089590912A0B9817D1F00E94ED918091BD
:10BFF0002A0B882359F041E75BE06DE67BE089E698
:10C000009BE00E94137410922A0B07C081E080937A
:10C010002A0B89E69BE00E94AB930C9451D70895BC
:10C0200080E00E94F15F60E070E080EC9FE70C949C
:10C03000929A1F93CF93DF9310912A0B80E00E9476
:10C04000F15F8FEF8093661180E090E0A0E2B1E4B1
:10C0500080930A0B90930B0BA0930C0BB0930D0BDA
:10C060008DEC9CECACECBDE380933E1190933F11C2
:10C07000A0934011B093411180EF9FEFA9E7B4EC7A
:10C080008093421190934311A0934411B0934511B2
:10C0900084E6E6EAFAE0DF011D928A95E9F7C0E05E
:10C0A000D0E020E030E0A9016D2F8C2F0E9446C027
:10C0B000DF5FD530B1F7CF5FC53091F7112329F09D
:10C0C000DF91CF911F910C94BAD9DF91CF911F913D
:10C0D0000895CF92DF92EF92FF920F931F93CF9329
:10C0E000DF93CDB7DEB72C970FB6F894DEBF0FBE47
:10C0F000CDBF7B018C01D42E9B01AC0160910A0B5A
:10C1000070910B0B80910C0B90910D0B0F948D493E
:10C11000882309F496C0C0902A0B80E00E94F15F4A
:10C1200020E030E0A901B701C8010F94D7521816DA
:10C1300024F0E12CF12C00E010E0C701D80180933D
:10C140000A0B90930B0BA0930C0BB0930D0B2DEBE4
:10C1500037E346E855EBB701C8010F94D75287FD86
:10C160000AC02DEB37E346E855E3B701C8010F9449
:10C170008D4918164CF49701A80160E070E080E842
:10C180009FE30F94715103C060E070E0CB016093B6
:10C190003E1170933F11809340119093411180EFB5
:10C1A0009FEFA9E7B4EC8093421190934311A093C1
:10C1B0004411B0934511CC2009F443C08091690B20
:10C1C00090916A0BA0916B0BB0916C0B89839A8351
:10C1D000AB83BC8380916D0B90916E0BA0916F0B24
:10C1E000B091700B8D839E83AF83B8878091710B64
:10C1F0009091720BA091730BB091740B89879A8701
:10C20000AB87BC8781E00E94F15FDD20D1F04CE07C
:10C2100050E069E67BE0CE0101960F94E954892B4A
:10C2200081F02C960FB6F894DEBF0FBECDBFDF9124
:10C23000CF911F910F91FF90EF90DF90CF900C94D2
:10C24000BAD92C960FB6F894DEBF0FBECDBFDF91E2
:10C25000CF911F910F91FF90EF90DF90CF900895B5
:10C26000EF92FF921F93CF93DF9386EAE82E8AE046
:10C27000F82E15E0C0E0D0E0F701EC0FFD1F608163
:10C280007181828193819B01AC010F94C453811110
:10C290000CC02496C431D10579F7115084E1E80E21
:10C2A000F11C1111E7CF81E001C080E0DF91CF9157
:10C2B0001F91FF90EF900895CF92DF92EF92FF923F
:10C2C0006B017C0183E3C816D104E104F10470F032
:10C2D00082E3C81AD108E108F10862E370E080E067
:10C2E00090E00F947E340E942CB3ECCFC701B601CE
:10C2F0000F947E34FF90EF90DF90CF900C942CB38E
:10C30000FF920F931F93CF93DF931F92CDB7DEB7AA
:10C31000F82E0FE91FE241E050E0B801CE0101968E
:10C320000F94C74889818F1102C081E007C00F5F59
:10C330001F4F8FE2083B180771F780E00F90DF91E5
:10C34000CF911F910F91FF90089580915402909189
:10C350005502A0915602B091570280939C10909381
:10C360009D10A0939E10B0939F1008958091500847
:10C37000811107C00F94DC17882319F081E08093A6
:10C3800050080895E1E9FBE01082118208958F9230
:10C390009F92AF92BF92CF92DF92EF92FF920F9354
:10C3A000CF93DF931F92CDB7DEB75C016B017A01AB
:10C3B0004901F501808191810F94BD4F898300234C
:10C3C00011F0F6018083BE016F5F7F4FC4010F94AF
:10C3D0000A2EF50180819181019691838083FFEF80
:10C3E000CF1ADF0A81E0E81AF10819F780E00F9010
:10C3F000DF91CF910F91FF90EF90DF90CF90BF90A2
:10C40000AF909F908F9008959091C00095FFFCCFC2
:10C410008093C6000895CF93C82FCC2329F080E2E3
:10C420000E940462C150F9CFCF910895CF93DF935A
:10C43000FC018491EF012196882321F00E9404627F
:10C44000FE01F7CFDF91CF910895CF9382EC95E471
:10C450000E941662C0912A0B8EED90E30E94166234
:10C46000C11103C08AED90E302C08DED90E30E94FC
:10C47000166282ED90E30E94166262E370E080E053
:10C4800090E0CF910C945C610F931F93CF93DF9357
:10C490008B010E941662E8018991882319F00E949D
:10C4A0000462FACFDF91CF911F910F91089584EB31
:10C4B00090E30C9416628EEA90E30C9416627F92DD
:10C4C0008F929F92AF92BF92CF92DF92EF92FF92A4
:10C4D0000F931F93CF93DF931F92CDB7DEB77C01ED
:10C4E00059018B016B01C40ED51E0C151D0559F1A8
:10C4F000F70180809180F80171908F017982C401E9
:10C500000F94BD4F781691F0672DC4010F94C54F5D
:10C51000C4010F94BD4F9981891741F00E945B625D
:10C5200085E89FE20E94166281E00EC0BE016F5F47
:10C530007F4FC5010F940A2EF701808191810196EA
:10C5400091838083D2CF80E00F90DF91CF911F91B4
:10C550000F91FF90EF90DF90CF90BF90AF909F90A2
:10C560008F907F9008958F929F92AF92BF92EF929B
:10C57000FF920F931F93CF93DF93CDB7DEB7A097B2
:10C580000FB6F894DEBF0FBECDBF611571058105F2
:10C59000910591F100E0842E912CA12CB12C102F4B
:10C5A000EE24E394F12CEC0EFD1EE00EF11C07FDD1
:10C5B000FA94A50194010F94E34FF7016083B90148
:10C5C000CA010F5F611571058105910541F71F3F94
:10C5D00031F1E1E0F0E0EC0FFD1FE10FF11D17FD7F
:10C5E000FA9580818A3010F097E301C090E3890FBB
:10C5F0000E9404621150EBCF80E3A0960FB6F8942E
:10C60000DEBF0FBECDBFDF91CF911F910F91FF9085
:10C61000EF90BF90AF909F908F900C940462A09683
:10C620000FB6F894DEBF0FBECDBFDF91CF911F9143
:10C630000F91FF90EF90BF90AF909F908F900895D3
:10C64000CF92DF92EF92FF926A017B010E94166205
:10C650004AE0C701B601FF90EF90DF90CF900C94B5
:10C66000B362CF93DF93EB010E941662BE0180E0BC
:10C6700090E04AE0DF91CF910C94B362CF92DF92C9
:10C68000EF92FF926B017C0197FF0BC08DE20E943D
:10C690000462F094E094D094C094C11CD11CE11CBD
:10C6A000F11C4AE0C701B601FF90EF90DF90CF90F8
:10C6B0000C94B362AB01672B11F40C940462BC01BF
:10C6C000990F880B990B4A30510511F40C943E6375
:10C6D0000C94B362CF93DF93EB010E9416626AE081
:10C6E00070E0CE01DF91CF910C945A638F929F92AC
:10C6F000AF92BF92CF92DF92EF92FF92CF936B01F6
:10C700007C01B42E20E030E0A9010F948D4987FF11
:10C7100007C08DE20E940462F7FAF094F7F8F094F3
:10C72000C0E060E070E080E09FE3CB1541F02DECCD
:10C730003CEC4CEC5DE30F94F349CF5FF6CF9B01EB
:10C74000AC01C701B6010F9477506B017C010F94C7
:10C75000EA514B015C014AE00E94B362CC2391F1A3
:10C76000C501B4010F9492499B01AC01C701B60108
:10C770000F9476506B017C018EE20E94046220E0EF
:10C7800030E040E251E4C701B6010F94F3494B0198
:10C790005C010F94E3516B017C016AE070E0C6011B
:10C7A0000E945A63B601DD0C880B990B0F949449D3
:10C7B0009B01AC01C501B4010F9476506B017C0163
:10C7C000C150E9F6CF91FF90EF90DF90CF90BF90EE
:10C7D000AF909F908F9008950C947663AF92BF9224
:10C7E000CF92DF92EF92FF920F931F93CF93DF933D
:10C7F0000E943061882309F453C00E945B6287EC79
:10C8000090E30E94166296EAC92E9AE0D92EC0E003
:10C81000D0E0760100E010E0F70160817181828153
:10C8200093819B01AC010F94C453811129C00E94D4
:10C830005B62BE018EEB90E30E946A63B8018BEBF2
:10C8400090E30E946A638EE0A82E86E0B82EF50180
:10C8500081915F01882319F00E940462F8CFF701EB
:10C86000608171818281938144E00E9476638AE0D5
:10C870000E9404626BE470E080E090E00E945C61E2
:10C880000F5F1F4FF4E0EF0EF11C0530110521F68C
:10C89000219684E1C80ED11CC530D10509F0B9CF6D
:10C8A000DF91CF911F910F91FF90EF90DF90CF908C
:10C8B000BF90AF900895CF92DF92EF92FF926A01FE
:10C8C0007B010E94166242E0C701B601FF90EF9023
:10C8D000DF90CF900C9476638DE00E9404628AE032
:10C8E0000C940462CF93DF93EC018991882319F0B3
:10C8F0000E940462FACFDF91CF910C946C64CF93C5
:10C90000DF93CDB7DEB7A8970FB6F894DEBF0FBEA2
:10C91000CDBF8C010E94C2F80E9457628EE890E35E
:10C920000E9416620115110511F405E810E38091CB
:10C930000A0880FD75C0816080930A0881E196E055
:10C940000E947264882483948AE5982E909232150E
:10C95000809231158FE090E09093341580933315D9
:10C9600097E0A92EA092251522E8B22EB0922815A4
:10C9700034E8C32ED12CE12CF12CC0922915D09291
:10C980002A15E0922B15F0922C150F94732E90928D
:10C9900032158092311588E590E09093341580939C
:10C9A0003315A0922515B0922815C0922915D09262
:10C9B0002A15E0922B15F0922C150F94732E63E03C
:10C9C00070E080E090E00E942BC08AE289838A8335
:10C9D0008B838C83DE011596F801CE0101969D01B3
:10C9E000281B390B44913196442311F04D93F7CF16
:10C9F000FC01E20FF31F2AE2AF01481B590B48323A
:10CA0000510511F02193F8CF40E650E160E070E06D
:10CA10000F94222E6AE070E080E090E00E942BC02C
:10CA200061E08CE790E30E946FCA89EE93E030E604
:10CA3000019729F0232F2A950000E9F7F9CFF89400
:10CA400089EE93E038EE019729F0232F2A95000014
:10CA5000E9F7F9CF0E94C2F8A895FECF2F923F9236
:10CA60004F925F926F927F928F929F92AF92BF92FE
:10CA7000CF92DF92EF92FF920F931F93CF93DF93AA
:10CA8000CDB7DEB727970FB6F894DEBF0FBECDBF88
:10CA90008A830E947F2E0F94B8346B017C018091B1
:10CAA0004F0B81112FC080910002882359F1809192
:10CAB0004208882339F14091510850915208609101
:10CAC00053087091540897018601041B150B260B1F
:10CAD000370B37FD2AC0833079F03CF4813094F075
:10CAE0000E945B6287EE9FE20BC0843059F40E9483
:10CAF0005B6288EB9FE204C00E945B6280ED9FE274
:10CB00000E9416622091000230E0A8EEB3E00F947C
:10CB10003750C60ED71EE81EF91EC0925108D0929B
:10CB20005208E0925308F0925408809149028823F9
:10CB300019F180916E0881111FC08091AD1682FDA0
:10CB400008C080913A0B813021F08091330A88230C
:10CB500099F0F8946499CFC360919C1070919D10E6
:10CB600080919E1090919F10789420E030E0A90170
:10CB70000F948D4987FD4AC38091310A843020F497
:10CB80000E9401E90E94D0C80F94B8346B017C0167
:10CB900040913C0850913D0860913E0870913F08DB
:10CBA000411551056105710529F18091901390910E
:10CBB0009113A0919213B0919313840F951FA61F08
:10CBC000B71FA7019601281B390B4A0B5B0B57FDBA
:10CBD00011C00E9457626091670B7091680B82E4EC
:10CBE00090E30E9444628AE00E94046280E090E048
:10CBF0000E947F6440910102509102026091030201
:10CC000070910402411551056105710509F44EC08A
:10CC10009091AD148091AE14981759F00F94B834D8
:10CC20006093901370939113809392139093931346
:10CC30003DC08091330A811137C00A81011134C08F
:10CC40008091901390919113A0919213B0919313AE
:10CC5000840F951FA61FB71FA7019601281B390B2C
:10CC60004A0B5B0B57FD20C08091650881111EC0E7
:10CC700081E0809365085F9A809198138E7F8093FE
:10CC800098138A9A809198138D7F8093981380913E
:10CC900008018095817080930601809198138B7FA5
:10CCA00080939813129A02C01092650880916108CF
:10CCB00090916208A0916308B0916408B701A60141
:10CCC000481B590B6A0B7B0B77FDCDC19091AD14BE
:10CCD0008091AE1460915C0250915D02598398136B
:10CCE00017C08091910B869FB0011124660F672FAA
:10CCF000661F770B71956A838091920B859FB001B7
:10CD00001124660F672F661F770B719569832AC000
:10CD10008091AE1478E4879FC00111248554944F0C
:10CD2000FC01EA5BFF4F2081269FB0011124660FB2
:10CD3000672F661F770B71956A8331968081998181
:10CD4000899FB0011124660F672F661F770B7195BD
:10CD500069838091AE149091AD14981719F08F5F8C
:10CD60008F70F9CF0A81002349F10F94B8340091F4
:10CD7000590810915A0820915B0830915C08DC0139
:10CD8000CB01011511052105310579F48C599F4F0F
:10CD9000AF4FBF4F8093590890935A08A0935B08F8
:10CDA000B0935C081FEF1A8311C0801B910BA20B7C
:10CDB000B30BB7FF0BC00FEF0A8308C010925908DE
:10CDC00010925A0810925B0810925C081A81612F29
:10CDD00070E089E00F9496330981002349F10F94A4
:10CDE000B83400915D0810915E0820915F08309181
:10CDF0006008DC01CB01011511052105310579F42D
:10CE00008C599F4FAF4FBF4F80935D0890935E0842
:10CE1000A0935F08B09360081FEF198311C0801BB7
:10CE2000910BA20BB30BB7FF0BC00FEF098308C028
:10CE300010925D0810925E0810925F0810926008D0
:10CE40001981612F70E087E00F9496338091111360
:10CE5000882309F4FBC020903602309037020091FD
:10CE600038020F83109139021E836091AC0B7091D0
:10CE7000AD0B6E5F7F4F072E000C880B990B0F9444
:10CE800094499101A8010F948D4987FDDFC000915D
:10CE9000AE1409831A821B821C821D828091AD14FC
:10CEA0001981811709F460C0812F90E028E4289F40
:10CEB000F001299FF00D1124E554F44F458956895E
:10CEC0006789708D452B462B472B81F4418D528D00
:10CED000638D748D452B462B472B41F4458D568D24
:10CEE000678D70A1452B462B472BC9F138E4389F3D
:10CEF0008001399F100D11240554144FF8016181F0
:10CF00007281838194810F9475534B015C01F80108
:10CF100061A172A183A194A10F9492492B013C01BC
:10CF2000F80165A176A187A190A50F9492499B0174
:10CF3000AC01C301B2010F947151A50194010F948A
:10CF4000F3495B018C012A813B814C815D810F9407
:10CF5000D752181624F4AA82BB820C831D838981C0
:10CF60008F5F8F7089839ACF20913A0230913B0274
:10CF700040913C0250913D026A817B818C819D8170
:10CF80000F94F34991014F815E810F9477505B01BB
:10CF90008C01609032027090330280903402909045
:10CFA00035029B01AC01B1018F819E810F94D75254
:10CFB00018167CF09301A401B501C8010F94D75253
:10CFC000181624F413018F829E8203C015010F836B
:10CFD0001E838090550890905608A0905708B090F6
:10CFE000580891014F815E81C501B4010F94D75259
:10CFF0001816D4F420E037ED43EA5CE3B1018F81E9
:10D000009E810F94F3492B013C0128E431EE4AE75D
:10D010005FE3C501B4010F94F349A30192010F949A
:10D0200077501B018F839E83C101AF81BE818093A6
:10D03000550890935608A0935708B0935808B1012B
:10D04000CD010F94E351CB010E94978AF4E6CF0EF5
:10D05000D11CE11CF11CC0926108D0926208E092E0
:10D060006308F09264080E942CB380913A0B8130DF
:10D0700009F06EC00F94B8346B017C0180916A088E
:10D0800090916B08A0916C08B0916D089701860192
:10D09000081B190B2A0B3B0B37FD3AC080903B0B4A
:10D0A00090903C0BA0903D0BB0903E0B0E94F3FF84
:10D0B00060933B0B70933C0B80933D0B90933E0B26
:10D0C00000918F081091900820919108309192085A
:10D0D000081919092A093B09DC01CB01800F911FAE
:10D0E000A21FB31F80938F0890939008A09391087C
:10D0F000B0939208D701C601805F984DAF4FBF4FE4
:10D1000080936A0890936B08A0936C08B0936D08A5
:10D110008091660890916708A0916808B0916908AD
:10D12000A7019601281B390B4A0B5B0B57FD10C05A
:10D1300030E8C30E3EEED31EE11CF11CC09266081F
:10D14000D0926708E0926808F09269080E94BC904B
:10D1500080914F0B8111FEC080913708882391F098
:10D160000F94B83400913308109134082091350899
:10D1700030913608DC01CB01801B910BA20BB30B65
:10D18000B7FFCAC00F94B8346B017C0120913208FC
:10D19000222309F4DFC080912E0890912F08A091DE
:10D1A0003008B0913108B701A601481B590B6A0B32
:10D1B0007B0B77FDCFC030E0A8EEB3E00F94375083
:10D1C000C60ED71EE81EF91EC0922E08D0922F0858
:10D1D000E0923008F092310827960FB6F894DEBF3F
:10D1E0000FBECDBFDF91CF911F910F91FF90EF90B8
:10D1F000DF90CF90BF90AF909F908F907F906F9077
:10D200005F904F903F902F900C94CB6C11E0109357
:10D210006E088091330A81116BC08CE196E00E9408
:10D22000726484E080932C0B10920F0882E080934C
:10D230000B0881E09AE590933215809331158EE4C6
:10D2400090E0909334158093331587E080932515F3
:10D2500082E88093281584E890E0A0E0B0E0809315
:10D26000291590932A15A0932B15B0932C150F9484
:10D27000732E109346110E9493CA40E061E370E35D
:10D2800082ED94E40E949FCA80E30E9404628AE0D7
:10D290000E9404620E9487CA8091400860E01827BB
:10D2A0001983112319F082EB93E40DC08FE190E311
:10D2B0000E946FCA80E30E9404628AE00E940462B6
:10D2C00060E089EF9FE20E946FCA8DE090E30E94C8
:10D2D000166280E30E9404628AE00E94046209816F
:10D2E000002331F08FEF9FE29093AE088093AD085A
:10D2F0000E94ED9141CC8091540290915502A091F1
:10D300005602B091570280939C1090939D10A09369
:10D310009E10B0939F1020CC0F94B8346B017C0109
:10D320002091370830E0A8EEB3E00F943750C60ED6
:10D33000D71EE81EF91EC0923308D0923408E0923E
:10D340003508F092360880E00E942DF18AE00E94B4
:10D35000046218CF27960FB6F894DEBF0FBECDBF7C
:10D36000DF91CF911F910F91FF90EF90DF90CF90C1
:10D37000BF90AF909F908F907F906F905F904F90F5
:10D380003F902F900895EAE0F2E180818183089533
:10D3900080910A1290910B12981759F0E92FF0E042
:10D3A000E65FFD4E82819F5F9F7790930B1290E026
:10D3B00008958FEF9FEF08951F920F920FB60F926F
:10D3C00011240F900FBE0F901F9018951F920F926F
:10D3D0000FB60F9211240BB60F920F931F932F933A
:10D3E0003F934F935F936F937F938F939F93AF93ED
:10D3F000BF93CF93DF93EF93FF9300910B12D091E4
:10D400000A1211E01D0F1F77C091C60090914F08BE
:10D41000492F092E000C550B660B770B4131510536
:10D4200008F064C0FA018827E256FF4F8F4F0D9431
:10D430006E50CD3449F0CE34B9F481E006C0CA3321
:10D4400038F0CD3409F043C082E080934F0876C0B5
:10D45000C03308F073C0C03209F470C0CD32B9F5E2
:10D460006DC0C13351F018F4C03289F567C0C433C0
:10D4700031F0C83361F58BE0E8CF83E0E6CF88E098
:10D48000E4CFC03321F0C13311F586E0DECF84E074
:10D49000DCCFC833E1F485E0D8CFC233C1F487E0F4
:10D4A000D4CFC133A1F489E0D0CFC03381F48AE076
:10D4B000CCCFC73361F48CE0C8CFC63341F48DE0E4
:10D4C000C4CFC032D9F1C33511F48EE0BECF80E1B4
:10D4D000BCCF80ED8C0F8A3088F59FE090934F0889
:10D4E00080934E082BC0CA3049F526C0CA3031F5AA
:10D4F00080919315882301F1973089F03CF49530A1
:10D50000D9F4109214021092641316C09A3059F094
:10D510009F3091F480914E080E94CBCA0DC081E0EB
:10D520008093BE1009C00E9484930E94ED918EEFFB
:10D530000E94E3D60E9451D710924F08011731F094
:10D54000ED2FF0E0E65FFD4EC283D12FD0930A129B
:10D55000FF91EF91DF91CF91BF91AF919F918F910B
:10D560007F916F915F914F913F912F911F910F91FB
:10D570000F900BBE0F900FBE0F901F9018958EBD91
:10D580000DB407FEFDCF08958FEF8EBD0DB407FEDD
:10D59000FDCF8EB50895909164009B7F90936400B9
:10D5A000982F906A96959CBD80FD03C091E08630CF
:10D5B00009F490E09DBD0895CF92DF92EF92FF9223
:10D5C0000F931F93CF93DF936C017A018B01C0E01F
:10D5D000D0E0CE15DF0581F0D8016D918D01D60127
:10D5E000ED91FC910190F081E02DC6011995892BF8
:10D5F00011F02196EECF7E01C701DF91CF911F91EF
:10D600000F91FF90EF90DF90CF900895089580E004
:10D6100090E00895FC01538D448D252F30E0842F38
:10D6200090E0821B930B541710F0CF96089501974A
:10D630000895FC01918D828D981761F0828DDF0134
:10D64000A80FB11D5D968C91928D9F5F9F73928FF5
:10D6500090E008958FEF9FEF0895FC01918D828DEA
:10D66000981731F0828DE80FF11D858D90E00895B7
:10D670008FEF9FEF0895FC01918D228D892F90E00F
:10D68000805C9F4F821B91098F739927089589E9C8
:10D6900093E10E943B6B21E0892B09F420E0822F6B
:10D6A0000895FC01848DDF01A80FB11DA35ABF4F5F
:10D6B0002C91848D90E001968F739927848FA68991
:10D6C000B7892C93A089B1898C91837080648C93E5
:10D6D000938D848D981306C00288F389E02D808194
:10D6E0008F7D80830895EF92FF920F931F93CF93C6
:10D6F000DF93EC0181E0888F9B8D8C8D981305C0A2
:10D70000E889F989808185FD26C0F62E0B8D10E011
:10D710000F5F1F4F0F731127E02E8C8DE8120CC086
:10D720000FB607FCFACFE889F989808185FFF5CF2C
:10D73000CE010E94516BF1CF8B8DFE01E80FF11DE0
:10D74000E35AFF4FF0829FB7F8940B8FEA89FB8969
:10D75000808180620AC09FB7F894EE89FF89608358
:10D76000E889F98980818370806480839FBF81E02C
:10D7700090E0DF91CF911F910F91FF90EF9008956E
:10D78000CF93DF93EC01888D8823C9F0EA89FB8968
:10D79000808185FD05C0A889B9898C9186FD0FC05F
:10D7A0000FB607FCF5CF808185FFF2CFA889B98934
:10D7B0008C9185FFEDCFCE010E94516BE7CFDF91B9
:10D7C000CF91089580E090E0892B41F080E090E0D7
:10D7D000892B21F00E940000811121C080E090E09F
:10D7E000892B41F080E090E0892B21F00E9400001D
:10D7F000811118C080E090E0892B21F00E94476BD6
:10D80000811113C080E090E0892BA1F080E090E0CE
:10D81000892B81F00E94000081110AC008950E94A6
:10D820000000DCCF0E940000E5CF0E940000EACF9C
:10D830000C9400000895FC0120E03EE2DB014C91D5
:10D84000403241F0283011F430833196DB014C91A5
:10D85000408331962F5F6F5F7F4F2B3079F71082B7
:10D8600008950F94DC540F931F93CF93DF938B0194
:10D87000EA01DB016D917C910E943F83D801ED911B
:10D88000FC91119790818881992349F0893638F469
:10D890003196ED93FC9388818F5F8883EFCF893633
:10D8A00058F48FE28083F801808191810196918301
:10D8B000808388818F5F8883DF91CF911F910F9143
:10D8C00008951F920F920FB60F9211240BB60F926C
:10D8D0002F933F934F935F936F937F938F939F9378
:10D8E000AF93BF93EF93FF9389E993E10E94516B4C
:10D8F000FF91EF91BF91AF919F918F917F916F9128
:10D900005F914F913F912F910F900BBE0F900FBEE3
:10D910000F901F9018951F920F920FB60F9211241F
:10D920000BB60F922F938F939F93EF93FF93E091FA
:10D93000A913F091AA138081E091AF13F091B01375
:10D9400082FD12C090818091B2138F5F8F732091FE
:10D95000B313821751F0E091B213F0E0E756FC4E9A
:10D96000958F8093B21301C08081FF91EF919F91B9
:10D970008F912F910F900BBE0F900FBE0F901F90A5
:10D9800018958BE1EFE8F4E1A4E7B4E101900D9282
:10D990008A95E1F708958091AD1682FF1FC08CE74C
:10D9A00093E30E9416626091A9167091AA16809165
:10D9B000AB169091AC164AE00E94B3628FE20E94CF
:10D9C00004626091A5167091A6168091A716909199
:10D9D000A8164AE00E94B3620C946C648EE893E34C
:10D9E0000C9416621092330A8091AD168F7D8B7F56
:10D9F0008093AD160E94C2C8882321F086E394E18B
:10DA00000C94A58508958091AD1683FF03C08460B2
:10DA10008093AD160895CF92DF92EF92FF920F930D
:10DA20001F93CF93DF93CDB7DEB7EDB6FEB6DC0123
:10DA30000D900020E9F79D01281B390B2C5F3F4F0B
:10DA40004DB75EB7421B530B0FB6F8945EBF0FBEC7
:10DA50004DBF0DB71EB70F5F1F4F9F938F9388E782
:10DA600092E39F938F931F930F930F94254968011F
:10DA700054E0C50ED11C0F900F900F900F900F9097
:10DA80000F90F6018081882349F0082E000C990B35
:10DA90000F94E154F60181936F01F3CFC8010E9406
:10DAA00095EA84E792E30E94C7EA0FB6F894FEBEB7
:10DAB0000FBEEDBEDF91CF911F910F91FF90EF90C0
:10DAC000DF90CF9008958F929F92AF92BF92CF92A6
:10DAD000DF92EF92FF92CF938091AD16877F809374
:10DAE000AD1680919214882321F08FE894E10E9472
:10DAF000A585109273141092701485E380936F14AF
:10DB00000F94B8346B017C0120EDC20E27E0D21EC9
:10DB1000E11CF11CA89561E080916F140F942B33E8
:10DB200061E080916F140F945A33209A289A219AB9
:10DB30002398229A81E00E94CB6A85E08093711439
:10DB40000E94CB6ACAE08FEF0E94BF6AC150D9F72A
:10DB5000A89520E030E0A90160E08FE694E10E9402
:10DB6000858480937214813061F00F94B834DC01A5
:10DB7000CB018C199D09AE09BF09B7FDEACF81E041
:10DB800062C0A8952AEA31E040E050E068E08FE604
:10DB900094E10E948584853011F481E00AC0C4E0DC
:10DBA0000E94C46A80937214C150D1F78A3A61F41A
:10DBB00082E080937314A89580917314823081F071
:10DBC000812C912C540111C00F94B834DC01CB018D
:10DBD0008C199D09AE09BF09B7FDD4CF82E033C0CF
:10DBE000812C912CA12C80E4B82E20E030E0A901FA
:10DBF00067E38FE694E10E948584A501940169E2C0
:10DC00008FE694E10E94858480937214882361F0EA
:10DC10000F94B834DC01CB018C199D09AE09BF0902
:10DC2000B7FDE3CF8AE00FC080917314823021F5F5
:10DC300020E030E0A9016AE38FE694E10E94858448
:10DC4000882361F088E0809370148FE694E10E944D
:10DC50007D840E945B6286E692E322C00E94C46AD1
:10DC6000807C803C19F483E0809373140E94C46A22
:10DC70000E94C46A0E94C46A8FE694E10E947D8477
:10DC80001092711481E00F941A3781110CC080E05A
:10DC90000F941A37811107C00E94576282E592E300
:10DCA0000E9416621AC061E574E18FE894E10E9457
:10DCB000D082811105C00E94576281E492E3F0CFC7
:10DCC0008091AD1688608093AD160E945B6285E3FB
:10DCD00092E30E9416620E94B661CF91FF90EF908E
:10DCE000DF90CF90BF90AF909F908F900C94C16CBD
:10DCF0002F923F925F926F927F928F929F92AF92FC
:10DD0000BF92CF92DF92EF92FF920F931F93CF9328
:10DD1000DF93CDB7DEB7C356D1090FB6F894DEBF97
:10DD20000FBECDBF8C016B014A012DB63EB6512C02
:10DD30007E0187E5E80EF11CF6018381823008F44C
:10DD40001FC180859185A285B3858F719927AA27E8
:10DD5000BB27892B8A2B8B2B09F012C11092131928
:10DD600043E159E1BE016F5F7F4FC6010E943A87D0
:10DD700018160CF005C18C85982F9871903129F4F4
:10DD80002091A10A2150223078F42981222309F41C
:10DD9000F7C0253E89F22E3279F2209113192E32E6
:10DDA00059F28A7049F67CC06DB67EB6BE016F5FCF
:10DDB0007F4FC7010E941B6C0115110521F0F8016E
:10DDC0008081811163C021E081E090E0F701019042
:10DDD0000020E9F73197EE19FF09E80FF91F329695
:10DDE0008DB79EB78E1B9F0B0FB6F8949EBF0FBECC
:10DDF0008DBFEDB7FEB731965F01211102C0B801AA
:10DE000002C06AE776E0C5010F942855B701C50145
:10DE10000F9412556AE776E0C5010F94125519A2C6
:10DE20001CA221E0A701B601CE0181960E94918932
:10DE300081110DC08091A10A811109C00E945B620D
:10DE400081E292E30E941662C7010E9472648BE134
:10DE5000FE01B196DE01DC9601900D928A95E1F704
:10DE600040E050E0BE01645C7F4FC5010E94786EC7
:10DE7000CE01CC960E94AE85CE0181960E94AE85E1
:10DE80000FB6F8947EBE0FBE6DBE56CFF80101905E
:10DE90000020E9F73197CF01801B910B20E096CF4E
:10DEA00021E0903109F020E08091AD1620FB84F94B
:10DEB0008093AD16903141F08985873409F03CCFCD
:10DEC0008A858E3709F438CF8091A10A813021F0FC
:10DED00068F08230C1F130CF8091A40A9091A50AF8
:10DEE00001969093A50A8093A40A26CFBE016F5F86
:10DEF0007F4F85E599E10E941B6C0115110529F4FE
:10DF000085E5A82E89E1B82E09C05801F501819157
:10DF10005F018823A9F30E940462F8CFF501819183
:10DF20005F01882319F00E940462F8CF80E20E940A
:10DF300004626D8D7E8D8F8D98A14AE00E94B36240
:10DF40000E946C64F9CEBE016F5F7F4F85E599E159
:10DF50000E941B6C8114910441F065E579E1C401D4
:10DF60000F94FF54892B51F40BC0852D90E0209124
:10DF7000A20A3091A30A8217930711F05394DCCEC2
:10DF80000FB6F8943EBE0FBE2DBECD59DF4F0FB673
:10DF9000F894DEBF0FBECDBFDF91CF911F910F91DF
:10DFA000FF90EF90DF90CF90BF90AF909F908F90B9
:10DFB0007F906F905F903F902F900895CF93DF9365
:10DFC000CDB7DEB76B970FB6F894DEBF0FBECDBFEF
:10DFD00081E08093A10A1092A50A1092A40A84E716
:10DFE00094E10E9478848BE1E4E7F4E1DE0111968C
:10DFF00001900D928A95E1F740E050E0BE016F5F1D
:10E000007F4F80E090E00E94786ECE0101960E94E2
:10E01000AE858091A40A9091A50A6B960FB6F894EC
:10E02000DEBF0FBECDBFDF91CF9108950F931F9339
:10E03000CF93DF93CDB7DEB76B970FB6F894DEBF03
:10E040000FBECDBF8B0122E02093A10A9093A30ABB
:10E050008093A20A84E794E10E9478848BE1E4E74C
:10E06000F4E1DE01119601900D928A95E1F7A80185
:10E07000BE016F5F7F4F80E090E00E94786ECE011E
:10E0800001960E94AE856B960FB6F894DEBF0FBE68
:10E09000CDBFDF91CF911F910F910895DF92EF9245
:10E0A000FF920F931F93CF93DF9300D01F92CDB7B2
:10E0B000DEB72091AD1623FF3DC1F42EE62E8C0174
:10E0C0000E94C2C8882309F481C0FF2009F48CC0D3
:10E0D0008091A416882351F00E94576287E393E34E
:10E0E0000E94166280E090E00E947F6489E39AE0DB
:10E0F0009A8389838FE28093380A81E08B83F12CA5
:10E100009BE1D92E8091A316F81678F4DF9CC0010C
:10E110001124AE014D5F5F4FBE016F5F7F4F8B5685
:10E120009A4E0E94336CF394EDCF8B818B3578F44B
:10E13000AE014D5F5F4FBE016F5F7F4F86E394E19D
:10E140000E94336C89819A8101979A838983E9813E
:10E15000FA811082E091A41684E0E89FF001112476
:10E16000EC5CF54F8091A9169091AA16A091AB1680
:10E17000B091AC1680839183A283B3830E945B62CB
:10E18000B8018EE193E30E9444626091A41689E68F
:10E19000689FB0011124685C754F83E193E30E948E
:10E1A00044624091A9165091AA166091AB167091E5
:10E1B000AC168DE093E30E9420638AE00E94046223
:10E1C0008091A4168F5F8093A41626C0FF2039F09B
:10E1D0000E945B628DEF92E30E9416621DC0109256
:10E1E000A41682E0F82E02C0FF24F3940E945B6222
:10E1F00088EF92E30E94166281E0F81609F497C056
:10E2000084EE92E30E941662B80180EF92E30E94CE
:10E2100044628AE00E9404620E94F26CB801CE015E
:10E2200003960F94CF2F8C01009709F483C06B8164
:10E230007C81EE2009F450C021E0AC0186E394E13A
:10E240000E949189882309F43FC0809147149091DE
:10E250004814A0914914B0914A148093A516909344
:10E26000A616A093A716B093A8161092A9161092FE
:10E27000AA161092AB161092AC16B80186ED92E376
:10E280000E9444624091A5165091A6166091A7166F
:10E290007091A8168EEC92E30E9420638AE00E949F
:10E2A00004628FEB92E30E941662B80180E090E076
:10E2B0000E94167080911319811102C0C80102C01A
:10E2C00083E199E160E030C0B8018BEA92E30E94FB
:10E2D000446288EA92E30FC026E5AC0186E394E14C
:10E2E0000E94918981110AC0B80184E992E30E94D9
:10E2F000446281E992E30E9416621CC08091AD16CF
:10E3000081608093AD16B80180E090E00E941670A5
:10E3100010929315B8018FE792E30E9444628AE05D
:10E320000E94046260E0C8010F948D0303C08AEE6E
:10E3300092E368CF0F900F900F900F90DF91CF91E5
:10E340001F910F91FF90EF90DF900895CF92DF9291
:10E35000EF92FF92CF936B017C01C42F809108193B
:10E3600090910919A0910A19B0910B198C159D056E
:10E37000AE05BF05D1F00E943285811102C080E058
:10E3800018C028E037E1B701A601809111199091DA
:10E3900012190E94B485882391F3C0920819D09273
:10E3A0000919E0920A19F0920B1981E0C1118093CA
:10E3B0001019CF91FF90EF90DF90CF9008954F927A
:10E3C0005F926F927F928F929F92AF92BF92CF9205
:10E3D000DF92EF92FF920F931F93CF93DF93EC01A5
:10E3E000423051056105710510F480E069C08985EE
:10E3F0009A85AB85BC850196A11DB11D8417950733
:10E40000A607B70790F38F89803149F4852E962EA1
:10E41000A72EBB248B899C89AD89BE890FC0803211
:10E4200021F78B889C88AD88BE88DB01CA01E7E0B4
:10E43000B695A79597958795EA95D1F7880E991E79
:10E44000AA1EBB1E280139016A017B0141E0C501FA
:10E45000B4010E94A671882341F29F89903161F432
:10E46000DD24EE24FF249601220F331FF901E85F1B
:10E47000F84E5182408211C0E894C7F8DD24EE24A2
:10E48000FF249601220F331F220F331FF901E85F8B
:10E49000F84E40825182628273829A89923080F073
:10E4A0004D815E816F817885840E951EA61EB71EF4
:10E4B00080920C1990920D19A0920E19B0920F191A
:10E4C000DF91CF911F910F91FF90EF90DF90CF9050
:10E4D000BF90AF909F908F907F906F905F904F9084
:10E4E0000895CF92DF92EF92FF920F931F93CF93F5
:10E4F000DF93FC0181859285A385B4850196A11DDA
:10E50000B11D84179507A607B70710F480E061C016
:10E510008789803149F4BB27A72F962F852FC38881
:10E52000D488E588F6880FC0803281F78389948982
:10E53000A589B6896A017B01C7E0F694E794D79470
:10E54000C794CA95D1F78C0D9D1DAE1DBF1DE90165
:10E550006A017B018F01409108195091091960915E
:10E560000A1970910B1984179507A607B70739F098
:10E5700040E0BC01CD010E94A671882339F2F80168
:10E580008789803179F4B701A60155276627772757
:10E59000440F551FFA01E85FF84E80819181A0E099
:10E5A000B0E012C0B701A6014F775527662777273D
:10E5B000440F551F440F551FFA01E85FF84E808144
:10E5C0009181A281B381BF7088839983AA83BB8321
:10E5D00081E0DF91CF911F910F91FF90EF90DF903D
:10E5E000CF9008954F925F926F927F92AF92BF92B9
:10E5F000CF92DF92EF92FF920F931F93CF93DF930F
:10E6000000D01F92CDB7DEB78C0149835A836B834C
:10E610007C835901C12CD12C7601412C82E0582EEB
:10E62000612C712C49815A816B817C819E012F5F05
:10E630003F4FC8010E947172882341F1D301C2018A
:10E64000F801058404C0880F991FAA1FBB1F0A94F4
:10E65000D2F7C80ED91EEA1EFB1E49815A816B8172
:10E660007C818789803139F481E0483F5F4F6105C3
:10E67000710538F4D7CF81E0483F5F4F6F4F7F403F
:10E6800088F2F501C082D182E282F3820F900F906E
:10E690000F900F90DF91CF911F910F91FF90EF900E
:10E6A000DF90CF90BF90AF907F906F905F904F9032
:10E6B00008954F925F926F927F928F929F92AF9246
:10E6C000BF92CF92DF92EF92FF920F931F93CF935F
:10E6D000DF93CDB7DEB768970FB6F894DEBF0FBEF5
:10E6E000CDBF2A013B015901E82EF12CF701E25B75
:10E6F000FB4CE491CC24C3941E160CF4C12CDD24F5
:10E70000D39420E030E0A901C301B2010F94D752A5
:10E7100018160CF0D12C80E00E94189369837A833C
:10E720008B839C8381E00E9418936D837E838F830B
:10E73000988782E00E94189369877A878B879C87E5
:10E7400083E00E9418936D877E878F87988BEE0CED
:10E75000FF1CEE0CFF1C88248394912C8C0E9D1EB4
:10E760008E0C9F1CF40110821182128213829E0172
:10E77000235F3F4FAE01475F5F4FBE016B5F7F4F2F
:10E78000CE0101960E944392F4014082518262823E
:10E7900073821D8A1E8A1F8A188E20E030E0A9012C
:10E7A000B801C5010F948D49811109C0F701EB5FD4
:10E7B000FB4C85919591A591B4918C015D01C801A7
:10E7C000D501898B9A8BAB8BBC8BCE0145967C0196
:10E7D0008E010F5E1F4F9E01235F3F4FAE01475FCB
:10E7E0005F4FBE016B5F7F4F44970E94FFA10E9465
:10E7F000ED91CD100E94F2D768960FB6F894DEBF67
:10E800000FBECDBFDF91CF911F910F91FF90EF9081
:10E81000DF90CF90BF90AF909F908F907F906F9040
:10E820005F904F9008958F929F92AF92BF92EF9218
:10E83000FF920F931F93CF93DF9320912A0B2223F4
:10E8400049F1EA017B018C01CA010E94A5CF4B016D
:10E850005C0120E030E0A9010F948D49882369F024
:10E86000B701C8010E94AE969B01AC01C501B4017D
:10E870000F94F3499B01AC0103C020E030E0A901F3
:10E88000688179818A819B810F947750688379832D
:10E890008A839B83DF91CF911F910F91FF90EF901F
:10E8A000BF90AF909F908F900895CF92DF92EF929C
:10E8B000FF9280911B0B882371F1C090200BD090A8
:10E8C000210BE090220BF090230B20E030E0A90117
:10E8D000C701B6010F948D498823E9F020E030E0AC
:10E8E00040E05FE3C701B6010F94F3499B01AC011F
:10E8F0000F94F3492BED3FE049E450E40F94F349C2
:10E900009B01AC0160E070E080E89FE30F947151DF
:10E910006B017C0106C0C12CD12C80E8E82E8FE36E
:10E92000F82EC0921C0BD0921D0BE0921E0BF092A1
:10E930001F0B6091300270913102072E000C880B82
:10E94000990B0F9494492AE037ED43E25CE30F946E
:10E95000F349A70196010F94F34960934302709322
:10E9600044028093450290934602FF90EF90DF901F
:10E97000CF9008954F925F926F927F928F929F9265
:10E98000AF92BF92CF92DF92EF92FF920F931F93BD
:10E99000CF93DF93CDB7DEB768970FB6F894DEBF9D
:10E9A0000FBECDBF8C015B015A834983DC01D69633
:10E9B0006D917D918D919C91D9970F9492496B01A6
:10E9C0007C01F50120813181428153810F94F3490B
:10E9D0000F9455510F94EA5169877A878B879C87EA
:10E9E000A981BA812D913D914D915C91C701B601EC
:10E9F0000F94F3490F9455510F94EA516D877E8718
:10EA00008F87988B29853A854B855C85283731051A
:10EA10004105510540F488E790E0A0E0B0E0898727
:10EA20009A87AB87BC872D853E854F8558892837C7
:10EA300031054105510540F488E790E0A0E0B0E0E1
:10EA40008D879E87AF87B88BF801EE5BFF4F2081E3
:10EA500031814281538129833A834B835C83CA018C
:10EA6000B9010F9494492B013C0169857A858B8506
:10EA70009C850F949249698B7A8B8B8B9C8B20E0C1
:10EA800030E0A901C301B2010F948D49882329F117
:10EA9000A7019601C701B6010F94F3494B015C0130
:10EAA00029893A894B895C89CA01B9010F94F349D4
:10EAB0009B01AC01C501B4010F9476504B015C0180
:10EAC000A3019201C301B2010F9477509B01AC01E5
:10EAD000C501B4010F94715103C060E070E0CB0137
:10EAE0000F9455510F94EA516D837E838F839887DD
:10EAF00069817A818B819C819095809570956195D3
:10EB00007F4F8F4F9F4F0F9494494B015C016D8550
:10EB10007E858F8598890F94924969837A838B8348
:10EB20009C8320E030E0A901C501B4010F948D4918
:10EB3000882349F129813A814B815C81CA01B9015D
:10EB40000F94F3496D8B7E8B8F8B988FA701960165
:10EB5000C701B6010F94F3499B01AC016D897E8911
:10EB60008F89988D0F9476506B017C01A5019401DB
:10EB7000C501B4010F9477509B01AC01C701B601E8
:10EB80000F94715103C060E070E0CB010F941952F3
:10EB9000D80195968D909D90AD90BC9098977501F9
:10EBA00064012D813E814F815885C21AD30AE40A3F
:10EBB000F50A0F94EA51C61AD70AE80AF90AF7FECD
:10EBC00075C020E030E0A901C301B2010F948D4966
:10EBD000882309F443C0C501B4010F9492496B0125
:10EBE0007C01A3019201C301B2010F9477509B01F4
:10EBF000AC01C701B6010F94F3496B017C0129896F
:10EC00003A894B895C89CA01B9010F94F3499B0188
:10EC1000AC01C701B6010F9476506B017C012981CC
:10EC20003A814B815C81CA01B9010F94F3499B0180
:10EC3000AC01C701B6010F9477506B017C0120E055
:10EC400030E040E850E4C301B2010F94F3499B0166
:10EC5000AC01C701B6010F94715103C060E070E0D0
:10EC6000CB010F9455517B018D83998320E030E0D7
:10EC7000A9010F94D752181624F0E12CF12C1D8213
:10EC80001982B7018D8199810F94EA516D837E833A
:10EC90008F83988786169706A806B90620F48D827A
:10ECA0009E82AF82B886C12CD12C76018D819E8147
:10ECB000AF81B885F80181A792A7A3A7B4A7C80E12
:10ECC000D91EEA1EFB1EC5A6D6A6E7A6F0AA298570
:10ECD0003A854B855C8522AF33AF44AF55AFFE9686
:10ECE0002D853E854F855889208331834283538308
:10ECF00068960FB6F894DEBF0FBECDBFDF91CF91FF
:10ED00001F910F91FF90EF90DF90CF90BF90AF9049
:10ED10009F908F907F906F905F904F900895CF92CB
:10ED2000DF92EF92FF92CF93DF93EC01C090180235
:10ED3000D0901902E0901A02F0901B0228813981CC
:10ED40004A815B81C701B6010F94D752181624F48B
:10ED5000C882D982EA82FB82C0901C02D0901D0238
:10ED6000E0901E02F0901F02288139814A815B8168
:10ED7000C701B6010F948D4987FF04C0C882D982AC
:10ED8000EA82FB82C0902002D0902102E090220211
:10ED9000F09023022C813D814E815F81C701B60135
:10EDA0000F94D752181624F4CC82DD82EE82FF82B3
:10EDB000C0902402D0902502E0902602F090270215
:10EDC0002C813D814E815F81C701B6010F948D4931
:10EDD00087FF04C0CC82DD82EE82FF82C0902802D1
:10EDE000D0902902E0902A02F0902B0228853985E4
:10EDF0004A855B85C701B6010F94D752181624F4D3
:10EE0000C886D986EA86FB86C0902C02D0902D0257
:10EE1000E0902E02F0902F02288539854A855B8587
:10EE2000C701B6010F948D4987FF04C0C886D986F3
:10EE3000EA86FB86DF91CF91FF90EF90DF90CF9035
:10EE40000895CF93DF9324E0829FC0011124EC0149
:10EE5000C15CD44FFC01E056F74FDC01A25FB44F18
:10EE60002D913D914D915C91608171818281938161
:10EE70000F947750688379838A839B83DF91CF9146
:10EE800008954F925F926F927F928F929F92AF926E
:10EE9000BF92CF92DF92EF92FF920F931F93CF9387
:10EEA000C82FE82EF12CF701E25BFB4CB4908230C6
:10EEB00029F481E00E94A38C811101C16701CC0C6F
:10EEC000DD1CCC0CDD1CF601EE5BFB4C4590559037
:10EED000659074906B2DBB0C770B880B990B0F947E
:10EEE00094494B015C0120E030E040EC5FE3C3015A
:10EEF000B2010F94F349A50194010F94F349AB01BA
:10EF0000BC0100E010E098018C2F0E945973C230C0
:10EF100061F0F601EA5CFB4C85919591A591B49165
:10EF2000E82F792F6A2F8B2F04C0E0E070E060EAB1
:10EF300080E42E2F372F462F582FC501B4010F9490
:10EF4000F3494B015C0120E030E0A9010F948D49A9
:10EF5000882309F446C0C23021F000E010E0980197
:10EF600004C000E010E020E830E4B501A4017058CE
:10EF70008C2F0E945973C23011F1F701ED5CFB4CEC
:10EF80006491611107C00E945B6281E194E30E9479
:10EF900016626AE0F601EB5FFB4C45905590659078
:10EFA000749070E080E090E00F9494499B01AC0174
:10EFB000C301B2010F9471512B013C0105C0412CDA
:10EFC000512C612C90E4792EA5019401C501B40166
:10EFD0000F947750AB01BC01930182018C2F0E94EA
:10EFE000597381E090E00C2E01C0880F0A94EAF773
:10EFF00090919813982B9093981390911A0B892BBA
:10F0000080931A0BF601E25FF44F10821182128294
:10F0100013828C2F0E942177F601E750FC4C8591DA
:10F020009591A591B491F601E759F44F80839183AE
:10F03000A283B383C230D1F420914B0B30914C0B9F
:10F0400040914D0B50914E0B6091710B7091720B72
:10F050008091730B9091740B0F9476506093710BA9
:10F060007093720B8093730B9093740B10929713A1
:10F07000109296130E9451D7F601EA5AF44FD60126
:10F08000A759B44F8D919D910D90BC91A02D808377
:10F090009183A283B383C23091F480E0CF911F911A
:10F0A0000F91FF90EF90DF90CF90BF90AF909F9027
:10F0B0008F907F906F905F904F900C94A38CCF9126
:10F0C0001F910F91FF90EF90DF90CF90BF90AF9086
:10F0D0009F908F907F906F905F904F9008951F93B7
:10F0E000CF93DF93882329F0D0911A0BD095D1705C
:10F0F00001C0D0E0662339F010911A0B16951170FB
:10F1000081E0182701C010E0442341F0C0911A0BA0
:10F11000C2FBCC27C0F981E0C82701C0C0E0D111F3
:10F1200005C0111103C0CC2309F444C00E945B62E6
:10F1300083EF93E30E941662DD2319F088E50E94B5
:10F140000462112319F089E50E940462CC2319F0AE
:10F150008AE50E9404628BEE93E30E941662C1115D
:10F1600003C04DE555E002C04FE056E0111103C069
:10F170002DE535E002C02CE736E0D11103C08DE566
:10F1800095E002C08EE796E05F934F933F932F93F5
:10F190009F938F9389ED93E39F938F931F920F9487
:10F1A00070038DB79EB709960FB6F8949EBF0FBE39
:10F1B0008DBFC1E08C2FDF91CF911F9108952F92C9
:10F1C0003F924F925F926F927F928F929F92AF92F7
:10F1D000BF92CF92DF92EF92FF920F931F93CF9344
:10F1E000DF93CDB7DEB7C657D1090FB6F894DEBFAF
:10F1F0000FBECDBF80911502882321F086E59BE0EC
:10F200000E948F7680913B1083FD7DC0C090620B81
:10F21000D090630BE090640BF090650B2091750B20
:10F220003091760B4091770B5091780BC701B60166
:10F230000F948D49882309F466C08091A30B811136
:10F240001FC06091A80B7091A90B8091AA0B90919F
:10F25000AB0B0F94E35120914702309148026217A3
:10F26000730774F4C092750BD092760BE092770B13
:10F27000F092780B0E945B628EEB93E30E94166221
:10F280008090620B9090630BA090640BB090650B24
:10F290002091750B3091760B4091770B5091780B44
:10F2A000C501B4010F9476506B017C0120E030E081
:10F2B000A9010F94D75287FF04C0F7FAF094F7F82A
:10F2C000F0942091430230914402409145025091C4
:10F2D0004602C701B6010F94F34920E030E04AEF3F
:10F2E00053E40F94D752181674F48092750B9092D1
:10F2F000760BA092770BB092780B0E945B628FE93D
:10F3000093E30E94166280912A0B009116021091DD
:10F310001702882309F1C0900A0BD0900B0BE090E4
:10F320000C0BF0900D0B20E030E0A901C701B601F5
:10F330000F948D49882309F455C020915E0B3091BC
:10F340005F0B4091600B5091610BC701B6010F94A8
:10F35000D75218160CF446C0B801110F880B990B40
:10F360000F94944920913F02309140024091410214
:10F37000509142020F94F3492AE037ED43E25CE3F7
:10F380000F94F34969837A838B839C83C12CD12C9E
:10F3900076018E010F5F1F4F22E63BE04EE55BE0FA
:10F3A0006AE57BE086E59BE00E9435B10E941FD0B4
:10F3B000CA58DF4F0FB6F894DEBF0FBECDBFDF9146
:10F3C000CF911F910F91FF90EF90DF90CF90BF9062
:10F3D000AF909F908F907F906F905F904F903F90F5
:10F3E0002F900895B801110F880B990B0F94944931
:10F3F00020913F02309140024091410250914202DF
:10F400000F94F3492AE037ED43E25CE30F94F349AC
:10F410006DA77EA78FA798ABB091690BBFABE091AA
:10F420006A0BEBAFF0916B0BFFAFE0906C0B21968A
:10F43000EFAE219700916D0B10916E0B20916F0B29
:10F440003091700B25960CAF1DAF2EAF3FAF2597B7
:10F450008091710B9091720BA091730BB091740B12
:10F46000A3968CAF9DAFAEAFBFAFA397E090750BE7
:10F47000F090760B0091770B1091780BA796ECAE7D
:10F48000FDAE0EAF1FAFA797C090560BD090570B95
:10F49000E090580BF090590BC982DA82EB82FC8223
:10F4A00080905A0B90905B0BA0905C0BB0905D0B22
:10F4B0008D829E82AF82B88600915E0B10915F0BA9
:10F4C0002091600B3091610B09AB1AAB2BAB3CABBD
:10F4D00009871A872B873C874090620B5090630BFB
:10F4E0006090640B7090650B4D865E866F86788A9F
:10F4F00020E030E040E751E46FA97E2F8F2F219666
:10F500009FAD21970F94765024EB32EC46E65CE3F6
:10F510000F94F3490F94E351653014F064E002C096
:10F5200067FD60E0262F660F330B3EAB2DAB20E06E
:10F5300030E040E751E425966CAD7DAD8EAD9FADDA
:10F5400025970F94765021EA3EE04AE65CE30F945B
:10F55000F3490F94E351653014F064E002C067FD95
:10F5600060E0862F660F990B2D969FAF8EAF2D977B
:10F5700020E030E040E751E4C701B6010F94765037
:10F5800024EB32EC46E65CE30F94F3490F94E3512D
:10F5900029966FAF299765302CF094E029969FAF9C
:10F5A000299708C02996AFAD2997A7FF03C02996D0
:10F5B0001FAE29972996EFAD29970E2E000CFF0B51
:10F5C0002F96FFAFEEAF2F9720E030E040E751E4F9
:10F5D000C501B4010F94765021EA3EE04AE65CE3AF
:10F5E0000F94F3490F94E35128966FAF2897653035
:10F5F0002CF0F4E02896FFAF289708C028960FADAE
:10F60000289707FF03C028961FAE289728962FAD8E
:10F610002897022E000C330B27963FAF2EAF27976B
:10F620008DA99EA92F96AEADBFAD2F978A179B07C8
:10F6300009F01CC12D960EAD1FAD2D9727962EAD4E
:10F640003FAD27970217130709F010C189809A80F0
:10F65000AB80BC8029968FAD29970E9480969B0134
:10F66000AC012F966EAD7FAD2F976F5F7F4FA5E0FA
:10F67000A69FC001A79F900D11242796EEADFFAD68
:10F680002797E80FF91FEE0FFF1FEE0FFF1FEA5538
:10F69000F54FE080F18002811381EFAAF8AE09AF47
:10F6A0001AAF2F960EAD1FAD2F97A09FB001A19F4F
:10F6B000700D11242796EEADFFAD2797E60FF71FCB
:10F6C000EE0FFF1FEE0FFF1FEA55F54F40805180F0
:10F6D000628073802796AEADBFAD27971196FC016F
:10F6E000EA0FFB1FEE0FFF1FEE0FFF1FEA55F54F4E
:10F6F000E080F18002811381EBAEFCAE0DAF1EAF56
:10F70000A60FB71FAA0FBB1FAA0FBB1FAA55B54F45
:10F71000CD90DD90ED90FC9029960FAD29970430A7
:10F7200089F1C501B4010F94765024EB32EC46E622
:10F730005CE30F94F3494B015C01A30192016FA9B3
:10F7400078AD89AD9AAD0F947650A50194010F94D0
:10F75000F349A30192010F9477502B013C01A701BB
:10F7600096016BAD7CAD8DAD9EAD0F947650A5012D
:10F7700094010F94F349A70196010F9477506B0100
:10F780007C0105C0C12CD12C7601260137018D806A
:10F790009E80AF80B88428968FAD28970E9452969D
:10F7A0009B01AC0128961FAD2897143059F1C50173
:10F7B000B4010F94765021EA3EE04AE65CE30F94F0
:10F7C000F3494B015C01A3019201C701B6010F94FB
:10F7D00076509B01AC01C501B4010F94F349A3011C
:10F7E00092010F9477506B017C01CE0109960E9423
:10F7F000A5CF9B01AC01C701B6010F94F3496B0182
:10F800007C0103C0C12CD12C76011D8A1E8A1F8A5F
:10F81000188E89849A84AB84BC84A7019601C701A1
:10F82000B6010F94C453882319F0C12CD12C760152
:10F83000A7019601C501B4010F947750698B7A8BAB
:10F840008B8B9C8B9E012B5E3F4F79018E01035D5C
:10F850001F4F28503109AE014F5E5F4FBE016B5FF5
:10F860007F4FCE0101960E94FFA1A0CD2FA93BADF5
:10F870004FAD21965FAD2197C701B6010F94765029
:10F880006B017C0125962CAD3DAD4EAD5FAD25974E
:10F89000C501B4010F9476504B015C0181E090E00A
:10F8A0002B969FAF8EAF2B9720E030E0A901C501CA
:10F8B000B4010F948D4987FD04C02B961FAE1EAE78
:10F8C0002B9720E030E0A901C701B6010F948D49C4
:10F8D00087FF0AC097018601305863960CAF1DAFB1
:10F8E0002EAF3FAF639706C06396CCAEDDAEEEAEF3
:10F8F000FFAE639720E030E0A901C501B4010F9489
:10F900008D4987FF0AC0D501C401B05867968CAFF6
:10F910009DAFAEAFBFAF679706C067968CAE9DAE8A
:10F92000AEAEBFAE6797ADA9BEA92F96EEADFFAD47
:10F930002F97AE17BF0781F020E030E0A901C70183
:10F94000B6010F948D4987FF0CC00FEF1FEF6D9626
:10F950001FAF0EAF6D970BC06D961FAE1EAE6D97AD
:10F9600006C021E030E06D963FAF2EAF6D972D962B
:10F970008EAD9FAD2D972796AEADBFAD27978A1759
:10F980009B0781F020E030E0A901C501B4010F948C
:10F990008D4987FF0CC0EFEFFFEF6F96FFAFEEAF23
:10F9A0006F970BC06F961FAE1EAE6F9706C001E03B
:10F9B00010E06F961FAF0EAF6F9767962CAD3DAD01
:10F9C0004EAD5FAD679763966CAD7DAD8EAD9FAD6F
:10F9D00063970F94D75218161CF01401850102C0CA
:10F9E00016018701A7962CAD3DAD4EAD5FADA79733
:10F9F000C301B2010F94765069A77AA78BA79CA781
:10FA00009101A8010F947151AB966CAF7DAF8EAF91
:10FA10009FAFAB97A3962CAD3DAD4EAD5FADA39719
:10FA200069A97AA98BA99CA90F9476509101A80184
:10FA30000F947151E1966CAF7DAF8EAF9FAFE197A0
:10FA4000A7019601C501B4010F9471516B966CAF7B
:10FA50007DAF8EAF9FAF6B979B01AC016FA97BAD64
:10FA60008FAD21969FAD21970F94F3499B01AC0177
:10FA700025966CAD7DAD8EAD9FAD25970F947650DC
:10FA8000E5966CAF7DAF8EAF9FAFE597AB964CAC74
:10FA90005DAC6EAC7FACAB97E89477F86D962EAD0D
:10FAA0003FAD6D97232B09F038C12D962EAC3FAC9E
:10FAB0002D972B968EAD9FAD2B97280E391E27962E
:10FAC000AEADBFAD2797A80FB91F2B96BFAFAEAF96
:10FAD0002B976B960CAD1DAD2EAD3FAD6B973F7761
:10FAE00009AB1AAB2BAB3CAB2B962EAD3FAD2B9796
:10FAF0002215330509F463C46F968EAD9FAD6F97E1
:10FB0000280E391E122D822D0E9452966B017C0107
:10FB10002FEF3FEF4FE75FE769A97AA98BA99CA96F
:10FB20000F94C45381110CC02FEF3FEF4FE75FE7F5
:10FB300069A97AA98BA99CA90F948D491816ACF0D4
:10FB4000E5962CAD3DAD4EAD5FADE597C701B60175
:10FB50000F9476506B962CAD3DAD4EAD5FAD6B976F
:10FB60000F947151362F272F06C03FA92BAD8FADB3
:10FB700021969FAD2197432F522FBC014D8F5E8F51
:10FB80006F8F78A395E02916310450F4A1016DA977
:10FB90007EA9CE014D960E943ECF6B017C0103C031
:10FBA000C12CD12C7601CE0109960E94A5CFA701C8
:10FBB00096010F94F3496B017C019B01AC010F94FA
:10FBC000C453882319F0C12CD12C7601812F0E94B7
:10FBD00052964B015C01698F7A8F8B8F9C8F9B01B2
:10FBE000AC0125966CAD7DAD8EAD9FAD25970F9484
:10FBF0008D49882309F478CF2FEF3FEF4FE75FE778
:10FC0000C301B2010F94C45381110BC02FEF3FEF1A
:10FC10004FE75FE7C301B2010F948D4918160CF44A
:10FC200050C067962CAD3DAD4EAD5FAD6797639606
:10FC30006CAD7DAD8EAD9FAD63970F94D752181606
:10FC40005CF42FA93BAD4FAD21965FAD21976D8D33
:10FC50007E8D8F8D98A108C025962CAD3DAD4EAD03
:10FC60005FAD2597C501B4010F9476504B015C013F
:10FC70009B01AC01AB966CAD7DAD8EAD9FADAB97EE
:10FC80000F94F349A7962CAD3DAD4EAD5FADA79750
:10FC90000F94775069A77AA78BA79CA7A501940119
:10FCA000E1966CAD7DAD8EAD9FADE1970F94F349BC
:10FCB000A3962CAD3DAD4EAD5FADA3970F9477509D
:10FCC0000CC08D859E85AF85B88989A79AA7ABA7FB
:10FCD000BCA769857A858B859C851D8A1E8A1F8AAB
:10FCE000188EA70196010F947750698B7A8B8B8BB6
:10FCF0009C8BDE0155967D018E01035D1F4F9E0199
:10FD0000275D3F4FAE014F5E5F4FBE01675E7F4F85
:10FD1000CE014D960E94FFA1E7CEE1E0F0E0FAAB04
:10FD2000E9AB20E030E0A901C701B6010F948D498D
:10FD300087FD02C01AAA19AA2DA83EA8E9A8FAA808
:10FD40002E0C3F1C6F960EAD1FAD6F97012B09F067
:10FD5000FDC02F962EAD3FAD2F972E0D3F1D3AAB18
:10FD600029AB89A99AA98215930509F428C36D9630
:10FD7000AEADBFAD6D972A0E3B1E122D822D0E9497
:10FD800080969B01AC016B966CAD7DAD8EAD9FAD49
:10FD90006B970F94F349E5962CAD3DAD4EAD5FAD3D
:10FDA000E5970F9477506D8F7E8F8F8F98A3B5E076
:10FDB0002B16310460F42D964EAD5FAD2D97B10139
:10FDC000CE014D960E94D7CE6B017C0103C0C12CA1
:10FDD000D12C7601CE0109960E94A5CFA7019601EC
:10FDE0000F94F3496B017C019B01AC010F94C45348
:10FDF000882319F0C12CD12C7601812F0E94809686
:10FE00004B015C01698F7A8F8B8F9C8F9B01AC01BA
:10FE10006FA97BAD8FAD21969FAD21970F948D4932
:10FE2000882309F49ECF2FEF3FEF4FE75FE7C30131
:10FE3000B2010F94C45381110BC02FEF3FEF4FE776
:10FE40005FE7C301B2010F948D4918160CF450C03E
:10FE500067962CAD3DAD4EAD5FAD679763966CADCB
:10FE60007DAD8EAD9FAD63970F94D75218164CF4AD
:10FE70002FA93BAD4FAD21965FAD2197C501B401D0
:10FE80000AC025962CAD3DAD4EAD5FAD25976D8D6D
:10FE90007E8D8F8D98A10F9476504B015C019B0154
:10FEA000AC01AB966CAD7DAD8EAD9FADAB970F94B5
:10FEB000F349A7962CAD3DAD4EAD5FADA7970F941E
:10FEC000775069A77AA78BA79CA7A5019401E19613
:10FED0006CAD7DAD8EAD9FADE1970F94F349A396C8
:10FEE0002CAD3DAD4EAD5FADA3970F9477500CC0D8
:10FEF0008D859E85AF85B88989A79AA7ABA7BCA732
:10FF000069857A858B859C851D8A1E8A1F8A188E35
:10FF1000A70196010F947750698B7A8B8B8B9C8B02
:10FF2000FE0175967F018E01035D1F4F9E01275DC7
:10FF30003F4FAE014F5E5F4FBE01635E7F4FCE010C
:10FF400049960E94FFA181110CCF39C22D968EAD2A
:10FF50009FAD2D972796EEACFFAC27978E199F0982
:10FF60006DA97EA92F960EAD1FAD2F97601B710B4B
:10FF700077FF03C0719561957109E7967FAF6EAF0A
:10FF8000E79797FF03C0919581959109AD969FAF33
:10FF90008EAFAD973EAA2DAA2D962EAC3FAC2D97D5
:10FFA0002B962EAD3FAD2B97220E331EE7968EADCE
:10FFB0009FADE797892B39F4AD96AEADBFADAD9748
:10FFC000AB2B09F4FCC18DA96C96BFAD6C978B0F60
:10FFD0000E9480966DA37EA38FA398A76E968FAD87
:10FFE0006E97820D0E9452964B015C0169A37AA321
:10FFF0008BA39CA3CDA0DEA0EFA0F8A4A70196013F
:020000021000EC
:100000006B966CAD7DAD8EAD9FAD6B970F94F34944
:10001000E5962CAD3DAD4EAD5FADE5970F947750B5
:100020006D8F7E8F8F8F98A3E5962CAD3DAD4EAD35
:100030005FADE597C501B4010F9476506B962CAD7A
:100040003DAD4EAD5FAD6B970F9471519B01AC010F
:10005000698F7A8F8B8F9C8F01E010E0C701B6010A
:100060000F948D4987FD02C000E010E0E9A9FAA9CC
:100070000E171F0709F0CEC06F96EEACFFAC6F975E
:100080002E0C3F1C6DA97EA96E1B7F0B6530710580
:1000900060F405E02016310440F4A101CE01499638
:1000A0000E943ECF6B017C0103C0C12CD12C760194
:1000B000CE0109960E94A5CFA70196010F94F3499E
:1000C0006B017C019B01AC010F94C453882319F090
:1000D000C12CD12C76012FEF3FEF4FE75FE7C30133
:1000E000B2010F94C45381110BC02FEF3FEF4FE7C4
:1000F0005FE7C301B2010F948D4918160CF452C08A
:1001000067962CAD3DAD4EAD5FAD679763966CAD18
:100110007DAD8EAD9FAD63970F94D75218165CF4EA
:100120002FA93BAD4FAD21965FAD2197698D7A8D9B
:100130008B8D9C8D0AC025962CAD3DAD4EAD5FAD2F
:10014000259769A17AA18BA19CA10F9476504B01B0
:100150005C019B01AC01AB966CAD7DAD8EAD9FADEE
:10016000AB970F94F349A7962CAD3DAD4EAD5FAD67
:10017000A7970F94775069A77AA78BA79CA7A5018B
:100180009401E1966CAD7DAD8EAD9FADE1970F947E
:10019000F349A3962CAD3DAD4EAD5FADA3970F9443
:1001A00077500CC08D859E85AF85B88989A79AA7A1
:1001B000ABA7BCA769857A858B859C851D8A1E8A1D
:1001C0001F8A188EA70196010F947750698B7A8B3E
:1001D0008B8B9C8B9E012B5E3F4F79018E01035DC3
:1001E0001F4F2C5E3F4FAE014F5E5F4FBE016F5DF4
:1001F0007F4FCE0149960E94FFA1882309F4DFC0FA
:10020000AD968EAD9FADAD970197AD969FAF8EAF7A
:10021000AD97D2C0EDA9FEA96D96EEACFFAC6D977F
:10022000EE0DFF1DFEABEDABE530F10590F4A10145
:100230002B960EAD1FAD2B97401B510B4530510532
:1002400040F4BF01CE014D960E94D7CE6B017C01D8
:1002500003C0C12CD12C7601CE0109960E94A5CFF6
:10026000A70196010F94F3496B017C019B01AC013E
:100270000F94C453882319F0C12CD12C76012FEF91
:100280003FEF4FE75FE7C301B2010F94C453811101
:100290000BC02FEF3FEF4FE75FE7C301B2010F94B1
:1002A0008D4918160CF452C067962CAD3DAD4EAD7D
:1002B0005FAD679763966CAD7DAD8EAD9FAD639777
:1002C0000F94D75218165CF42FA93BAD4FAD219671
:1002D0005FAD21976DA17EA18FA198A50AC025963B
:1002E0002CAD3DAD4EAD5FAD25976D8D7E8D8F8D67
:1002F00098A10F9476504B015C019B01AC01AB9629
:100300006CAD7DAD8EAD9FADAB970F94F349A796C5
:100310002CAD3DAD4EAD5FADA7970F94775069A75B
:100320007AA78BA79CA7A5019401E1966CAD7DAD42
:100330008EAD9FADE1970F94F349A3962CAD3DADE3
:100340004EAD5FADA3970F9477500CC08D859E8501
:10035000AF85B88989A79AA7ABA7BCA769857A8515
:100360008B859C851D8A1E8A1F8A188EA70196017F
:100370000F947750698B7A8B8B8B9C8B9E012B5EB5
:100380003F4F79018E01035D1F4F2C5E3F4FAE0141
:100390004F5E5F4FBE01635E7F4FCE0185960E9428
:1003A000FFA1882361F0E7968EAD9FADE797019797
:1003B000E7969FAF8EAFE797019609F0F7CD2981B9
:1003C0003A814B815C816091690B70916A0B8091DD
:1003D0006B0B90916C0B0F948D49811137C92D8156
:1003E0003E814F81588560916D0B70916E0B8091AD
:1003F0006F0B9091700B0F948D49811127C90C944C
:10040000D6798091260B9091270BA091280BB09163
:10041000290B80933F0290934002A0934102B09336
:1004200042028091240B9091250B909317028093A8
:100430001602089580913F0290914002A0914102DE
:10044000B09142028093260B9093270BA093280B28
:10045000B093290B80911602909117029093250B6F
:100460008093240B84E690E0909317028093160209
:1004700008958F929F92AF92BF92CF92DF92EF92A8
:10048000FF920F931F93CF93DF93EC018B81811128
:1004900002C080E078C009891A892B893C89041739
:1004A000150726073707A8F36A017B01823029F474
:1004B000C886D986EA86FB860DC0C114D104E10442
:1004C000F10451F4188619861A861B861C821D8237
:1004D0001E821F8281E057C088849984AA84BB84CD
:1004E000E98DFA8D258530E0275F3F4FB501A401E6
:1004F0004150510961097109022E04C07695679532
:10050000579547950A94D2F7D701C6010197A109DB
:10051000B10904C0B695A795979587952A95D2F706
:1005200084179507A607B70720F089288A288B2803
:1005300071F44D895E896F89788D4C835D836E83FC
:100540007F834C015D018E010C5F1F4F16C0841B21
:10055000950BA60BB70BF5CF4C815D816E817F812A
:100560009801898D9A8D0E94717291E0891A910883
:10057000A108B108882309F48CCF81149104A10447
:10058000B10451F795CFDF91CF911F910F91FF905B
:10059000EF90DF90CF90BF90AF909F908F90089595
:1005A0000F931F93CF93DF93FC012381222311F03C
:1005B00080E044C08B01EC01FB018789803139F177
:1005C0008032B1F783E08B83F801428D538D648DC7
:1005D000758D4D8B5E8B6F8B788F9E012F5E3F4F9D
:1005E000C8010E94F272882319F31A8F098F81E0E3
:1005F0008983188619861A861B861C821D821E8294
:100600001F82188A1C861D861E861F8617C082E0E0
:100610008B831D8A1E8A1F8A188EFB01808D918D07
:10062000A0E0B0E025E0880F991FAA1FBB1F2A9504
:10063000D1F7898B9A8BAB8BBC8BD7CFDF91CF91C6
:100640001F910F910895CF93DF93EC0141E0611169
:1006500001C040E06C857D858E859F850E94A671D6
:10066000882341F0888920E2829FC0011124885F9D
:10067000984E02C080E090E0DF91CF910895CF9333
:10068000DF93EB01FC012381211102C080E028C02F
:100690002250223020F48FE28883198220C060E04B
:1006A0000E942383009791F3FC0190E080E02EE20A
:1006B0003081303269F0883029F4DE01A90FB11D94
:1006C0002C939F5FDE01A90FB11D30813C939F5F8A
:1006D0008F5F31968B3061F7C90FD11D188281E091
:1006E000DF91CF9108953F924F925F926F927F92E8
:1006F0008F929F92AF92BF92CF92DF92EF92FF9232
:100700000F931F93CF93DF93CDB7DEB72C970FB620
:10071000F894DEBF0FBECDBF5C01DC0159968D9011
:100720009C905A97F40181859285A385B4859C019C
:10073000AD012F5F3F4F4F4F5F4F29873A874B8760
:100740005C87D5011496CD90DD90ED90FC901797C5
:10075000C114D104E104F10439F0BFEFCB1ADB0A74
:10076000EB0AFB0A312C07C0F401C080D180E28083
:10077000F38033243394260137011D821E821F82A9
:100780001886F40181859285A385B4852D813E81EB
:100790004F815885281739074A075B0708F064C05E
:1007A00089859A85AB85BC858C159D05AE05BF05F1
:1007B00050F482E0C82ED12CE12CF12C92E0492E8D
:1007C000512C612C712C9E012F5F3F4FB701A60168
:1007D000C4010E947172882309F446C089819A81FC
:1007E000AB81BC81892B8A2B8B2B41F026013701F1
:1007F0009FEF491A590A690A790A05C0C414D50439
:10080000E604F70491F02D813E814F8158852F5FDA
:100810003F4F4F4F5F4F2D833E834F8358873FEFAE
:10082000C31AD30AE30AF30AACCF0FEF1FEF2FEF7F
:100830003FE0B301A201C4010E94DF71F82E8823BA
:1008400099F0D50114964D915D916D917C9117971A
:10085000411551056105710549F093018201C401FB
:100860000E94DF71811102C0F12C29C0D5011496BC
:100870004D925D926D927C921797332051F0D30187
:10088000C2010196A11DB11DF40180839183A28351
:10089000B383F50185899689A789B08D892B8A2B29
:1008A0008B2B69F4D50155964D925D926D927C9299
:1008B000589711968C911197806811968C938F2D73
:1008C0002C960FB6F894DEBF0FBECDBFDF91CF914F
:1008D0001F910F91FF90EF90DF90CF90BF90AF905E
:1008E0009F908F907F906F905F904F903F90089572
:1008F00040E050E0BA010C94398261E0FC01808153
:100900000F942B338FEF0C94BF6AEF92FF921F93DB
:10091000CF93DF9300D01F92CDB7DEB77C01162FA7
:1009200029833A834B835C83FC0182810E94CB6ADA
:1009300060E0F70180810F942B330F94192F812FE2
:1009400080640E94BF6A8C810E94BF6A8B810E9472
:10095000BF6A8A810E94BF6A89810E94BF6A11238F
:1009600011F087E801C085E90E94BF6A1C3011F4CC
:100970000E94C46A10E00E94C46AF701838387FF63
:1009800004C01F3F11F01F5FF6CF0F900F900F9024
:100990000F90DF91CF911F91FF90EF9008950F93EB
:1009A0001F93CF93DF93EC0189018C81833039F061
:1009B00089E0440F551F661F771F8A95D1F79A016A
:1009C000AB0168E1CE010E948584811128C08EEFC1
:1009D0008EBDF801C8019E5F0DB407FEFDCF2081DA
:1009E0002EBD0DB407FEFDCF21812EBD32968E1790
:1009F0009F0791F70DB407FEFDCF8FEF0E94BF6AEE
:100A00008FEF0E94BF6A0E94C46A8B838F7185300A
:100A100041F083E18983CE010E947D8419C086E084
:100A200016C00F94192F882379F020E030E0A90137
:100A30006DE0CE010E948584811108C00E94C46AC5
:100A4000811104C011E005C087E101C086E18983FE
:100A500010E0CE010E947D84812FDF91CF911F9104
:100A60000F910895CF93809110198823B9F1409187
:100A700008195091091960910A1970910B1928E011
:100A800037E180911119909112190E94CF84C82FDB
:100A9000811102C0C0E023C040910C1950910D1982
:100AA00060910E1970910F1941155105610571057D
:100AB00091F028E037E180911119909112190E946C
:100AC000CF84882339F310920C1910920D191092CB
:100AD0000E1910920F191092101901C0C1E08C2F3D
:100AE000CF910895CF93DF93EC018B81882339F167
:100AF000898187FF20C061E0CE010E942383FC0131
:100B0000892BE9F08081853ED1F08B81823040F4E1
:100B100089899A89AB89BC89848F958FA68FB78F75
:100B20008D899E89AF89B88D938F828FB58BA48B69
:100B300089818F778983DF91CF910C94328581E011
:100B4000888380E0DF91CF910895CF93DF93EC010C
:100B50000E9472851B82DF91CF910895FC01238151
:100B600021110C94A5850895CF92DF92EF92FF9208
:100B70000F931F93CF93DF93EC0189018C81833016
:100B800039F089E0440F551F661F771F8A95D1F70A
:100B90009A01AB0161E1CE010E948584882339F07E
:100BA00084E08983CE010E947D8480E03EC00F9462
:100BB000B8346B017C012CE2C20E21E0D21EE11C94
:100BC000F11C0E94C46A8B838F3F61F40F94B83488
:100BD000DC01CB018C199D09AE09BF09B7FDF1CF2E
:100BE00081E11DC08E3FD1F48FEF8EBDF801D80199
:100BF000A150BE4F0DB407FEFDCF9EB591938EBDA3
:100C0000EA17FB07B9F70DB407FEFDCF8EB58C933D
:100C10000E94C46A0E94C46A11E003C08FE0898305
:100C200010E0CE010E947D84812FDF91CF911F9132
:100C30000F91FF90EF90DF90CF9008952F923F9209
:100C40004F925F926F927F928F929F92AF92BF92DC
:100C5000CF92DF92EF92FF920F931F93CF93DF9388
:100C600000D01F92CDB7DEB79C838B834B015A0116
:100C7000DC0113968C91811103C08FEF9FEFE3C0CD
:100C8000EB81FC81818180FFF8CFEB81FC81818940
:100C90009289A389B4894085518562857385841BB7
:100CA000950BA60BB70BA50160E070E084179507C4
:100CB000A607B70708F45C0175018B819C81049637
:100CC0009A838983612C42E0742EE114F10409F4C3
:100CD0008BC0AB81BC8118964D915D916D917C91DB
:100CE0001B976A01B1E0DB22EB81FC812381818DBE
:100CF000928D1A012B0139E056944794379427942A
:100D00003A95D1F7223061F4FC01828D938DA48D48
:100D1000B58DBC01CD01620D731D841D951D4AC0AA
:100D2000DC0114961C9111501221C114D10401F55B
:100D300011111EC0452B462B472B59F4EB81FC812A
:100D400085899689A789B08D84839583A683B78387
:100D50000FC0AB81BC8114964D915D916D917C91DA
:100D6000179729813A810E947172882309F485CFEF
:100D7000EB81FC81218D328D84819581A681B781A3
:100D80000297A109B109F901058404C0880F991FD0
:100D9000AA1FBB1F0A94D2F74685578560897189BF
:100DA000840F951FA61FB71FBC01CD01610F711DD8
:100DB000811D911D93012C193D0987012E153F05B9
:100DC00008F489010115F2E01F0779F5209108194F
:100DD0003091091940910A1950910B196217730744
:100DE0008407950719F421C0C5012DC09401AB01FA
:100DF000BC0180911119909112190E94B485882329
:100E000009F43BCF800E911EEB81FC81808591859A
:100E1000A285B385800F911FA11DB11D8087918789
:100E2000A287B387E01AF10A50CF40E00E94A67172
:100E3000882309F422CFB601685F784EA801C40167
:100E40000F94F654DFCF0F900F900F900F90DF911B
:100E5000CF911F910F91FF90EF90DF90CF90BF90B7
:100E6000AF909F908F907F906F905F904F903F904A
:100E70002F900895DF92EF92FF920F931F93CF93DD
:100E8000DF938C01EB017A018DE0D82E40E250E037
:100E9000BE01C8010E941E868032910539F021E012
:100EA000892B09F420E0822F819544C028812223D8
:100EB000C9F1253E11F02E3231F4E114F10431F381
:100EC000F7011082E3CFE114F10441F13B853F7358
:100ED0003F3021F54A8D5B8D452B01F52F713FEF9A
:100EE000320F3530D8F430E021503109D29EC001A4
:100EF000D39E900D1124D701A80FB91FFE0120E049
:100F0000AD01253088F431813D932F5F32962D302D
:100F1000C1F7288126FF02C0FA0115862B8523FD23
:100F2000B5CF08C080E006C02B3010F43481ECCF80
:100F30003681EACFDF91CF911F910F91FF90EF9013
:100F4000DF9008954F925F926F927F929F92AF923F
:100F5000BF92CF92DF92EF92FF920F931F93CF93A6
:100F6000DF931F92CDB7DEB78C017B015A01C22EF1
:100F7000DB0159968D919C915A97F801928F818F40
:100F8000CB010E947884912CF70180859185A28500
:100F9000B385418952896389748984179507A607A7
:100FA000B70708F060C025E0B695A7959795879597
:100FB0002A95D1F7F82FFF70DF2ED70113968C9169
:100FC000823008F460C041E050E0BE016F5F7F4FA7
:100FD000C7010E941E86019719F4898190E002C022
:100FE0008FEF9FEF019609F44EC0F7018085918540
:100FF000A285B3854F96A11DB11D80879187A287D9
:10100000B387F0E2DF9EB0011124685F784E61156E
:101010007105C9F1DB018C91882319F0853EC1F47B
:101020006CC191100EC08091081990910919A0917E
:101030000A19B0910B19F80184879587A687B7879D
:10104000D08ADB018C91882361F0992493949CCF02
:101050004BE050E0C5010F94E954892B09F094CF7F
:1010600014C0992493948C2D8274823461F4992055
:1010700009F48BC0F801D08861E0C8010E94238385
:10108000009709F00DC180E03BC1C7FCFCCFF0E246
:10109000DF9EA00111249A01285F384ED9011B96CA
:1010A0008C91817121F08C2D827109F06AC0809140
:1010B000081990910919A0910A19B0910B19F8011A
:1010C00084879587A687B787D08ACA01885F984E9C
:1010D0007C01DC0154964D915C91559760E070E085
:1010E000DA0199278827858B968BA78BB08FF7011C
:1010F000428D538D60E070E0482B592B6A2B7B2B7F
:10110000D80155964D935D936D937C935897F90153
:101110008385887161F4F701848D958DA68DB78DD7
:10112000F801818B928BA38BB48B81E010C080314E
:1011300041F598012F5E3F4FD80159968D919C91B2
:101140005A970E94F2728823E1F084E0F8018383C9
:101150008C2D8F70D80111968C931197F801148201
:1011600015821682178218961D921D921D921C924E
:101170001B97C4FEB5C0C8010F943D2F8111B0C0AC
:1011800082CFD80113961C927ECFD70113968C91F3
:101190001397823009F477CF51968D919D910D90E0
:1011A000BC91A02D803E9F4FAF41B10508F06BCFA1
:1011B000C7010E947383882309F465CF0E9432859A
:1011C000882309F460CFD70159962D913C915A9705
:1011D00014968D919D910D90BC91A02D0297A1091F
:1011E000B109F901058404C0880F991FAA1FBB1F0C
:1011F0000A94D2F74684578460887188480E591E35
:101200006A1E7B1E81E0809310194092081950924B
:10121000091960920A1970920B1980E092E0E8E0D7
:10122000F7E1DF019C011D9221503040E1F7DD2400
:10123000D394D7015996ED91FC915A978481D81691
:1012400098F428E037E1B301A2014D0D511D611D55
:10125000711D80911119909112190E94CF848823D9
:1012600009F411CFD394E5CF80E092E0A0E0B0E0A4
:10127000058404C0880F991FAA1FBB1F0A94D2F7C8
:10128000F7014189528963897489840F951FA61FCC
:10129000B71F818B928BA38BB48B88E097E1D12C05
:1012A00020E2DC011D922A95E9F72BE0F501DC0133
:1012B00001900D922A95E1F721E238E2FC01318B91
:1012C000208B40E058E057874687338B228B318F45
:1012D000208F578B468B0E9432858111D8CED3CE7A
:1012E000C5FE09C0F8014189528963897489C80122
:1012F0000E94398205C081E003C09110A6CE93CE32
:101300000F90DF91CF911F910F91FF90EF90DF90A1
:10131000CF90BF90AF909F907F906F905F904F90D5
:1013200008952F923F924F925F926F927F928F9289
:101330009F92AF92BF92CF92DF92EF92FF920F9364
:101340001F93CF93DF93CDB7DEB7C254D1090FB649
:10135000F894DEBF0FBECDBF4C015B016A01322E97
:1013600019821C821C8E1F8E6115710511F410E00C
:10137000A6C0FC0183818111FACFFA0180818F32EE
:1013800009F09BC0F50183818250823010F4850101
:101390000CC0F501618D728DCE014C960E94D082F9
:1013A000882329F38E01045E1F4FC6016C0101964C
:1013B000F60120812F32D1F3CE0101967C013C0150
:1013C0002E019CE1490E511C2396EFAE23972F2C42
:1013D0009BE09150E7E3F0E0EC0FFD1FE90FF11DFA
:1013E00080E280839111F5CF960147E0D9018D917C
:1013F000882369F18F3259F18E3239F44A3009F479
:10140000B6CF98E04AE09D01F1CFE3E6F4E3249102
:10141000222321F031968213FACFA9CF491708F47D
:10142000A6CF813208F4A3CF8F3709F4A0CF21E0F3
:10143000290FE7E3F0E0EC0FFD1FE90FF11D9FE935
:10144000980F9A3108F480528083922FDCCF8FA9B5
:10145000803209F48CCF6901F90180812F5F3F4F01
:101460008F32C9F38823F9F021E0AE01495C5F4F68
:10147000B801C7010E94A287882309F478CF0A1512
:101480001B0519F0C8010E94A5856E147F0441F068
:1014900023969FAD2397822D8701E92EF82E98CFB2
:1014A000942D852DF9CF232DAE01495C5F4FB801F6
:1014B000C4010E94A287182F02C08B017DCFCE01EC
:1014C0004C960E94AE85CE0101960E94AE85812F7A
:1014D000CE5BDF4F0FB6F894DEBF0FBECDBFDF91FE
:1014E000CF911F910F91FF90EF90DF90CF90BF9021
:1014F000AF909F908F907F906F905F904F903F90B4
:101500002F900895CF93C82F0E945B6284E50E94BC
:1015100004626AE070E08C2F90E00E945A6380E2DF
:101520000E94046281E594E3CF910C9416622091AD
:101530001202309113022F503109821793070CF4D5
:101540009C013093AD0B2093AC0B80E00C94E2F83F
:101550008091AD149091AE14891B8F708F3021F45F
:1015600080E00E942E65F4CF8091AD148F5F8F7064
:10157000E091AD1498E49E9FF0011124E554F44FDE
:10158000DF011D929A95E9F798E090834091C3148A
:101590005091C4146091C5147091C614458B568B3C
:1015A000678B708F4091C7145091C8146091C91413
:1015B0007091CA14418F528F638F748F4091CB14F6
:1015C0005091CC146091CD147091CE14458F568FEC
:1015D000678F70A34091CF145091D0146091D114B3
:1015E0007091D21441A352A363A374A32091AD14AC
:1015F0009091AE14291303C094E69093AA1480939B
:10160000AD1480916F00826080936F0008950F93F6
:101610000FB70F9300916E000F930B7F00936E0036
:1016200000916F000D7F00936F000F930BB70F9326
:101630000CB70F921F922F933F934F935F936F932B
:101640007F938F939F93AF93BF93EF93FF93112457
:101650000E948CB7FF91EF91BF91AF919F918F91B5
:101660007F916F915F914F913F912F911F900F90BC
:101670000CBF0F910BBF0F910260F89400936F00A5
:101680000F9100936E000F910FBF0F9118958091ED
:101690009D0880FF03C089988FEF02C0899A81E07E
:1016A0008093981080919D08869580FF03C08F9A43
:1016B0008FEF02C08F9881E08093991080919D08F0
:1016C0008695869580FF08C080910B018095827079
:1016D000809309018FEF06C080910B018270809387
:1016E000090181E080939A1080919D0886958695E6
:1016F000869580FF03C016988FEF02C0169A81E08E
:1017000080939B1000000000000008958091AD14AC
:101710009091AE14891B8F7019F480E090E00895C9
:101720009091AA14992351F0833030F48FEF890FF0
:1017300019F08093AA14F1CF1092AA14E091AE147C
:1017400088E4E89FF0011124E554F44F808180FD86
:10175000E4CF8091AE148F5F8F708093AB14909123
:10176000AE148091AC14981304C08091AB14809394
:10177000AC14CF010895CF92DF92EF92FF92CF93F6
:10178000DF93EC016A017B0127E137EB41ED58EB78
:10179000C701B6010F94D75287FD23C023E030E084
:1017A0004BE953E4C701B6010F948D491816CCF0EC
:1017B000C880D980EA80FB8027E137EB41ED58EB08
:1017C000C701B6010F94D75287FD0BC0C1E023E0DB
:1017D00030E84DE953E4C701B6010F948D4918165E
:1017E0000CF4C0E08C2FDF91CF91FF90EF90DF9051
:1017F000CF9008958F929F92AF92BF92CF92DF9237
:10180000EF92FF921F93CF93DF9300D01F92CDB73B
:10181000DEB74B015C0169017A0120E030E048ED60
:1018200051E40F94775069837A838B839C83B7014B
:10183000A601CE0101960E94BB8B182F882351F17F
:101840002EE23FEF4FE950E4C501B4010F94D752A7
:1018500087FD1FC023E030E040E953E4C501B40137
:101860000F948D491816ACF02EE23FEF4FE950E48B
:10187000C701B6010F94D75287FD0BC011E023E0DA
:1018800030E848E953E4C701B6010F948D491816B2
:101890000CF410E0812F0F900F900F900F90DF91BC
:1018A000CF911F91FF90EF90DF90CF90BF90AF90BE
:1018B0009F908F900895CF92DF92EF92FF92CF93F7
:1018C000DF93CDB7DEB728970FB6F894DEBF0FBE13
:1018D000CDBF20E030E040EA50E46091710B7091A0
:1018E000720B8091730B9091740B0F948D49882328
:1018F000E9F01D821E821F821886C12CD12C80EA3D
:10190000E82E80E4F82EC982DA82EB82FC82BE01E6
:101910006B5F7F4FCE0101960E94A8D6C092710BDB
:10192000D092720BE092730BF092740B28960FB664
:10193000F894DEBF0FBECDBFDF91CF91FF90EF9047
:10194000DF90CF900895BF92CF92DF92EF92FF92F7
:101950000F931F93CF93DF93CDB7DEB728970FB6C2
:10196000F894DEBF0FBECDBF90919E08981709F482
:101970007DC0B82E882309F454C080E090E0A0E236
:10198000B1E48D839E83AF83B887C0904B0BD0901A
:101990004C0BE0904D0BF0904E0B20E030E0A90195
:1019A000C701B6010F948D4987FF0CC0A7019601AE
:1019B00060E070E080E291E40F9476506D837E8366
:1019C0008F83988720E030E048EC53E46D817E817E
:1019D0008F8198850F94D752181644F480E090E0D8
:1019E000A8ECB3E48D839E83AF83B8872D813E81BD
:1019F0004F8158856091710B7091720B8091730BC0
:101A00009091740B0F948D4987FF0BC019821A8235
:101A10001B821C82BE016F5F7F4FCE0105960E9424
:101A2000A8D66091690B70916A0B80916B0B9091B5
:101A30006C0B20916D0B30916E0B40916F0B5091A0
:101A4000700B19821A821B821C82E090710BF0903D
:101A5000720B0091730B1091740BFE0131966F01A4
:101A60000E94C9D5B0929E080E94E3D780E02896D4
:101A70000FB6F894DEBF0FBECDBFDF91CF911F919F
:101A80000F91FF90EF90DF90CF90BF9008952F922D
:101A90003F924F925F926F927F928F929F92AF92FE
:101AA000BF92CF92DF92EF92FF920F931F93CF934B
:101AB000DF93CDB7DEB7AE970FB6F894DEBF0FBE9B
:101AC000CDBF9DA78CA71B0149A72EA7DC01CD90F8
:101AD000DD90ED90FC90CDA2DEA2EFA2F8A6FB0176
:101AE00040805180628073800023B1F0A301920195
:101AF000C701B6010E94FA8B882309F488C220E04E
:101B000030E048ED51E4C701B6010F9477506DA362
:101B10007EA38FA398A709C0B301A201CE01859629
:101B20000E94BB8B882309F472C2E090710BF09085
:101B3000720B0091730B1091740B80903F02909088
:101B40004002A0904102B090420280E090E0A8ECF8
:101B5000B2E480933F0290934002A0934102B0937D
:101B6000420219821A821B821C826DA17EA18FA162
:101B700098A59E012F5F3F4F6901A30192010E942A
:101B8000C9D581E00E94A38C8111C9C180919813AD
:101B900082FF11C020914B0B30914C0B40914D0BAB
:101BA00050914E0B60E070E080E490EC0F94765022
:101BB0002B013C0106C0412C512C90E2692E91EC86
:101BC000792EC0904B0BD0904C0BE0904D0BF090C9
:101BD0004E0B20E030E0A901C701B6010F948D49FA
:101BE00087FF0BC0A701960160E070E080E791E4F9
:101BF0000F9476506B017C0106C0C12CD12C80E77C
:101C0000E82E81E4F82EA70196016091710B709186
